:0300000002003AC1
:10003A0075A800C293759074751E7475B0FF75D05B
:0F004A000075150075817690BEF4C082C08332B8
:101F4A003C4E414B3E003C41434B3E002530326201
:101F5A007525303262752530326275002573000CA2
:101F6A0025730A000C25730A01000C436F6E747204
:101F7A0061737420000C25730A2573000C25730005
:10204D00603F04DBFF1CAFFF1CC7FF1CE2FF1CFD44
:10205D00FF1D18FF1E8BFF1E8BFF1E8BFF1E8BFFA0
:10206D001D69FF1E0AFF1DC1FF1E8BFF1D95FF1D64
:10207D0033FF1E8BFF1E8BFF1E92FF1EF1FF1E36C0
:10208D00FF1D4E6081045AFF0FC1FF100BFF108121
:10209D00FF1110FF1168FF11D6FF0006FF0006FFAC
:1020AD000006FF13DCFF142DFF1897FF0006FF1429
:1020BD007EFF1221FF14CFFF1520FF1571FF17278B
:1020CD00FF18E8FF12A0FF1959FF19F3FF1A40FF7F
:1020DD001A8DFF1ADAFF0006FF19A6FF12FEFF1375
:1020ED004DFF1394FF1850FF0006FF18BFFF191086
:1020FD00FF1984FF1A1EFF19D1FF1A6BFF1AB8FFC3
:08210D001B05FF1B27FF000763
:100100009008FCE0FF12F38D40030201E69008FD29
:10011000E0FF12F38D40030201E69008F2E0FF12C7
:10012000F38D40030201E69008F3E0FF12F38D40E7
:10013000030201E690066FE0FF12F38D4003020117
:10014000E6900670E0FF12F38D40030201E6900A8C
:100150008EE0FF12F38D40030201E6900A8FE0FF6C
:1001600012F38D40030201E69006B3E0FF12F38D17
:1001700050749006B4E0FF12F38D506A900E23E0A5
:10018000FF12F38D5060900E24E0FF12F38D505655
:100190007B017A0879FC12F72490051BEFF07B01B4
:1001A0007A0879F212F72490051AEFF07B017A06AB
:1001B000796F12F724900458EFF07B017A0A798E58
:1001C00012F72490051DEFF07B017A0679B312F740
:1001D00024900459EFF07B017A0E792312F72490D2
:1001E000044DEFF080037F002290051BE0F9C394DB
:1001F00000500302028390051AE0FFD394005003DD
:10020000020283EFD3940C4003020283900458E06F
:10021000FED39400406DEED3941F506790051DE00F
:10022000FDC39400405DEDD394175057900459E0FE
:10023000FCC39400404DECD3943B504790044DE0F8
:10024000FBC39400403DEBD3943B503790044FEFF9
:10025000F0A3EEF0900452EDF090044EE9F090041B
:1002600053ECF0A3EBF0E4900451F0788F7C127D16
:10027000017B017A04794EFE7F0812E52C12CA0632
:060280007F01227F002235
:100286009012AAE09008FCF09012ABE09008FDF006
:10029600E4A3F09012A7E09008F2F09012A8E09084
:1002A60008F3F0E4A3F09012A4E090066FF0901229
:1002B600A5E0900670F0E4A3F09012AEE0900A8EEE
:1002C600F09012AFE0900A8FF0E4A3F09012B1E044
:1002D6009006B3F09012B2E09006B4F0E4A3F0906A
:1002E60012B4E0900E23F09012B5E0900E24F0E4E4
:1002F600A3F0EDF4707490056CE09008FCF09005A6
:100306006DE09008FDF0E4A3F090056EE09008F231
:10031600F090056FE09008F3F0E4A3F0900570E02C
:1003260090066FF0900571E0900670F0E4A3F090EF
:100336000572E0900A8EF0900573E0900A8FF0E463
:10034600A3F0900574E09006B3F0900575E0900672
:10035600B4F0E4A3F0900576E0900E23F0900577D4
:10036600E0900E24F0E4A3F0801890056CE012E50E
:100376009B90056DE090000112E5AD900002E4123D
:10038600E5AD120100EF701078F67C0C7D017BFF65
:100396007A1F794A12EA4F2278F67C0C7D017BFFA0
:0803A6007A1F795012EA4F2280
:1003AE007F0712B27A90096AE0B40211A3E0900EB0
:1003BE0023F090096CE0900E24F0E4A3F090095B1A
:1003CE00E0B40211A3E09006B3F090095DE0900650
:1003DE00B4F0E4A3F090095EE0B40211A3E0900A39
:1003EE008EF0900960E0900A8FF0E4A3F09009611E
:1003FE00E0B40211A3E090066FF0900963E090065E
:10040E0070F0E4A3F0900964E0B40211A3E0900848
:10041E00F2F0900966E09008F3F0E4A3F09009671B
:10042E00E0B40211A3E09008FCF0900969E0900896
:10043E00FDF0E4A3F0120100EF60067F0712B2197F
:0B044E00227F097D0A7B0312C33122CC
:1000D700740B2FF582E43409F583EDF0740C2FF5DA
:0900E70082E43409F583EBF022F8
:0E00F000EF2B240BF582E43409F583EDF022AA
:10045900EF2B240BF582E43409F583EDF01203AE9A
:010469002270
:10046A007F0D7D02E4FB1200F07D390B1200F00BC8
:04047A001200F0225A
:10047E007F17E4FDFB1200F07D300B1200F00B1223
:03048E0000F02259
:100491007F4B7D02E4FB1200F07D300B1200F00B6C
:0404A1001200F02233
:1004A5007F5C7D02E4FB1204597F5C7D397B011280
:0C04B50004597F5C7D357B021204592243
:1004C100900445EFF0E0FF7D02E4FB120459900433
:1004D10045E0FF7D307B01120459900445E0FF7D2A
:0704E100307B0212045922D6
:1004E800900446EFF0E0FF7D02E4FB12045990040B
:1004F80046E0FF7D307B01120459900446E0FF7D01
:07050800317B0212045922AD
:10050F00900447EFF0AF05AD0312D518900447E004
:10051F00240CF582E43409F583E0FF12D6AE900483
:10052F0047E0240DF582E43409F583E0FF12D6AEDF
:01053F002299
:0100060022D7
:100540009008FFE024A6F582E4340AF583E0645ABB
:1005500060030205F2900567E024A6F582E4340A00
:10056000F583E0B43F2F7BFF7A1F79569016701207
:10057000E72090129AE0901673F090129BE090168C
:1005800074F090129CE0901675F07B017A0C79F66D
:1005900012ED9B805A900567E0FF24A6F9E4340A27
:1005A000FA7B019016C812E720EF2401FFE433FE26
:1005B000900A91E0C39F9016CCF0E49E9016CBF089
:1005C0007A05796C12F599900567E004FF900A911D
:1005D000E0C39FFFBF0C0D7B017A0879FC7DFF1201
:1005E0000286800B7B017A0879FCE4FD1202867F8B
:1005F00001229008FFE024A6F582E4340AF583E0A6
:1006000064577071900567E024A6F582E4340AF51A
:1006100083E0B43F2F7BFF7A1F795690167012E764
:100620002090129EE0901673F090129FE090167446
:10063000F09012A0E0901675F07B017A0C79F6121A
:10064000ED9B802E900567E024A6F9E4340AFA7B3E
:10065000019016C812E7209016CBE4F0A37402F0C4
:100660007A05796C12F5997B017A0A798EE4FD128C
:1006700002867F01229008FFE024A6F582E4340A76
:10068000F583E064597031900567E024A6F9E434FD
:100690000AFA7B019016C812E7209016CBE4F0A36B
:1006A0007402F07A05796C12F5997B017A0879F277
:1006B000E4FD1202867F01229008FFE024A6F58265
:1006C000E4340AF583E064587031900567E024A6AD
:1006D000F9E4340AFA7B019016C812E7209016CB91
:1006E000E4F0A37402F07A05796C12F5997B017A33
:1006F00006796FE4FD1202867F01229008FFE02454
:10070000A6F582E4340AF583E064567031900567FB
:10071000E024A6F9E4340AFA7B019016C812E72017
:100720009016CBE4F0A37402F07A05796C12F59977
:100730007B017A0679B3E4FD1202867F01229008DC
:10074000FFE024A6F582E4340AF583E0645C7031AE
:10075000900567E024A6F9E4340AFA7B019016C8F4
:1007600012E7209016CBE4F0A37402F07A05796CBE
:1007700012F5997B017A0E7923E4FD1202867F013E
:04078000227F0022B2
:10078400E4FF7D0112D51890086812E717901670DF
:1007940012E7207BFF7A1F796612EDA17F097D0A9B
:0607A4007B0312C33122A9
:1007AA00740C2FF582E43409F583E0900448F07460
:1007BA000D2FF582E43409F583E0900449F0E4A3AF
:0B07CA00F07B017A04794812F724222A
:1007D500EFC39430400FEFD394395009EF24D0C4C0
:1007E50054F0FE8007EF24C9C454F0FEEDC39430E5
:1007F500400DEDD394395007ED24D02EFE8005ED44
:0708050024C92EFEAF0622FC
:10080C00900AA6E0FF900935E0FEEF6E600C9009AF
:10081C0037E0FEEF6E60030208C7900E4AE07003EB
:10082C000208C77B017A0A79A612F601EF640170FF
:10083C00030208C790091EE0FFB4011F900922E0D3
:10084C00B402189005677405F09008FF14F07B0152
:10085C007A097907900CEE12E72022EFB401209070
:10086C000922E0640260189005677404F09008FF98
:10087C0014F07B017A097985900CEE12E72022EFB7
:10088C006401601F900922E0B4021890056774049B
:10089C00F09008FF14F07B017A097989900CEE1224
:1008AC00E720229005677403F09008FF14F07B0199
:1008BC007A097991900CEE12E7202290091EE0FF44
:1008CC0064017032900922E0B4022B900567740425
:1008DC00F09008FF14F0900E4AE0600D7B017A094D
:1008EC007999900CEE12E720227B017A0979AB9072
:1008FC000CEE12E72022EF64017033900922E064C1
:10090C0002602B9005677403F09008FF14F0900EB2
:10091C004AE0600D7B017A09799D900CEE12E7207C
:10092C00227B017A0979AF900CEE12E72022EF645A
:10093C00016032900922E0B4022B9005677403F039
:10094C009008FF14F0900E4AE0600D7B017A097953
:10095C00A1900CEE12E720227B017A0E7911900CFB
:10096C00EE12E720229005677402F09008FF14F055
:10097C00900E4AE0600D7B017A0979A5900CEE127D
:10098C00E720227B017A0E7917900CEE12E72022D9
:10099C009006DFE0FF9006DDE0FD9006DAE0FB124A
:1009AC00D2BF7F4B1207AA900E1EEFF0700374217A
:1009BC00F07F171207AA900E1CEFF070049009221A
:1009CC00F090091EE0B40106A3E09008F5F0900940
:1009DC0020E0B40112900931E09006DEF09009217C
:1009EC00E0900568F08008900931E0900568F012FD
:0309FC00080C22C2
:1009FF007B017A0979E99016C812E7209016CBE4AB
:100A0F00F0A37402F07A05796412F599E490056603
:100A1F00F07B017A05796412F72490044BEFF07B99
:100A2F00017A0979EB9016C812E7209016CBE4F003
:100A3F00A37402F07A05796412F599E4900566F0D3
:100A4F007B017A05796412F724900456EFF0900435
:100A5F004BE0FF7003020F66900457E090044CF0D8
:100A6F00EF1412E7B20AD2000AD2010AD2020AD256
:100A7F00030AD2040AD2050AE7090B3E0A0B950BAB
:100A8F000BC80D0AD20E0C170F0C66100CB5110CFB
:100A9F00EA120D09130AD2140D3C150D71160DA68D
:100AAF00170DDB180E10190E431B0AD21C0AD21D8C
:100ABF000AD21E0E781F0EB73B0F123E0F5844007E
:100ACF00000F62EF75F003A42457F582E43404F5A8
:100ADF008312E71712E7D82290080212E717901631
:100AEF007012E7207BFF7A1F796912EDA190044BFA
:100AFF00E014FF900457F090044CE0B507087F1303
:100B0F00E4FDFB1200D790091EE064016003020FA1
:100B1F00C0A3E075F0039006E512E70B12E71790FC
:100B2F00167012E7207BFF7A1F796612EDA12290D3
:100B3F00080512E71790167012E7207BFF7A1F79CE
:100B4F006912EDA190044BE014FF900457F090044C
:100B5F004CE0B507087F15E4FDFB1200D790092084
:100B6F00E064016003020FC0A3E075F0039006E597
:100B7F0012E70B12E71790167012E7207BFF7A1F10
:100B8F00796612EDA1229007DB12E717901670120B
:100B9F00E7207BFF7A1F796E12EDA190044BE014D2
:100BAF00FF900457F090044CE0B5070312047E7FCA
:100BBF0017E4FD7B0112050F229007E112E7179052
:100BCF00167012E7207BFF7A1F796912EDA190044E
:100BDF004BE014FF900457F090044CE0B507097FE9
:100BEF00257D017B0D1200D7900931E075F0039040
:100BFF0006E512E70B12E71790167012E7207BFF3E
:100C0F007A1F796612EDA1229007E712E717901667
:010C1F007064
:100C200012E7207BFF7A1F796912EDA190044BE057
:100C300014FF900457F090044CE0B507097F297D1C
:100C4000017B061200D7900935E075F0039006E5A8
:100C500012E70B12E71790167012E7207BFF7A1F3E
:100C6000796612EDA1229007EA12E717901670122A
:100C7000E7207BFF7A1F796912EDA190044BE01405
:100C8000FF900457F090044CE0B507097F2B7D01DD
:100C90007B151200D7900937E075F0039006E51236
:100CA000E70B12E71790167012E7207BFF7A1F7987
:100CB0006612EDA1229007D812E71790167012E77E
:100CC000207BFF7A1F796912EDA190044BE014FF9D
:100CD000900457F090044CE0B507031289EFD24C12
:100CE000900F0E7401F01289C5229007CC12E717FD
:100CF00090167012E7207BFF7A1F796912EDA190A0
:100D0000044BE014900457F0229007ED12E717907F
:100D1000167012E7207BFF7A1F796E12EDA1900406
:100D20004BE014FF900457F090044CE0B507031219
:100D300004917F4BE4FD7B0112050F2290081412F1
:100D4000E71790167012E7207BFF7A1F796E12ED7D
:100D5000A190044BE014FF900457F090044CE0B5D0
:100D600007057F501204C17F507D087B0112050FDB
:100D70002290081712E71790167012E7207BFF7A6F
:100D80001F796E12EDA190044BE014FF900457F010
:100D900090044CE0B507057F531204C17F537D06D4
:100DA0007B0112050F2290082F12E7179016701280
:100DB000E7207BFF7A1F796E12EDA190044BE014BF
:100DC000FF900457F090044CE0B507057F561204DD
:100DD000E87F567D057B0112050F2290083212E74D
:100DE0001790167012E7207BFF7A1F796E12EDA123
:100DF00090044BE014FF900457F090044CE0B507CA
:100E0000057F591204E87F597D077B0112050F22E7
:100E100090083512E71790167012E7207BFF7A1FB3
:100E2000796E12EDA190044BE014FF900457F090FE
:100E3000044CE0B507031204A57F5C7D077B01121B
:100E4000050F2290085F12E71790167012E7207BBB
:100E5000FF7A1F796E12EDA190044BE014FF90040D
:0E0E600057F090044CE0B507057F5F1204C107
:100E6E007F5F7D087B0112050F2290084112E71764
:100E7E0090167012E7207BFF7A1F796E12EDA1900B
:100E8E00044BE014FF900457F090044CE0B50709B2
:100E9E007F687D017B301200D7E4FF7D0112D518EB
:100EAE00900974E0FF12D6AE227BFF7A1F7974127E
:100EBE00EDA1900456E070207F09FD12D5187F2B0E
:100ECE0012D6AE900E33E0C3949F5003E004F09020
:100EDE000E33E0FF12D27622900456E0B401217F49
:100EEE0009E4FD12D5187F2D12D6AE900E33E0D345
:100EFE0094804003E014F0900E33E0FF12D276227D
:100F0E00120784229008A712E71790167012E72096
:100F1E00900456E075F00390075A12E70B12E7178C
:100F2E0090167312E7207BFF7A1F797F12EDA19046
:100F3E000456E0FF7005900E30F022EFB4010790DA
:100F4E000E3074FFF022120784229004D512E71798
:100F5E0012E7D822120784229009EBE0FFA3E0FDEE
:100F6E001207D5900456EFF0C3945B503CA3E0FFFC
:100F7E0024F2602B24FA602724FA6023241324EB36
:100F8E00500824FD24F650028015EF75F003A424BA
:100F9E005AF582E43404F58312E71712E7D8227F5C
:100FAE00097D0A7B0312C331227F097D0A7B03125E
:030FBE00C331221A
:100FC10090066EE0702B90082012E71790167012B1
:100FD100E720900456E075F00390081A12E70B120F
:100FE100E71790167312E7207BFF7A1F797F12EDC6
:100FF100A1900456E0D39401400F90066EE0700377
:0A100100120784900E2774FFF022FE
:0100070022D6
:10100B0090066EE0702B9007B712E71790167012D0
:10101B00E720900456E075F00390082312E70B12BB
:10102B00E71790167312E7207BFF7A1F797F12ED7B
:10103B00A1900456E024FE601114601E2403702658
:10104B00E490056AF0900CD9F02290056A74FFF0D9
:10105B00E4900E2AF0900CD9F022900CD974FFF08A
:10106B00E4900E35F02290066EE070031207849028
:06107B000E2774FFF022B5
:1010810090066EE0702B9007C312E717901670124E
:10109100E720900456E075F00390074512E70B1224
:1010A100E71790167312E7207BFF7A1F797F12ED05
:1010B100A1900456E0FF70059006DFF022EFB40125
:1010C100079006DF7401F022EFB402079006DF7487
:1010D10002F022EFB403079006DF7403F022EFB4AD
:1010E10004079006DF7404F022EFB405079006DFD1
:1010F1007405F022EFB406079006DF7406F0229023
:0F110100066EE07003120784900E2774FFF02231
:1011100090066EE0702B9007C912E71790167012B8
:10112000E720900456E075F00390076C12E70B126D
:10113000E71790167312E7207BFF7A1F797F12ED75
:10114000A1900456E0FF70059006DAF022EFB4019A
:10115000079006DA7401F02290066EE07003120721
:0811600084900E2774FFF022B9
:1011680090066EE0702B9007C612E7179016701263
:10117800E720900456E075F00390076012E70B1221
:10118800E71790167312E7207BFF7A1F797F12ED1D
:10119800A1900456E0FF70059006DDF022EFB4013F
:1011A800079006DD7401F022EFB402079006DD74A3
:1011B80002F022EFB403079006DD7403F0229006D4
:0E11C8006EE07003120784900E2774FFF02271
:1011D6009007CF12E71790167012E720900456E09A
:1011E60075F00390075A12E70B12E7179016731261
:1011F600E7207BFF7A1F797F12EDA1900456E0FF6E
:101206007005900E2AF022EFB4010CE490056AF006
:0B121600900E2A74FFF02212078422C1
:1012210090066EE0702B9007E412E717901670128B
:10123100E720900456E075F0039007BA12E70B120D
:10124100E71790167312E7207BFF7A1F797F12ED63
:10125100A1900456E0FF700D900E4AF0900E0FF031
:101261009008D4F022EFB40110900E4A74FFF09070
:1012710008D4F0E4900E0FF022EFB40212900E4A5F
:1012810074FFF0E49008D4F0900E0F74FFF02290F8
:0F129100066EE07003120784900E2774FFF022A0
:1012A00090066EE070309007F012E71790167012FB
:1012B000E720900456E0FFC374289F75F003900662
:1012C000E512E70B12E71790167312E7207BFF7AFF
:1012D0001F797F12EDA1900456E0FF7007900E2653
:1012E00074FFF022EFB40106E4900E26F02290067F
:0E12F0006EE07003120784900E2774FFF02248
:1012FE0090083812E71790167012E720900456E007
:10130E0075F00390084412E70B12E717901673124C
:10131E00E7207BFF7A1F797F12EDA1900456E0FF44
:10132E007009900CD9F0900E35F022EFB4010C90AC
:0F133E000E3574FFF0E4900CD9F02212078422D0
:10134D0090083B12E71790167012E720900456E0B4
:10135D0075F00390084A12E70B12E71790167312F7
:10136D00E7207BFF7A1F797F12EDA1900456E0FFF5
:10137D00700790056074FFF022EFB40106E490054C
:07138D0060F0221207842228
:1013940090083E12E71790167012E720900456E06A
:1013A40075F00390085012E70B12E71790167312AA
:1013B400E7207BFF7A1F797F12EDA1900456E0FFAE
:1013C40070079006AB7478F022EFB401079006AB77
:0813D4007414F02212078422B8
:1013DC00900456E0FF7E00C3EE94004009D3EF94D6
:1013EC001FEE9400400A7F097D0A7B0312C3312251
:1013FC007F137D01900456E0FB1200D7E4FF12D559
:10140C0018900456E075F0039006E512E70B12E70E
:10141C001790167012E7207BFF7A1F796612EDA1E8
:01142C00229D
:10142D00900456E0FF7E00C3EE94004009D3EF9484
:10143D001FEE9400400A7F097D0A7B0312C33122FF
:10144D007F157D01900456E0FB1200D7E4FF12D505
:10145D0018900456E075F0039006E512E70B12E7BD
:10146D001790167012E7207BFF7A1F796612EDA197
:01147D00224C
:10147E00900456E0FF7E00C3EE94004009D3EF9433
:10148E001FEE9400400A7F097D0A7B0312C33122AE
:10149E007F257D01900456E0FB1200D7E4FF12D5A4
:1014AE0018900456E075F0039006E512E70B12E76C
:1014BE001790167012E7207BFF7A1F796612EDA146
:0114CE0022FB
:1014CF00900456E0FF7E00C3EE94004009D3EF94E2
:1014DF001FEE9400400A7F097D0A7B0312C331225D
:1014EF007F297D01900456E0FB1200D7E4FF12D54F
:1014FF0018900456E075F0039006E512E70B12E71B
:10150F001790167012E7207BFF7A1F796612EDA1F4
:01151F0022A9
:10152000900456E0FF7E00C3EE94004009D3EF9490
:101530001FEE9400400A7F097D0A7B0312C331220B
:101540007F2B7D01900456E0FB1200D7E4FF12D5FB
:1015500018900456E075F0039006E512E70B12E7C9
:101560001790167012E7207BFF7A1F796612EDA1A3
:011570002258
:1015710090066EE0702B9007D812E7179016701244
:10158100E720900456E075F0039006E512E70B1290
:10159100E71790167312E7207BFF7A1F797F12ED10
:1015A100A1900456E012E7B215E63015F23115FEAE
:1015B10032161533162134163835164F361666375E
:1015C100167238167E3916953A16AC3B16C33C1680
:1015D100CF3E16DB3F16E74016F34216FF44170BCA
:1015E1004500001717D24C900F0E7401F01289C5F7
:1015F10022D24C900F0E7405F01289C522D24C9064
:101601000F0E740FF01289C5D24D900F0F740FF0A9
:101611001289DA22D24C900F0E7409F01289C52278
:10162100D24C900F0E7410F01289C5D24D900F0F4D
:10163100740FF01289DA22D24C900F0E7414F0124A
:1016410089C5D24D900F0F740FF01289DA22D24C56
:10165100900F0E7415F01289C5D24D900F0F740FB3
:10166100F01289DA22D24C900F0E7402F01289C561
:1016710022D24C900F0E7403F01289C522D24C90E5
:101681000F0E7413F01289C5D24D900F0F740FF025
:101691001289DA22D24C900F0E7412F01289C5D23F
:1016A1004D900F0F740FF01289DA22D24C900F0E69
:1016B1007411F01289C5D24D900F0F740FF0128979
:1016C100DA22D24C900F0E740AF01289C522D24C44
:1016D100900F0E740DF01289C522D24C900F0E742A
:1016E10007F01289C522D24C900F0E7408F01289AE
:1016F100C522D24C900F0E740CF01289C522D24C27
:10170100900F0E740EF01289C522D24C900F0E74F8
:1017110006F01289C52290066EE0700312078490CC
:061721000E2774FFF02208
:1017270090066EE070159007CC12E71790167012AE
:10173700E7207BFF7A1F798612EDA1900456E024FB
:10174700CF606B1470030217E224FE700302180FB8
:101757002404600302183C900E54E0602AE4F090E1
:10176700066EE0600302184F90086B12E717901699
:101777007012E7207BFF7A1F796612EDA17F097D42
:101787000A7B0312C3312290066EE070159007752D
:1017970012E71790167012E7207BFF7A1F796612FF
:1017A700EDA1D24D900F0F7401F01289DA22900645
:1017B7006EE0701590077812E71790167012E72001
:1017C7007BFF7A1F796612EDA1D24D900F0F74053A
:1017D700F01289DA900E5474FFF02290066EE070D2
:1017E700159007A512E71790167012E7207BFF7A6E
:1017F7001F796612EDA1D24D900F0F7408F0128970
:10180700DA900E5474FFF02290066EE07015900780
:10181700AB12E71790167012E7207BFF7A1F7966E5
:1018270012EDA1D24D900F0F740CF01289DA900EC1
:101837005474FFF02290066EE07003120784900E36
:091847002774FFF0900E54F0220A
:10185000E4FF7D0112D518900456E0FFC394304098
:1018600006EFD39439401B7F097D0A7B0312C331F5
:101870007F687D017B301200D7900974E0FF12D69B
:10188000AE227F687D01900456E0FB1200D79004E1
:0718900056E0FF12D6AE2264
:101897007F177D01E4FB1200F0900456E0FD0B1268
:1018A70000F09004577421F0E4FF7D0112D51890E1
:0818B7000456E0FF12D6AE2238
:1018BF007F177D02E4FB1200F0900456E0FD7B02DF
:1018CF001200F0900457740BF07F017D0112D518B0
:0918DF00900456E0FF12D6AE227F
:1018E8007F4B7D01E4FB1200F0900456E0FD0B12E3
:1018F80000F09004577422F0E4FF7D0112D518908F
:081908000456E0FF12D6AE22E6
:101910007F4B7D02E4FB1200F0900456E0FD7B0259
:101920001200F09004577413F07F017D0112D51856
:10193000900456E0FF12D6AE7F4B1207AAEFD39465
:101940002040157F097D0A7B0312C3311204917F69
:091950004BE4FD7B0112050F229E
:101959007F507D02E4FB1204597F50900456E0FD4C
:101969007B011204599004577423F07F087D0112FA
:0B197900D518900456E0FF12D6AE22F5
:101984007F50900456E0FD7B021204599004577472
:1019940015F07F097D0112D518900456E0FF12D688
:0219A400AE2271
:1019A6007F5F7D02E4FB1204597F5F900456E0FDE1
:1019B6007B011204599004577425F07F087D0112AB
:0B19C600D518900456E0FF12D6AE22A8
:1019D1007F5F900456E0FD7B021204599004577416
:1019E1001BF07F097D0112D518900456E0FF12D635
:0219F100AE2224
:1019F3007F537D02E4FB1204597F53900456E0FDAC
:101A03007B011204599004577424F07F067D011260
:0B1A1300D518900456E0FF12D6AE225A
:101A1E007F53900456E0FD7B0212045990045774D4
:101A2E0016F07F077D0112D518900456E0FF12D6EE
:021A3E00AE22D6
:101A40007F567D02E4FB1204597F56900456E0FD58
:101A50007B011204599004577426F07F057D011212
:0B1A6000D518900456E0FF12D6AE220D
:101A6B007F56900456E0FD7B021204599004577484
:101A7B0017F07F067D0112D518900456E0FF12D6A1
:021A8B00AE2289
:101A8D007F597D02E4FB1204597F59900456E0FD05
:101A9D007B011204599004577427F07F077D0112C2
:0B1AAD00D518900456E0FF12D6AE22C0
:101AB8007F59900456E0FD7B021204599004577434
:101AC80018F07F087D0112D518900456E0FF12D651
:021AD800AE223C
:101ADA007F5C7D02E4FB1204597F5C900456E0FDB2
:101AEA007B011204599004577428F07F077D011274
:0B1AFA00D518900456E0FF12D6AE2273
:101B05007F5C900456E0FD7B0212045990045774E3
:101B150019F07F087D0112D518900456E0FF12D602
:021B2500AE22EE
:101B2700900456E024CEF090066EE0702B9008AD3E
:101B370012E71790167012E720900456E075F0032D
:101B47009008B012E70B12E71790167312E7207B85
:101B5700FF7A1F797F12EDA1900456E014601014EC
:101B6700601A1460242403702DE49006E0F022909C
:101B770006E074FFF09006E47408F0229006E07423
:101B8700FFF09006E47410F0229006E074FFF090E6
:101B970006E47420F02290066EE07003120784902A
:061BA7000E2774FFF0227E
:101BAD00900E337485F0FF12D27612046A7F107D89
:101BBD00017B301200D77F13E41DFB1200D77F1578
:101BCD00E41200D712047E7F257D017B0D1200D714
:101BDD007F297B061200D77F2B7B151200D71204AD
:101BED00917F687D017B301200D7900931E090051F
:101BFD0068F0E49006E0F0900E2674FFF09005601A
:101C0D00F0900E29F0900CF4F0900A7FF090066D94
:101C1D00F0E49008D4F090056AF0900E0FF0900E5D
:101C2D0035F0900E2AF0900CD9F09006A7F0900E9A
:101C3D0021F0900E31F0900E4AF0900E1FF0900AA8
:101C4D0092F090055BF0900672F09006DF7405F04F
:101C5D00E49006DAF09006DD7402F0900E1E742109
:101C6D00F09005697401F0E4900CD8F09006AB7417
:101C7D0014F07F050DE4FB12D2BF9005677402F0DE
:101C8D009008FF14F090098D7480F0A3F0E4A3F098
:101C9D001289EFD24C900F0E7401F01289C5120902
:021CAD009C2277
:101CAF00900567E024A6F582E4340AF583E024D09A
:081CBF00900456F0120FC1223F
:101CC700900567E024A6F582E4340AF583E024D082
:0B1CD700900456F012100B12099C2222
:101CE200900567E024A6F582E4340AF583E024D067
:0B1CF200900456F012108112099C2291
:101CFD00900567E024A6F582E4340AF583E024D04C
:0B1D0D00900456F012111012099C22E5
:101D1800900567E024A6F582E4340AF583E024D030
:0B1D2800900456F012116812099C2272
:101D3300900567E024A6F582E4340AF583E024D015
:0B1D4300900456F012122112099C229D
:101D4E00900567E024A6F582E4340AF583E024D0FA
:0B1D5E00900456F01212A012099C2203
:101D6900900567E024A6F582E4340AF583E0FBC315
:101D790094004011EBD3941F500B7F137D01120087
:0C1D8900D712099C22900E2774FFF02254
:101D9500900567E024A6F582E4340AF583E0FBC3E9
:101DA50094004011EBD3941F500B7F257D01120049
:0C1DB500D712099C22900E2774FFF02228
:101DC100900567E0FF24A6F582E4340AF583E0FE7E
:101DD100C39430402DEED39439502774A72FF58248
:101DE100E4340AF583E0FFC394304016EFD394390D
:101DF10050109009227402F0A3EEF0A3EFF0120943
:091E01009C22900E2774FFF022D0
:101E0A00900567E024A6F582E4340AF583E0FBC373
:101E1A0094004011EBD3941F500B7F157D011200E3
:0C1E2A00D712099C22900E2774FFF022B2
:101E3600900567E0FF24A6F582E4340AF583E0FE08
:101E4600C394304039EED39439503374A72FF582BA
:101E5600E4340AF583E0FFC394304022EFD394398B
:101E6600501C9009567402F0A3EEF0A3EFF07F4BDE
:101E76001207AA900E1EEFF0700A7421F022900E3F
:051E86002774FFF022AB
:071E8B00900E2774FFF02206
:101E9200900567E024A6F582E4340AF583E0FFC3E7
:101EA200941B4044EFD3947F503EEFB41B0512893C
:101EB200EF8029900567E024A6F582E4340AF583D1
:101EC200E0FF641B6016900E27E07010900456EF3E
:101ED200F0121571900567E004F080D7D24C900F94
:0F1EE2000E7401F01289C522900E2774FFF022B2
:101EF100900567E024A6F582E4340AF583E0FFC388
:101F0100941B403EEFD3947F5038EFB41B051289E8
:101F1100EF8023900567E024A6F582E4340AF58377
:101F2100E0FF641B6010900456EFF0121727900534
:101F310067E004F080DDD24C900F0E7401F012893D
:091F4100C522900E2774FFF02266
:106993003C6E756C3E2020202020202020202020CB
:1069A300003C736F683E20202020202020202020E0
:1069B30020003C7374783E202020202020202020BB
:1069C3002020003C6574783E2020202020202020B9
:1069D300202020003C656F743E20202020202020B2
:1069E30020202020003C656E713E202020202020A6
:1069F3002020202020003C61636B3E2020202020AB
:106A0300202020202020003C62656C3E2020202096
:106A130020202020202020003C62733E20202020C4
:106A23002020202020202020003C68743E202020AD
:106A3300202020202020202020003C6C663E2020A7
:106A430020202020202020202020003C76743E207F
:106A53002020202020202020202020003C66663E8D
:106A6300202020202020202020202020003C637292
:106A73003E202020202020202020202020003C73A6
:106A83006F3E202020202020202020202020003C9A
:106A930073693E2020202020202020202020200059
:106AA3003C646C653E2020202020202020202020D4
:106AB300003C6463313E2020202020202020202021
:106AC30020003C6463323E20202020202020202010
:106AD3002020003C6463333E2020202020202020FF
:106AE300202020003C6463343E20202020202020EE
:106AF30020202020003C6E616B3E2020202020209F
:106B03002020202020003C73796E3E20202020206E
:106B1300202020202020003C6574623E202020207D
:106B230020202020202020003C63616E3E20202076
:106B33002020202020202020003C656D3E202020A6
:106B4300202020202020202020003C7375623E203E
:106B530020202020202020202020003C6573633E3D
:106B63002020202020202020202020003C66733E6F
:106B7300202020202020202020202020003C67737C
:106B83003E202020202020202020202020003C7296
:106B9300733E202020202020202020202020003C85
:106BA30075733E202020202020202020202020003C
:106BB300333030202020202020202020202020209F
:106BC30000363030202020202020202020202020AC
:106BD300200031323030202020202020202020208F
:106BE300202000323430302020202020202020207C
:106BF3002020200034383030202020202020202066
:106C03002020202000393630302020202020202052
:106C13002020202020003139323030202020202035
:106C23002020202020200064697361626C6520208D
:106C33002020202020202000656E61626C652020CA
:106C43002020202020202020006F6464202020208A
:106C5300202020202020202020006576656E202023
:106C630020202020202020202020006D61726B2016
:106C7300202020202020202020202000737061630A
:106C830065202020202020202020202000372020C5
:106C930020202020202020202020202020003820F9
:106CA3002020202020202020202020202020006EB3
:106CB3006F6E65202020202020202020202020000F
:106CC3005374642033206F66203920202020202035
:106CD30000496E742032206F66203520202020204A
:106CE300200045414E2F55504320202020202020B6
:106CF3002020004D6F6E61726368202020202020C9
:106D030020202000555043206F6E6C7920202020D6
:106D130020202020005550432F45414E202B203268
:106D23002020202020005550432F45414E202B206A
:106D3300352020202020004578742033206F6620E2
:106D43003920202020202000506861726D61636526
:106D53007574696320202020005550432D45206F12
:106D63006E6C792020202020200045414E2D3820B4
:066D73006F6E6C79202018
:106D7900202020200045414E2D3133206F6E6C7943
:106D890020202020200050616B6F2020202020200F
:106D99002020202020200000436F646520313238F4
:106DA900202020202020202000496E642032206FDE
:106DB900662035202020202020004D6174726978DA
:106DC90020322F352020202020200044656C74615A
:106DD900412049424D202020202020004D534920A8
:106DE900506C65737365792020202020005A656CEA
:106DF9006C77656765722020202020202000436F72
:106E090064652039332020202020202020200049BB
:106E1900544620313420202020202020202020000A
:106E2900496E746572666163653A202020202020CE
:106E39000044697361626C65202020202020202095
:106E490020004C7263632020202020202020202055
:106E590020200043686B73756D2032353620202061
:106E6900202020004261756420526174653A202017
:106E790020202020005061726974793A2020202056
:106E89002020202020004461746120426974733AF3
:106E99002020202020200043686B20446967697402
:106EA9003A2020202020200A00586F6E20586F6653
:106EB900663A202020202020200043686172446522
:106EC9006C61793A2020202020200A6D732E20350C
:106ED900302A00486F737420542E3A202020202035
:106EE9002020200A6D732E2035302A0042617263FA
:106EF9006F6465547970653A2020202000537461CD
:106F0900742E416464723A2020202020200A005304
:106F1900746172744F665478743A20202020200AD4
:106F290000456E644F66546578743A20202020200D
:106F39002000426C6B20436865636B3A2020202057
:106F490020200041636B20547970653A202020206D
:106F5900202020004E616B20547970653A20202052
:106F69002020202000436F646553697A6543686B6C
:106F79003A202020200A00426565703A202020200E
:106F890020202020202020000A202020202020202E
:106F9900202020202020202020002020205365614F
:106FA900726368696E67212020200A2020205761BA
:106FB9006974506C656173652020200044656C65B7
:106FC900746520436F64653A202020200A00202040
:106FD900204D656D6F727946756C6C2020200020FC
:106FE90020204E6F7420466F756E6421202020008A
:106FF90053746172744F66426C6B3A2020202020D2
:1070090000456E644F66426C6B3A20202020202098
:1070190020005761726E696E673A20202020202077
:1070290020200A0053656172636820436F64653AE2
:10703900202020200A002020202020762E302F72A8
:107049002E302020202000202020436F6465204618
:107059006F756E6420202000436C6F636B0A4D6965
:107069006E7574653A00436C6F636B0A486F75728D
:107079003A0046756C6C204475706C657820202048
:1070890020200048616C66204475706C657820206A
:10709900202020005258204D6F64653A202020207E
:1070A900202020200052532D32333243202020202B
:1070B90020202020200052532D343232202020203D
:1070C9002020202020200052532D34383520202024
:1070D9002020202020202000456176657364726F8E
:1070E900702020202020202000446174650A44611A
:1070F900793A00446174650A4D6F6E74683A0044C8
:107109006174650A596561723A20200050726F7482
:107119006F636F6C3A2020202020202000545820D3
:107129004D6F64653A2020202020202020004D61E9
:10713900726B2054696D653A202020202020004E72
:10714900756C6C20436861723A2020202020200A47
:0671590000537464205095
:10715F00726F742E20202020202020005370656332
:10716F002E50726F742E2020202020200054582083
:10717F00496D6D65642E202020202020200054585A
:10718F002053657475702020202020202020003689
:10719F002D33207365632E202020202020202000F7
:1071AF00312D31207365632E2020202020202020B8
:1071BF000020202020205363616E6E6572202020F6
:1071CF00200A002020426172636F6465204D656E56
:1071DF0075202000436F64653A00436C6F636B0A40
:1071EF005365636F6E643A005174793A0020202022
:1071FF00202044656661756C74202020200A2020B1
:10720F00202020526573746F726564202020002047
:10721F0020204E6F742056616C696420202020005E
:10722F000C202020536574205570204E6F74202041
:10723F00200A202020205265616461626C65202045
:10724F00202000202020202044656C6574652020BC
:10725F00202020002020204C61737420456E747212
:10726F007920202000202020416C6C20456E747204
:10727F006965732020002020202020204F6E636539
:10728F00202020202020002020202053746420461E
:10729F00696C652020202000202052657374617274
:1072AF0074205265632E202000202020204164642A
:1072BF00205174792E202020200044656661756C62
:1072CF0074004E6F54696D652D4F70743A202020F5
:1072DF002020004E6F446174652D4F70743A20204A
:1072EF00202020005174792E204669656C6420207F
:1072FF00202020200A6C656E6774683A200053695D
:10730F006E676C65204172742E3A20202020004356
:10731F006F6D706374204D6F64653A2020202000DC
:10732F00446973702E44656C61793A2020202020C7
:10733F000053656172636800536561726368204E24
:10734F006578742020202020002020202020204439
:10735F006174612020202020200020202020205236
:10736F0065636F726420202020200053772F4F66B3
:10737F006620542E202020202020200A35536563BC
:10738F002A0044656C20496D6D65642E20202020F5
:10739F00202000004C6F6E6752616E67653A2020A7
:1073AF00202020200030207365632E2020202020F5
:1073BF00202020202000302C3235207365632E20B2
:1073CF0020202020202000302C35207365632E20B4
:1073DF00202020202020200031207365632E2020C4
:1073EF002020202020202020004C616E67756167CF
:1073FF00653A2020202020202000456E676C69739D
:10740F0068202020202020202020004974616C69F2
:10741F00616E202020202020202020004672656EE3
:10742F006368202020202020202020200047657224
:10743F006D616E20202020202020202020005370FE
:10744F00616E697368202020202020202020000CEE
:10745F00205374616E646172642046696C652020EC
:10746F00004E6F537441646472202020202020202E
:10747F0020002B242D25002B2D242500252D242BFA
:10748F0000252B242D000C436F6465202020202025
:10749F002020202020202000000C5174793A202039
:1074AF002020202020202020202000000C20202021
:1074BF0020205363616E6E6572202020200A2020E9
:1074CF00204D656D6F72792046756C6C2020000021
:1074DF000C202020202020537572653F2020202073
:1074EF0020003C454F543E0025303262757C00250C
:1074FF00303262752F25303262752F25303262752A
:10750F007C0025303262753A25303262757C007C02
:10751F000025303262752530326275005E25735B4F
:10752F0025732563005B25732563005D2573000CB0
:06753F002573002020204E
:1075450020202020202020202020202020002573FE
:107555000020202020202020202000202020202066
:107565002020000A456E61626C65202020202020C5
:1075750020202020000A44697361626C6520202068
:10758500202020202020000C257325732F6E000C51
:1075950020203732352020456D756B657920200A0E
:1075A5002020205365742055702046363420202035
:1075B500000C20202052657475726E20746F202097
:1075C500200A202020202044656661756C742020E7
:1075D5002020004F7074456E61626C65202020206C
:1075E500202020004F707444697361626C6520200F
:1075F5002020202000256C64000C202020204465DC
:107605006C6574652120202020200031000C257335
:107615000A2573003132386B206279746573002056
:1076250020313238206B72616D2020003235366B87
:10763500206279746573002020323536206B7261C3
:107645006D2020003531326B20627974657300201E
:1076550020353132206B72616D202000313032349B
:107665004B6279746573003130323420206B72615E
:107675006D202000323034384B62797465730032E6
:1076850030343820206B72616D202000464F524DFA
:10769500554C41373235003C4253593E003C52551A
:1076A5004E3E003C41434B3E00762E302F722E302D
:1076B500005772697474656E20627920466572722E
:1076C50065726F204B617469610046373235000C75
:1076D500202020537065632E50726F742E20202059
:1076E5000A202020446C6F6164204461746120206D
:1076F50020000C202020436C6F7365207468652082
:107705002020200A202020205365745570204636FD
:1077150034202020000C25732573002020257300BC
:107725000C2563202563202563000C2020202044A0
:10773500656C657465642120202020000C202044A0
:10774500656C2E205265636F72643F20200A2020ED
:107755002046313D4E202046323D59202020002430
:10776500252D0024252B00242F2400242F2F000C49
:10777500436F64653A20202020202023253034647F
:10778500000C446174653A202020202020232530F8
:1077950034640A25303262752F25303262752F2503
:1077A50030326275000C54696D653A202020202026
:1077B5002023253034640A25303262753A2530326B
:1077C5006275000C5174793A202020202020202356
:1077D500253034640A257300253032627500253062
:1077E5003262752F25303262752F25303262750071
:1077F50025303262753A253032627500464F524D5A
:10780500554C4137323520302D39393900464F52E4
:107815004D554C4137323520302D25303364003CF1
:10782500464E463E003C44454C3E003C434C523E91
:10783500003C4E414B3E0030312020656E7472692C
:107845006573202830312900256C642062797465C0
:10785500732066726565003C454F463E0025635BB7
:1078650030302020202020205E25732563000C2049
:107875002020537065632E50726F742E2020200ACD
:10788500202020202057616974696E672020202000
:10789500000C20203732352020456D754B65792049
:1078A50020200A2020205365742055702046363448
:1078B500202020000C2020496E7365727420373219
:1078C50035202020200A202020696E20746865203C
:1078D5003932352020200025737C000C2020202003
:1078E5005458204461746120202020200A20202043
:1078F5002020746F204636342020202020002020B0
:107905003732352020456D754B6579202020000ADA
:10791500202020446C6F6164204461746120202024
:06792500000A20202020D2
:10792B00456E71756972792020202020000C202073
:10793B0020205458205365747570202020200A2075
:10794B0020202020746F2046363420202020200059
:10795B0001012000010000FF7495FF74A7010009CD
:10796B0000010000FF74A8FF74BA000120000100A1
:10797B0000FF74BBFF74DE01012000010000FF74E7
:10798B00DFFF74DE01012000010000FF74DEFF74D5
:10799B00DE01010103010000FF74DEFF74DE010450
:1079AB000400010000FF74DEFF74DE0101200007FC
:1079BB000000FF74DEFF74DE01000900070000FF0A
:1079CB0074DEFF74DE01012000070000FF74DEFF90
:1079DB0074DE01012000070000FF74DEFF74DE017E
:1079EB00012000070000FF74DEFF74DE01010103BC
:1079FB00070000FF74DEFF74DE01000000060000CC
:107A0B00FF74DEFF74DE01012000010000FF74DE55
:037A1B00FF74DE17
:1021150061EF06E5FF6993FF69A4FF69B5FF69C62D
:10212500FF69D7FF69E8FF69F9FF6A0AFF6A1BFFC4
:102135006A2CFF6A3DFF6A4EFF6A5FFF6A70FF6A9D
:1021450081FF6A92FF6AA3FF6AB4FF6AC5FF6AD678
:10215500FF6AE7FF6AF8FF6B09FF6B1AFF6B2BFF3E
:102165006B3CFF6B4DFF6B5EFF6B6FFF6B80FF6B17
:1021750091FF6BA2FF6BB3FF6BC4FF6BD5FF6BE6E3
:10218500FF6BF7FF6C08FF6C19FF6C2AFF6C3BFFB8
:102195006C4CFF6C5DFF6C6EFF6C7FFF6C90FF6C91
:1021A500A1FF6CB2FF6CC3FF6CD4FF6CE5FF6CF64E
:1021B500FF6D07FF6D18FF6D29FF6D3AFF6D4BFF32
:1021C5006D5CFF6D6DFF6D7EFF6D8FFF6DA0FF6D0B
:1021D500A1FF6DB2FF6DC3FF6DD4FF6DE5FF6DF619
:1021E500FF6E07FF6E18FF6E29FF6E3AFF6E4BFFFD
:1021F5006E5CFF6E6DFF6E7EFF6E8FFF6EA0FF6ED5
:10220500B2FF6EC3FF6EDCFF6EF5FF6F06FF6F1842
:10221500FF6F2AFF6F3BFF6F4CFF6F5DFF6F6EFF18
:102225006F80FF6F91FF6FA3FF6FC5FF6FD7FF6FC4
:10223500E8FF6FF9FF700AFF701BFF702DFF703FFD
:10224500FF7050FF7061FF706FFF707BFF708CFF38
:10225500709DFF70AEFF70BFFF70D0FF70E1FF7023
:10226500F2FF70FCFF7108FF7115FF7126FF7137D2
:10227500FF7148FF715AFF716BFF717CFF718DFF14
:10228500719EFF71AFFF71C0FF71D2FF71E3FF71E6
:10229500E9FF71F7FF71FCFF721EFF722FFF72528B
:1022A500FF7263FF7274FF7285FF7296FF72A7FF5C
:0E22B50072B8FF72C9FF72D1FF72E2FF72F3BE
:1022C300FF730DFF731EFF732FFF7340FF7347FFF1
:1022D3007358FF7369FF737AFF7391FF73A2FF73E0
:1022E300A3FF73B4FF73C5FF73D6FF73E7FF73F8E0
:1022F300FF7409FF741AFF742BFF743CFF744DFFC6
:10230300745EFF74704108F600410E37004108D433
:102313000041056A00410E0F00410E3500410E2AAF
:1023230000410E1D00410CD9004106A70041066E75
:1023330000410E3000410E3100410E2100410E1FBD
:1023430000410E4A00410E270041055B00410E4942
:1023530000410A920041067200410A7FFF410E26A6
:10236300FF410560FF410E29FF410CF4FF410E546C
:10237300FF41066DFF4106E0004108F5024106DE1C
:1023830003410E1C014105680D410A80004106DA34
:10239300004106DF054106AB144106DD02410E1E76
:1023A30021410CD800410E3385410569014108FFE5
:1023B30001410567026078090B000000000000007E
:1023C300000000000000000000000000000000000A
:1023D30000000000000000000000000000000000FA
:1023E30000000000000000000000000000000000EA
:1023F30000000000000000000000000000000000DA
:1024030000000000000000000000000000000000C9
:1024130000000000000000000000000000000000B9
:1024230000000000000000000000000000000000A9
:102433000044090701020305440985010204054418
:102443000989010305004409910104050044099920
:102453000203050044099D020405004409A1030584
:1024630000004409A5040500004409AB0203000071
:102473004409AF02040000440E1103000000440E9F
:102483001704000000410E360060720A0C24252F49
:1024930000838424252E008385242531008386240C
:1024A3002524008387242432008997242424008050
:1024B3009724242D008B9724242B008C97242425E8
:1024C300008D97242431008E97242433008F972482
:1024D3002434009097242F24006297242F2F0092F6
:1024E3009724252D00839324252B008394242B2BC1
:1024F30000A39724242E00959724243600A4975AEA
:102503000DF51011122050F0A0A1A2B0B1B2D0D19C
:10251300D2E0E1E2A8803040607090215A08D83EB2
:102523003D3F423C4830494A344B4C384D4E3A4F7C
:102533005032454344463647524106AA00410E53A2
:1025430000410CDB00410CF500410E2200410E1B43
:10255300004106B8004108D70041099800410984A9
:1025630000410A0A0041056100410A0B004108FBD2
:1025730000410E2F00410AA3004109E800410AA5CA
:1025830000410CED004109900041066C004106B189
:10259300FF410983FF410AA4FF410A7EFF410E2048
:1025A30000410CDA004109E700410E2800410E10FA
:1025B300004108F709410E3401410E2E004206AFD7
:1025C3000000420E2B00004206DB0000420CF1002B
:1025D3000042056200004206B600004208D5000032
:1025E3004106E100420A9300004209A9000343099E
:1025F30095FF74814308F8FF7486430E50FF748B74
:10260300430904FF7490602106B900000000000034
:1026130000000000000000000000000000000000B7
:0B2623000000000000000000000000AC
:101F8A00E4FF74152FF8E4F60FEFB401F5E4FFEF60
:0F1F9A00C394005009742A2FF8E4F60F80F12247
:10295800900CF3E0601990066BE0FF7D527B047ADF
:102968000012B6C87F03127C39E4900CF3F0229071
:10297800066BE0FF7D527B647A0012B6C87F0412B2
:092988007C39900CF37401F0227B
:0A1FA900900CF37401F01229582285
:101FB300E4FF127C3990066BE0FF7D49E4FBFA12E3
:031FC300B6C8227B
:10299100AB07AA067C027D7612E5E3900A96ECF07D
:1029A100A3EDF0AE02AF037C027D7612E5E3EF24E6
:1029B10005900A99F0E43E900A98F07B017A8079BB
:1029C10000900A9A12E720900A96E0FEA3E0FF7CAD
:1029D100007D3412E5CF900A9BEE8FF012E638228B
:1029E10090051E12E72012299112D408900A99E04D
:1029F100FF12D423900A9A12E717AE02AF01900595
:102A01005EEEF0A3EFF0F8AC027D0190051E12E737
:0C2A1100177E007F3412E52C12D4102236
:102A1D0012299112D408900A99E0FF12D42378B3A9
:102A2D007C097D01900A9A12E7177E007F3412E52A
:052A3D002C12D4102250
:101FC60090055E7480F0A3E4F09006DBF0A3F022A7
:102A4200900CF2E02401900522F0900CF1E03400A9
:102A5200900521F09006DBE0FCA3E0FD900521E06B
:102A6200FEA3E0FFC39DEE9C5039122A1D78A47C80
:102A72000C7D017B017A0979B37E007F3412E52C4B
:102A8200900522E024FFFF900521E034FFFE7B0148
:102A92007A0C79A41229E1900521E475F00112E67D
:0E2AA2003880B19006DB74FFF5F012E63822A2
:102AB000900523EFF0A3EDF0E4A3F0900524E0FFF0
:102AC000A3E0C39F50409006AAE07006900E26E057
:102AD00060237B017A0679AC127B71900523E0FFBD
:102AE0007D327B0112C331E4FFFE0FBF00010EBE39
:102AF00005F8BFDCF57B017A0E794D127B719005EC
:072B000025E004F080B5227E
:102B0700900526EDF07D01122AB07F067D047C003A
:0E2B170012B2DB900526E0FF7D01122AB022EB
:102B2500EF75F00DA4245BF9747935F0FA7BFF7825
:102B3500817C0A7D017E007F0D12E52C9006E0E088
:102B45006010900A81E0FF9006E4E0FEEF4E900AE7
:032B550081F022EA
:102B5800900E2DE0FF7D49E4FBFA12B6C8900E34C2
:102B6800E0C394075012E004F090055CE4F0A3740D
:102B780016F07F0612B21922E4FF127C247F061297
:032B8800B27A22FC
:102B8B00900569E070087F28FE12C4BD800E900589
:102B9B0069E075F050A4FFAEF012C4BD12C4A522BB
:071FD600127FE612D902227E
:101FE700121FD67F057D03122AB07F067D147C0061
:041FF70012B2DB2225
:102BAB00E4FF127C247F0612B2197F0712B219229E
:102BBB00E4900E27F0900AA2F0900A95F0FF12D045
:022BCB00A52241
:0D2BCD00900E4AE06006900AA374FFF0220B
:102BDA0090052712E72090052712E71712438090E5
:102BEA00052712E717A801AC02AD037BFF7A7479B7
:102BFA00F112E966EF7004FF127C249008D5E4759F
:062C0A00F00112E6382281
:102C1000E4FEFDEE7018900CEE12E7178D827583BE
:102C20000012E56EB507027EFF0DEDB404E5AF06B8
:012C30002281
:102C3100E4900A91F0FF12D0A590055CE4F0A37432
:082C41001BF07F0612B27A229B
:102C490090052A12E72090052DEDF0E4A3F0FFFE90
:102C5900900E0FE06061E490052DE0FDEFD39D50EB
:102C69001390052A12E7178F8275830012E56E2EDD
:102C7900FE0F80E3EEC4540F90052EF0E4FF90059B
:102C89002EE0FDD394094012ED2437FC74A82FF5EA
:102C990082E43406F583ECF08010ED2430FD74A84D
:102CA9002FF582E43406F583EDF0EE540F90052EEE
:102CB900F00FEFB402C8229008D4E06029E4FF9035
:102CC900052DE0FDEFD39D501390052A12E7178FCC
:102CD9008275830012E56E6EFE0F80E3EE70027E50
:072CE900809006A8EEF02226
:102CF000122A1D7E007FFF7D007B017A0C79F6127F
:102D0000EC1B900A7FE0701D7BFF7A7479F79016B8
:102D10007012E720900E1CE0901673F07B017A0C85
:102D200079F612ED9B9009D4E0FF6464603B7BFF71
:102D30007A7479FE90167012E7209009D6E090160A
:102D400073F09009D5E0901674F0A3EFF07B017A50
:102D500005796C12ED9B7B017A05796C9016AD12AA
:102D6000E7207A0C79F612F4019009D8E0FF641993
:102D700060357BFF7A75791190167012E7209016F6
:102D800073EFF09009D9E0901674F07B017A057921
:102D90006C12ED9B7B017A05796C9016AD12E720E1
:102DA0007A0C79F612F4017B017A0979B39016ADA9
:102DB00012E7207A0C79F612F4017BFF7A75791EFE
:102DC0009016AD12E7207B017A0C79F612F4017BA4
:102DD000017A0979DC12F601EF4E60287B017A094D
:102DE00079DC9016AD12E7207A0C79F612F4017BAB
:102DF000FF7A75791E9016AD12E7207B017A0C7967
:052E0000F612F40122AE
:102E0500E490052FF0A3F0A3F07B017A0C79F6127C
:102E1500F601E4900530F0900530E0FEC39F501CAC
:102E250074F62EF582E4340CF583E0FE900531E06E
:102E3500FDEE6DF0900530E004F080DB90066CE06F
:102E45007004EF20E009900531E0547FF0800EEF2B
:102E55005401FEBE0107900531E04480F090053134
:102E6500E0FEC4540F90052FF0A37401F090052FD8
:102E7500E0540F4440FEF074F62FF582E4340CF56F
:102E850083EEF0900531E090052FF00FA3E004F0FC
:052E9500E0B403D922A6
:102E9A00122A1D9009D8E0FF641960557BFF7A75E4
:102EAA00792090167012E720901673EFF09009D9E6
:102EBA00E0901674F07B017A0A799D12ED9B7BFFF4
:102ECA007A75792B90167012E7207B017A0A799D20
:102EDA0090167312E7207A0979B390167612E720D2
:102EEA009009E6E0901679F07A0C79F612ED9B805B
:102EFA00277BFF7A75793490167012E7207B017A66
:102F0A000979B390167312E7209009E6E0901676D5
:102F1A00F07A0C79F612ED9B7B017A0979DC12F6CC
:102F2A0001EF4E60327BFF7A75793A90167012E79C
:102F3A00207B017A0979DC90167312E7207A0579E9
:102F4A006C12ED9B7B017A05796C9016AD12E72025
:102F5A007A0C79F612F40190091EE064017034A328
:102F6A00E090056CF0E4A3F07B017A0C79F69016F8
:102F7A00AD12E7207A05796C12F401E4900CF6F0B0
:102F8A007B017A05796C9016AD12E7207A0C79F6F6
:102F9A0012F401900CDBE060187B017A0C79F612CE
:102FAA00F60174F62FF582EE340CF5837403F08083
:102FBA00167B017A0C79F612F60174F62FF582EE79
:102FCA00340CF5837417F0E4900CDBF0122E052212
:102FDA00900A0BE070519006DBE07002A3E07002E9
:102FEA00FF22E49006B6F0A3F0FFFE122A1D900A13
:102FFA000B74FFF0E4900E15F0A3F07F097D011227
:10300A002AB012D90278647C157D017BFF7A7A791D
:10301A00047E007F0D12E52C12D7B490055CE4F013
:10302A00A3740BF07FFF2212D90278647C157D010C
:10303A007BFF7A7A79047E007F0D12E52C12D7B4D1
:10304A0090055CE4F0A3740BF09009E7E0704290FD
:10305A000E15F0A3F09006B7E024FF9006B6E03410
:10306A00FFC364809480500A7F027D01122AB07FD8
:10307A00FF229006B674FFF5F012E6389006B6E025
:10308A00FEA3E0FF122A1D7F097D01122AB07FFFED
:10309A0022900E15E0FEA3E0FFEE7065EF605B1470
:1030AA00604F1460311470599009D8E06419600BAC
:1030BA00900E15E4F0A37402F080469009D4E064FF
:1030CA0064600A900E15E4F0A304F08034E4900ED4
:1030DA0015F0A3F0802B9009D4E06464600A900E86
:1030EA0015E4F0A304F08019E4900E15F0A3F08023
:1030FA0010E4900E15F0A3F08007E4900E15F0A3EB
:0B310A00F07F097D01122AB07FFF2238
:10311500900A0BE070649006DCE024FFFF9006DB6C
:10312500E034FFFE9006B6F0A3EFF0C3EE648094A2
:103135008050037F00229006B6E0FEA3E0FF122A2E
:103145001D900A0B74FFF0E4900E15F0A3F07F09B3
:103155007D01122AB012D90278647C157D017BFFAE
:103165007A7A79047E007F0D12E52C12D7B490058A
:103175005CE4F0A3740BF07FFF2212D90278647C23
:10318500157D017BFF7A7A79047E007F0D12E52C8F
:1031950012D7B490055CE4F0A3740BF09009E7E056
:1031A5007052900E15F0A3F09006B7E02401FF9041
:1031B50006B6E03400FE9006DBE0FCA3E0FDC3EFBD
:1031C5009DEC6480F8EE648098400A7F027D0112D0
:1031D5002AB07FFF229006B6E475F00112E638901A
:1031E50006B6E0FEA3E0FF122A1D7F097D01122A23
:1031F500B07FFF22900E15E0FEA3E0FFEE60030214
:1032050032A4EF14604D14607514700302329B24D0
:103215000360030232A49009D4E06464600A900E4E
:1032250015E4F0A304F080779009D8E06419600BE9
:10323500900E15E4F0A37402F080647B017A09799D
:10324500DC12F601EF4E6057900E15E4F0A37403FF
:10325500F0804C9009D8E06419600B900E15E4F0ED
:10326500A37402F080397B017A0979DC12F601EF4B
:103275004E602C900E15E4F0A37403F080217B01C1
:103285007A0979DC12F601EF4E6014900E15E4F020
:10329500A37403F08009900E15E4F0A37403F07F86
:0932A500097D01122AB07FFF220D
:1032AE009006AAE07021121FD6122FDAEF70107F4F
:1032BE000B7D01122AB090055CE4F0A37402F07F3E
:0832CE000612B21912C4A52278
:1032D6009006AAE07021121FD6123115EF70107FEA
:1032E6000B7D01122AB090055CE4F0A37402F07F16
:0832F6000612B21912C4A52250
:1032FE00121FD678647C157D017BFF7A7A79047E65
:10330E00007F0D12E52C12D7B47F0612B21912C42B
:02331E00A522E6
:1033200090053212E720900535ECF0A3EDF0E4A310
:10333000F090053212E71712E55570030233D19071
:1033400006B1E060159007F612E71790167012E7C5
:10335000207BFF7A75793E12EDA1900535E0FFA341
:10336000E0900538CFF0A3EFF09006DBE0FCA3E09F
:10337000FD900538E0FEA3E0FFC39DEC6480F8EE0D
:10338000648098504C900537E07046122A1D78B33F
:103390007C097D0190053212E71712E966EF70256E
:1033A00090053774FFF0A3E0FEA3E0FF900CF1EE70
:1033B000F0A3EFF0900562EEF0A3EFF09006B17489
:1033C000FFF07F0122900538E475F00112E63880A5
:1033D00098900537E0600B90053212E71712E5551B
:1033E000702B9006B1E060259007FF12E71790164A
:1033F0007012E7207BFF7A75793E12EDA1121FE76C
:10340000E4900E53F090055CF0A37402F09006B1C6
:0634100074FFF07F0022B2
:1034160090053A12E720E490053EF0A3F090053DB2
:10342600F090053A12E71712F60190053DE0C39FAA
:10343600EE6480F8748098502E90053A12E7179043
:10344600053DE0F58275830012E56EFF12F38D40AF
:103456000E90053DE090053FF090053EE004F090AB
:10346600053DE004F080BA90053EE0FF601F640170
:10347600703690053A12E71790053FE0F58275839E
:103486000012E56EFF642E6004EFB42C1B90053A23
:1034960012E71712F6019008F7E0FDD3EF9D74804E
:0B34A600F86E9850037F01227F002287
:1034B10090054012E720900543EDF0E0FFA3E0FD09
:1034C10012D5187BFF7A75794212EDA1900543E080
:1034D100FFA3E004FD12D5187BFF7A75794212ED46
:1034E100A1900543E0FFA3E0FD12D518900540121D
:1034F100E71712F601D3EF9410EE64809480501612
:1035010090054012E71790167012E7207BFF7A753D
:10351100795312EDA122E4900545F0900545E0FFB5
:10352100D3940F501A90054012E7178F82758300CC
:1035310012E56EFF12D6AE900545E004F080DC90F6
:103541000543E0FFA3E004FD12D518900545741072
:10355100F090054012E71712F601900545E0C39F70
:10356100EE6480F8748098501E90054012E7179021
:103571000545E0F58275830012E56EFF12D6AE9027
:083581000545E004F080CA22B8
:1035890090054612E720900E4BE07004A3E0640614
:103599007028FF7D0112D5187BFF7A75794212EDEB
:1035A900A1E4FF7D0212D5187BFF7A75794212EDED
:1035B900A1E4FF7D0112D5188068900E4BE07004DC
:1035C900A3E06407705C900E49E060297F067D01E5
:1035D90012D5187BFF7A75795612EDA17F067D0207
:1035E90012D5187BFF7A75795612EDA17F067D01F8
:1035F90012D518802D900A92E060277F097D01126B
:10360900D5187BFF7A75796012EDA17F097D0212C9
:10361900D5187BFF7A75796012EDA17F097D0112BA
:10362900D51890054612E71790167012E7207BFF10
:083639007A75795312EDA1220C
:10364100EF600B7BFF7A75796812EDA180097BFF32
:103651007A75797A12EDA17F067D127C0012B2DBB8
:013661002246
:0B3662007FE07E2E12C4BD12C4A52222
:10366D009006AA74FFF0900E54F0FF127B5C7F0160
:10367D0012CFEE90085612E71790167012E72090B1
:10368D00085912E71790167312E7207BFF7A7579A8
:10369D008C12EDA11236627F067D0D122B07E49080
:0C36AD0008FBF090055CF0A3740CF02208
:1036B900E49006AAF0FF127B5CE4FF12CFEE9008BB
:1036C9005612E71790167012E72090085912E7175B
:1036D90090167312E7207BFF7A75798C12EDA1128F
:1036E900099C900457E004F07F0D7D06122B07908A
:0936F900055CE4F0A37402F02268
:1037020090055B74FFF0900672F0900E1DF0900829
:10371200D4F0E4900E0FF0900CD9F0900E35F07BBF
:10372200FF7A75799412EDA1E49006DBF0A3F01212
:103732003662E49008FBF090055CF0A37418F02266
:10374200121BAD7F087D02122AB07BFF7A7579B613
:1037520012EDA17F067D147C0012B2DBE49008FB1F
:0A376200F090055CF0A37402F02261
:10376C00E49008FBF090055CF0A37402F09009EB78
:10377C00E0FFB4241E900E2974FFF0900CF4F0E4DA
:10378C00900E21F0900A92F0900E31F0900A7F7416
:10379C00FFF022EFB42D15900E29E070047F01800C
:1037AC00027F00900E29EFF0123641229009EBE0D7
:1037BC00B42B15900CF4E070047F0180027F009014
:1037CC000CF4EFF0123641229009EBE064317055A5
:1037DC00FF7D0112D518900A92E0702C900E31E00A
:1037EC0070047F0180027F00900E31EFF0600F7B40
:1037FC00FF7A7579D812EDA1E4900E21F0227BFFAF
:10380C007A7579E912EDA1227F057D03122AB09019
:10381C00086812E71790167012E7207BFF7A75790B
:10382C005312EDA1229009EBE064337025900E2128
:10383C00E070047F0180027F00900E21EFF06009A0
:10384C00E4900E31F0900A92F0900E21E0FF1236C7
:10385C0041229009EBE0B4341590066DE070047FC2
:10386C000180027F0090066DEFF012364122900924
:10387C00EBE0B4251C900A9274FFF0E4900E31F04A
:10388C00900E21F012366290055CE4F0A37407F000
:10389C00229009EBE0B42E13900E4974FFF012360F
:1038AC006290055CE4F0A37407F0229009EBE0FF52
:1038BC00B43210900E1F74FFF090055CE4F0A3740A
:1038CC0006F022EFB43614900A7FE070047F01807A
:0C38DC00027F00900A7FEFF012364122BC
:1038E800900E5374FFF0E49008FBF09006DBE07054
:1038F80002A3E070167F057D03122AB090055CE4F0
:10390800F0A37402F0E4900E53F0229009EBE0FF6C
:10391800B4240A90055CE4F0A37404F022EFB42FF9
:10392800237B017A0679B9900563E02401FD9005AF
:1039380062E03400FC123320EF600990055CE4F08B
:05394800A3740AF02247
:10394D0090055CE4F0A37402F09009EBE0FF642DA8
:10395D006004EFB42B29E49008FBF09006DBE070D7
:10396D0002A3E070087F057D03122AB0227F087D37
:10397D0002122AB09006DB74FFF5F012E6382290A1
:10398D0009EBE0642F6003023A539008FBF09006B8
:10399D00DBE0FEA3E0FFD39400EE6480948050033F
:1039AD00023A4BEF24FFFFEE34FFFE122A1D7B017E
:1039BD007A0979DC12F61690054912E6FF7F017E31
:1039CD00007D007C0090054912E6F3C312E6D66037
:1039DD00069009DCE070127F087D02122AB0900675
:1039ED00DB74FFF5F012E6382290054912E6E77B0D
:1039FD00FF7AFF79FF78FF12E66490054912E6FF22
:103A0D007A7579FA90167012E72090054912E6E75B
:103A1D0090167312E6FF7B017A0C79CD12ED9B7F28
:103A2D00087D02122AB09006DCE024FFFF9006DB31
:103A3D00E034FFFE7B017A0C79A41229E1227F0587
:103A4D007D03122AB0229009EBE0642470459008A2
:103A5D00FBE070047F0180027F009008FBEFF060B7
:103A6D00117F067D0D122B0790055CE4F0A3740306
:103A7D00F0227BFF7A7579FE12EDA1E49006DBF062
:103A8D00A3F07F0D7D06122B077F067D147C00129F
:103A9D00B2DB229009EBE0FF642E6005EF6431701C
:103AAD003CE49008FBF0D39006DCE094009006DB3C
:103ABD00E064809480401F9009EBE0B42E089009DB
:103ACD008474FFF08006900A0A74FFF090055CE4A0
:0E3ADD00F0A37403F0227F057D03122AB022AD
:103AEB0078A47C0C7D017B017A0979E912EA4FE419
:103AFB00FFFEEF702974F52EF582E4340DF583E0AB
:103B0B00FD9006B2E0B5051174D82EF582E43408A9
:103B1B00F583E0900CD7F07FFF0EEEB41AD490062D
:103B2B006DE060097F067D0A7C0012B2DB900A9281
:103B3B00E0F46007900E1FE0B4FF0A90055CE4F020
:103B4B00A37406F022900E31E0601978CD7C0C7DC9
:103B5B00017BFF7A76791012EA4F90055CE4F0A3B3
:103B6B007409F022900E21E07003023C18E49006D9
:103B7B00B1F07B017A0979E9FDFC123320EF701962
:103B8B0078CD7C0C7D017BFF7A76791012EA4F9011
:103B9B00055CE4F0A37409F02290056174FFF090CA
:103BAB000CF1E0FEA3E0FF122A1D78A47C0C7D0132
:103BBB007B017A0979B37E007F3412E52C900CCD12
:103BCB00E0700F78CD7C0C7D017BFF7A767910123B
:103BDB00EA4F7B017A0C79CD12F616EF2401FFE444
:103BEB003EFEE43DFDE43CFC90167312E6FF7BFFCA
:103BFB007A7579FA90167012E7207B017A0C79CDE1
:103C0B0012ED9B90055CE4F0A37409F02278CD7C57
:103C1B000C7D017BFF7A6D79A012EA4F90055CE475
:063C2B00F0A37409F02271
:103C310090099512E717A801AC02AD037B017A093F
:103C410079E912E966EF700412366D229008F812D4
:103C5100E717A801AC02AD037B017A0979E912E902
:103C610066EF700412370222900E5012E717A80176
:103C7100AC02AD037B017A0979E912E966EF7004C0
:103C8100123742227B017A0979E912F601EF6403C6
:103C91004E6003023D939009E9E064246003023D14
:103CA1009390054DF090054DE075F006A4240CF9B4
:103CB100740A35F0A801FC7D017B017A0979E912CA
:103CC100E966EF600E90054DE0C394135005E004E2
:103CD100F080D290054DE0C394134003023D7DE096
:103CE100FF75F006A42410F582E4340AF583E0752B
:103CF100F0039006E512E70B12E71790167012E732
:103D010020EF75F006A42411F582E4340AF583E06E
:103D110075F0039006E512E70B12E7179016731280
:103D2100E7207BFF7A76791212EDA17F067D147C64
:103D31000012B2DB9009EAE0B4240412376C22903D
:103D410009EAE0B42F041238E8229009EAE0B42528
:103D51000412394D229009EAE0642B6003023DE12F
:103D6100A3E0642B707A90055CF0A37402F0E490F8
:103D71000CD9F0900E35F09008FBF0227F057D0301
:103D8100122AB090055CE4F0A37402F0E49008FB01
:103D9100F022900990E070319008FBF0900E1EE047
:103DA100D3942050207B017A0979E912F601900E13
:103DB1001EE06F7001EE600D121FE790055CE4F0EC
:103DC100A37402F022123AEB22900990E06011E410
:103DD1009008FBF0121FE790055CE4F0A37402F079
:013DE10022BF
:103DE200121FC6121F8A7E297F5812B66490066B74
:103DF200EFF07E2B7F5812B664900E2DEFF0E51691
:103E020024FBFFE434FFFE9009A9F0A3EFF0643F26
:103E12004E700B900A93747DF0A3E4F08017900922
:103E2200A9E0FEA3E0FF7C027D7612E5CF900A9323
:103E3200EEF0A3EFF09009A9E07004A3E064037030
:103E42002178387C0E7D017BFF7A76791912EA4F50
:103E520078DC7C0C7D017BFF7A76792412EA4F02B2
:103E62003F069009A9E07004A3E064077020783847
:103E72007C0E7D017BFF7A76793112EA4F78DC7C09
:103E82000C7D017BFF7A76793C12EA4F80769009AD
:103E9200A9E07004A3E0640F702078387C0E7D01E5
:103EA2007BFF7A76794912EA4F78DC7C0C7D017BC4
:103EB200FF7A76795412EA4F804A9009A9E0700499
:103EC200A3E0641F702078387C0E7D017BFF7A7638
:103ED200796112EA4F78DC7C0C7D017BFF7A76797E
:103EE2006C12EA4F801E78387C0E7D017BFF7A7659
:103EF200797912EA4F78DC7C0C7D017BFF7A767946
:103F02008412EA4F9006AE7401F09006ADF090066E
:103F1200ACF0E4900E4FF0900E4EF0900E4DF090FB
:103F220009677402F0900964F0900961F090095EEB
:103F3200F090095BF090096AF0121BAD12D0BE50EE
:0E3F42000C90055CE4F0A37402F0122BAB228D
:103F5000900E33E0FF12D2769008F6E060057FFF06
:103F600012D168900984E06002E4F0900A0AE060EF
:103F700002E4F012D0BE5012900E4BE0FFA3E0908E
:0B3F8000055CCFF0A3EFF0122BAB228A
:103F8B00121FD6900A0BE0601678647C157D017BBE
:103F9B00FF7A7A79047E007F0D12E52C12D7B422BA
:103FAB00900E2FE0705D900E3274FFF0FF12D0A5D3
:103FBB00900AA2E0FF900A95E06F6016900AA2E0CB
:103FCB0004F074A52FF582E4340BF583E0FF12D3D4
:103FDB002A22E4900E32F0122BBB900CD9E0701E0B
:103FEB00900E4AE07006900983E07012900E35E057
:103FFB006011900560E0600B900983E070057F060F
:04400B0012B21922B2
:10400F00900E3274FFF0FF12D0A5900AA2E0FF903D
:10401F000A95E06F601C7F0112D401900AA2E0FFA5
:10402F0004F074A52FF582E4340BF583E0FF12D36F
:0C403F002A22E4900E32F0FF12D0A522DD
:10404B0090054EEFF0900E35E06071900560E070DA
:10405B006B900983E0706590054EE0B4061E900EE0
:10406B002DE0FF7D49E4FBFA12B6C8900E347401C3
:10407B00F07FFF127C247F0612B2192290054EE0CE
:10408B006415600302437FC39008D5E0648094807D
:10409B00500302437F900E2DE0FF7D49E4FBFA12A3
:1040AB00B6C8900E347401F090055CE4F0A374165E
:1040BB00F07FFF127C247F0612B2192290055BE081
:1040CB00603F90054EE0B406067F0612B2192290AF
:1040DB00054EE0FF640A6014900A91E0FE04F07450
:1040EB00A62EF582E4340AF583EFF022900A91E0D4
:1040FB0024A6F582E4340AF583EFF07F0612B21999
:10410B0022900E2AE0602590054EE0FFB413079035
:10411B000E2F74FFF022EFB41109E4900E2FF01262
:10412B003FAB22900CD9E0600302437F900AA3E0DF
:10413B00F47049900935E0FF90054EE0FEB507108D
:10414B0090055CE4F0A37412F0E4900AA3F08021D4
:10415B00900937E0B5060B90055CE4F0A37413F0FF
:10416B00800FE4900AA3F0FF127C247F0612B27A30
:10417B00227F0612B219E49009E8F022900A91E02E
:10418B00FF702F90054EE0FE74A62FF582E4340AE3
:10419B00F583EEF012080CE4900E10F0900CEE127A
:1041AB00E717900E10E0F58275830012E56E900E06
:1041BB0036F0900E36E012E7B241DD0141F60242D5
:1041CB003503426604430205433A06435F0700008A
:1041DB00437F900CEE12E717900E10E004F0F5827F
:1041EB0075830012E56E900E36F022900CEE12E7FE
:1041FB0017900E10E004F0F58275830012E56E90B7
:10420B000E36F09008F5E0FF90054EE0FE6F60066D
:10421B00E4900E36F022900A91E0FF04F074A62F82
:10422B00F582E4340AF583EEF022900E1CE0FF9049
:10423B00054EE0FEB5071A900A91E0FF04F074A654
:10424B002FF582E4340AF583EEF0900E367404F009
:10425B0022E4900E36F0900A91F022900920E0FFB4
:10426B00700C900568E0FE90054EE0B50611EF640A
:10427B000170379006DEE0FE90054EE06E602B90ED
:10428B000A91E0C394FC501A90054EE0FE900A91FF
:10429B00E0FD04F074A62DF582E4340AF583EEF00C
:1042AB008034900E2774FFF0802C90054EE0FE902A
:1042BB000A91E024A6F582E4340AF583EEF0900C23
:1042CB00EE12E717900E10E004F0F58275830012E2
:1042DB00E56E900E36F0900E36E0600302437FEFF2
:1042EB00700E90055CF0A37410F07F0612B21922C9
:1042FB00900E367407F0229009E874FFF090054E8B
:10430B00E09006E2F0900E0FE06007900E36740618
:10431B00F022900920E0B40107900E367407F022CA
:10432B0090055CE4F0A37410F07F0612B219229092
:10433B00054EE09006E3F0900920E0B40107900EE3
:10434B00367407F02290055CE4F0A37410F07F063E
:10435B0012B21922900568E0FF90054EE06F6006DF
:10436B00900E2774FFF090055CE4F0A37410F07FBF
:05437B000612B2192238
:1043800090054F12E720E4900AA2F0900A95F09071
:104390000552F0900E0FE070069008D4E0601F9078
:1043A00009E8E0B4FF18900935E0FF900A95E0FEB7
:1043B00004F074A52EF582E4340BF583EFF07F0250
:1043C000122C10EF60189008F5E0FF900A95E0FEBF
:1043D00004F074A52EF582E4340BF583EFF07F032F
:1043E000122C10EF6018900E1CE0FF900A95E0FE72
:1043F00004F074A52EF582E4340BF583EFF09005FC
:104400004F12E717900552E0F58275830012E56EB2
:10441000602B90054F12E717900552E0FF04F08FD4
:104420008275830012E56EFF900A95E0FE04F07439
:10443000A52EF582E4340BF583EFF080C1900920BE
:10444000E0B4011A9006DEE0FF900A95E0FE04F069
:1044500074A52EF582E4340BF583EFF080189005F7
:1044600068E0FF900A95E0FE04F074A52EF582E462
:10447000340BF583EFF07F05122C10EF700302452B
:1044800025900935E0FF7E00900BA5E0FD3395E017
:10449000FCEDB50734EEB504307B017A0B79A690BC
:1044A00016C812E720900A95E024FF9016CCF0EE93
:1044B00034FF9016CBF07A05796C12F599900A9535
:1044C000E024FE900552F08018786C7C057D017B1D
:1044D000017A0B79A512EA4F900A95E014900552E3
:1044E000F07B017A05796C900552E0FD122C499021
:1044F00006A8E0FF900A95E0FE04F074A52EF58270
:10450000E4340BF583EFF0900E0FE060189006A9ED
:10451000E0FF900A95E0FE04F074A52EF582E434E5
:104520000BF583EFF0900920E0B40118900568E0E6
:10453000FF900A95E0FE04F074A52EF582E4340B9A
:10454000F583EFF0900E32E07003123FAB7F06125E
:08455000B27AE4900A91F02216
:1045580090055312E720E4900AA2F0900A95F0FF24
:1045680090055312E7178F8275830012E56E602756
:1045780090055312E717AE070F8E8275830012E578
:104588006EFE900A95E0FD04F074A52DF582E434E2
:104598000BF583EEF080C9900A95E0FF04F074A54E
:1045A8002FF582E4340BF583740DF07F0612B27A8E
:0F45B800900E32E07003123FABE4900A91F022B4
:1045C7009008FFE024A5F582E4340AF583E0FE6451
:1045D7001B60037F0B22EEB41B1A900A91E024A5FF
:1045E700F582E4340AF583E0B41B06900E27E060F9
:1045F700037F0C22900567E0FF2402900556F0EF39
:104607002407A3F0120540EF60037F0A229008FFFA
:10461700E024A6F582E4340AF583E06430600302FF
:1046270046D874FF9008D5F0A3F0900567E024A65C
:10463700F582E4340AF583E0F9B42A0F900556E0D1
:10464700FF900A91E0B507037F0122E9B4240F9098
:104657000556E0FF900A91E0B507037F0222E9B40F
:104667002D0F900556E0FF900A91E0B507037F03F1
:1046770022E9B42B0F900556E0FF900A91E0B507A9
:10468700037F0422E9B42B0F900557E0FF900A91AE
:10469700E0B507037F0522900567E024A6F9E43417
:1046A7000AFA7B01C003C002C0017BFF7A767991C9
:1046B7009016C012E7209016C3E4F0A3740AF0D056
:1046C70001D002D00312F532EF70037F01227F067B
:1046D700229008FFE024A6F582E4340AF583E0641B
:1046E70031600302482074FF9008D5F0A3F09005CD
:1046F70067E024A6F582E4340AF583E0FEB42A0FC6
:10470700900556E0FF900A91E0B507037F0722EE78
:10471700B42D17900556E0FF900A91E0B5070B906E
:104727000E2BE4F0A304F07F0822EE642D70439073
:104737000557E0FF900A91E06F7037900567E02416
:10474700A7F9E4340AFA7B019016C812E7209016FD
:10475700CBE4F0A37405F07A05796C12F5997B0127
:104767007A05796C12F724900E2BEEF0A3EFF07F09
:104777000822900567E0FE24A6F582E4340AF58353
:10478700E0642F705A74A72EF582E4340AF583E0AB
:10479700B42A15EE2403FDE433FC900A91E0B50535
:1047A70007E4B504037F092274A72EF9E4340AFA53
:1047B7007B01C003C002C0017BFF7A767991901616
:1047C700C012E7209016C3E4F0A3740AF0D001D01A
:1047D70002D00312F532EF70037F09227F06229081
:1047E7000567E024A6F9E4340AFA7B01C003C00296
:1047F700C0017BFF7A7679919016C012E720901658
:10480700C3E4F0A3740AF0D001D002D00312F5324A
:10481700EF70037F07227F06229008FFE024A6F5AA
:1048270082E4340AF583E0643570299006AAE060D3
:104837001178F67C0C7D017BFF7A76799C12EA4F22
:10484700800F78F67C0C7D017BFF7A7679A212EADD
:104857004F7F0A229008FFE024A6F582E4340AF588
:1048670083E0B43618127CEC127C9C121BAD7BFFE4
:104877007A3F79AB127CBA127C867F0B229008FFB5
:10488700E024A6F582E4340AF583E0643770749077
:104897000567E0FF24A6F9E4340AFA7B019016C8FD
:1048A70012E720EF2401FFE433FE900A91E0C39F53
:1048B7009016CCF0E49E9016CBF07A05796C12F541
:1048C70099900567E0FF900A91E0C39FFFE4940089
:1048D700FE746B2FF582EE3405F583E4F07F0C123E
:1048E700D6AE7B017A05796CE4FD900544F012346D
:1048F700B178F67C0C7D017BFF7A7679A812EA4FB6
:0E4907007F0A229008FFE024A6F582E4340A1D
:10491500F583E0643860030249D6900567E024A674
:10492500F582E4340AF583E0B42A1E900556E0FFCB
:10493500900A91E0B5071278F67C0C7D017B017A2F
:104945000E793812EA4F0249D3900567E024A6F59F
:1049550082E4340AF583E0B4241D900556E0FF9007
:104965000A91E0B5071178F67C0C7D017BFF7A761C
:1049750079AE12EA4F8057900567E024A6F582E4E8
:10498500340AF583E0B4211D900556E0FF900A91A5
:10499500E0B5071178F67C0C7D017BFF7A7679B658
:1049A50012EA4F8029900567E02401FFE433FE9069
:1049B5000A91E0B50715E4B5061178F67C0C7D0182
:1049C5007BFF7A7679CF12EA4F80037F0C227F0A2C
:1049D500229008FFE024A6F582E4340AF583E0FF7F
:1049E500C394414067EFD3945A5061127C9C127C6A
:1049F500EC90066E74FFF09008FFE024A6F582E4C3
:104A0500340AF583E075F00390041812E70B12E7FA
:104A15001712E7D8E490066EF0900E27E0701E7826
:104A2500F67C0C7D017BFF7A7679A812EA4F127C21
:104A3500867BFF7A3F79AB127CBA7F0A22127C868D
:0F4A45007BFF7A3F79AB127CBA7F0C227F0C2269
:074A5400122BAB12C4A522D6
:074A5B00122BAB12C4A522CF
:04000E0012C4A52251
:104A6200121FD67F067D0D122B07E4FF12D168902C
:104A72000E35E0604274FF9008D5F0A3F0FB7A7621
:104A820079D412EDA1E4900983F0900E3404F07F02
:104A9200FF127C24900560E0600C90055CE4F0A3BA
:104AA2007417F0024B54E4FF127C2490055CE4F08E
:104AB200A37414F0024B5490055BE0604F7F057DB8
:104AC20001E4FB12D2BF900672E0601F7F097D03F2
:104AD200122AB07BFF7A7679F712EDA190055CE499
:104AE200F0A37418F07F0612B27A22E4900998F0CB
:104AF200900E1DE0600B90055CE4F0A3741FF08043
:104B02005190055CE4F0A3741AF0804690085612A6
:104B1200E71790167012E72090080E12E71790160A
:104B22007312E7207BFF7A77791A12EDA1E4FF7DF9
:104B32000212D5187B017A0C79DC90167012E720EC
:104B42007BFF7A77792012EDA190055CE4F0A374E3
:104B52000FF0E4FF12D0A5127C8690055BE0600B9B
:104B62007BFF7A40790F127CBA80097BFF7A3F790A
:104B7200AB127CBA900CD9E0603FD39006DCE09493
:104B8200009006DBE064809480402EE4900E2FF0CB
:104B9200900A7FE06005E4A3F08006900A8074FF2B
:104BA200F0122BBBE49008D5F0A3F07FFF127C2417
:104BB20090055CE4F0A3740EF07F0612B219900522
:104BC20060E06012900E35E0600C7F069006ABE06C
:074BD200FD7C0012B2DB22A2
:104BD900121FD67F067D0D122B07127CEC127C9CCE
:104BE9009008F6E060057FFF12D168900984E060C3
:104BF90002E4F0900A0AE06002E4F0900E35E06009
:104C090013900E2DE0FF7D49E4FBFA12B6C8900916
:104C19008374FFF0122BAB90055BE060069006727F
:104C2900E0700990055CE4F0A37402F09006AAE034
:064C3900600312366D223B
:104C3F009012B2E0FFFD3395E0FC900CDAE06D705E
:104C4F0001EC600E900CDAEFF07B017A1279AE1264
:034C5F007A1E2298
:104C6200900558EFF0E0B4030D900E20E06403606D
:104C72001A121FA98015900558E0FF127C39900680
:104C82006BE0FF7D49E4FBFA12B6C8900558E0904C
:044C92000E20F022DE
:04001600121FB322E0
:104C9600121FD6E4FF127C247F0512B27A7F071218
:034CA600B27A22BD
:104CA900AE037BFF7A777925901670EFF0A3EDF0CC
:074CB900A3EEF012EDA122B1
:104CC000EF12E7B24CE0014CE8024CF0034CF80460
:104CD0004D00054D08064D10074D180800004D1FEA
:104CE0007F0B7D01122AB0227F047D01122AB0229F
:104CF0007F057D01122AB0227F0D7D01122AB0228C
:104D00007F087D01122AB0227F097D01122AB0227C
:104D10007F087D01122AB0227F0A7D01122AB0226B
:104D2000EF24FA601A14604414605B2403707090DE
:104D30000A0BE0606A9009E77401F01232AE22902B
:104D40000A0BE0600A9009E77401F01232D6229053
:104D500008F6E0600BE4FF12D168E49008F6F02258
:104D60007FFF12D1689008F674FFF022D39006DC22
:104D7000E094009006DBE0648094804022E4900997
:104D8000E7F01232AE22D39006DCE094009006DB0E
:104D9000E0648094804008E49009E7F01232D62263
:104DA000EF24FE7003024E57147003024F1D14705F
:104DB00003024F4024FB7003024F7E24086003026D
:104DC0004FA9900A0BE06040900E37E0603A121F46
:104DD000D67F097D01122AB0E4900E37F09006B616
:104DE000E0FEA3E0FF122A1D78647C157D017BFFA5
:104DF0007A7A79047E007F0D12E52C12D7B49005E3
:104E00005CE4F0A3740BF022900E37E06003024FD5
:104E1000A9121FD67F057D01122AB090089B12E7C8
:104E20001790167012E7207BFF7A75793E12EDA17C
:104E30007B017A0679B9900563E02401FD90056253
:104E4000E03400FC123320EF7003024FA990055CA0
:104E5000E4F0A3740AF022900A0BE07003024F0002
:104E6000900E37E07003024F00121FD67F057D01C0
:104E7000122AB07F0112CFEEE4900E37F09006B602
:104E8000E0FFA3E0900CF1CFF0A3EFF0122A42E490
:104E9000FF12CFEE7BFF7A77792F12EDA19006DB20
:104EA000E0FEA3E0FF900CF1E0B5060FA3E0B5072C
:104EB0000A9006B674FFF5F012E638EF4E700D90CA
:104EC0000A0BF090055CF0A37402F0229006B6E0A5
:104ED000FEA3E0FF122A1D7F067D147C0012B2DBC8
:104EE00078647C157D017BFF7A7A79047E007F0DE2
:104EF00012E52C12D7B490055CE4F0A3740BF022F9
:104F0000900E37E06003024FA9121FD67F057D0186
:104F1000122AB090055CE4F0A37404F022900A0B0E
:104F2000E07003024FA9900E37E06003024FA97FA3
:104F30000B7D01122AB0900E3774FFF01232FE2260
:104F4000900A0BE07063121FD67F057D01122AB014
:104F500090088012E71790167012E7207BFF7A7591
:104F6000793E12EDA17F067D147C0012B2DB900E1B
:104F70001F74FFF090055CE4F0A37406F022900A21
:104F80000BE06025121FD67F097D01122AB0E4FFD5
:104F900012CFEEE4900A0BF0900E37F090055CF023
:0A4FA000A37402F07F0612B219227A
:0300080080002253
:074FAA00122BAB12C4A5227B
:104FB10090055CE0FEA3E0FFEE6003026923EF12BF
:104FC100E7B250270150670251230351B704521E23
:104FD1000554D60655550755E80858A60959140A27
:104FE10059580B5BF50C5C1F0D5C970E5E0D0F5E47
:104FF100311060AD1160B31262AF1362CA1462E185
:105001001662F517642918646C19653F1A65651BEA
:10501100667D1C672B1D68011E68941F68C320688C
:10502100E021000069237F02122B2578FF7C0E7D91
:10503100017B017A0A79817E007F0D12E52C127EB7
:105041004D78647C157D017BFF7A7979D07E007F74
:105051000D12E52C12D7B490055CE4F0A37405F0B1
:105061007F0612B27A2290055CE0FFA3E0900E4B1E
:10507100CFF0A3EFF0E4900990F0900E53F0900A76
:105081000BF0900E37F0122B8B900A93E0FEA3E009
:10509100FFC39006DCE09FEE6480F89006DBE064DD
:1050A100809840187F0B7D327B0112C331900990AB
:1050B10074FFF090055CE4F0A304F022E4FF122BEE
:1050C1002578FF7C0E7D017B017A0A79817E007F44
:1050D1000D12E52C127E4D78647C157D017BFF7AE3
:1050E1007979B67E007F0D12E52C12D7B47F04E4E6
:1050F100FD12D51890055BE060077F2A12D6AE80BD
:1051010012900E35E060077F2312D6AE80057F3AFC
:1051110012D6AE90055CE4F0A37405F07F0612B2DE
:105121007A229008FBE060337F03122B2578FF7C05
:105131000E7D017B017A0A79817E007F0D12E52CBB
:10514100127E4D78647C157D017BFF7A7979DD7E55
:10515100007F0D12E52C12D7B4804C7F04122B2551
:1051610078FF7C0E7D017B017A0A79817E007F0DBB
:1051710012E52C127E4D78647C157D017BFF7A7AD5
:1051810079117E007F0D12E52C12D7B4E4FFFD12D8
:10519100D5189007F912E71790167012E7207BFFD8
:1051A1007A75793E12EDA190055CE4F0A37405F0E7
:1051B1007F0612B27A22E4FFFD12D51890080B1275
:1051C100E71790167012E7207BFF7A75793E12ED92
:1051D100A1900E5374FFF07F04122B2578FF7C0EF3
:1051E1007D017B017A0A79817E007F0D12E52C1207
:1051F1007E4D78647C157D017BFF7A7979EA7E00AA
:055201007F0D12E52CF9
:1052060012D7B4E4900562F0A3F090055CF0A374A5
:1052160005F07F0612B27A22900F11E060197B0129
:105226007A0F7913E4FD90054404F01234B17F0B34
:105236007D01122AB08024901575E060127B017AF8
:10524600157977E4FD90054404F01234B1800CE43E
:10525600FF7D0112D5187F2012D6AE900F10E064A4
:105266004560030253997F0B7D01122AB07F02121B
:10527600CFEE900F54E09006B2F0121FD67B017A63
:105286000F7913E4FD90054404F01234B17F057DD7
:1052960001122AB078E97C097D017B017A0F791326
:1052A60012EA4FE4FF12CFEE900984E0F4600A9010
:1052B6000A0AE0F460030253637B017A0979E9E4A0
:1052C600FDFC123320EF7003025351900CF1E0FE07
:1052D600A3E0FF122A1D900984E0F46024900A0AD4
:1052E600E0B4FF227B017A0979DC12F6167B017A9B
:1052F6000079007800C312E6C060069009DCE07011
:1053060005122A4280457B017A0979DC12F616EFEE
:1053160024FFFFEE34FFFEED34FFFDEC34FFFC907E
:10532600167312E6FF7BFF7A7579FA90167012E70C
:10533600207B017A0979DC12ED9B900CF1E0FEA34B
:10534600E0FF7B017A0979B31229E1E4900984F040
:10535600900A0AF090055CF0A37402F022900E53B6
:10536600E0B4FF2B7B017A0979E9E4FDFC123320D6
:10537600EF700302692C78B97C067D017B017A09FE
:1053860079E912EA4F90055CE4F0A3740AF0221260
:105396003C3122900F10E0B44E0C121FE790055CD2
:1053A600E4F0A37402F0901574E0644560030254BF
:1053B600D07F0212CFEE9006B27420F0121FD67B79
:1053C600017A157977E4FD90054404F01234B1783A
:1053D600E97C097D017B017A15797712EA4FE4FFB2
:1053E60012CFEE900984E07009900A0AE070030279
:1053F600549A7B017A0979E9E4FDFC123320EF70B7
:1054060003025488900CF1E0FEA3E0FF122A1D90DF
:105416000984E07023900A0AE060227B017A097908
:10542600DC12F6167B017A0079007800C312E6C01A
:1054360060069009DCE07005122A4280457B017AFD
:105446000979DC12F616EF24FFFFEE34FFFEED3489
:10545600FFFDEC34FFFC90167312E6FF7BFF7A75B6
:1054660079FA90167012E7207B017A0979DC12ED41
:105476009B900CF1E0FEA3E0FF7B017A0979B31261
:1054860029E1E4900984F0900A0AF090055CF0A303
:105496007402F022900E53E0B4FF2B7B017A097957
:0F54A600E9E4FDFC123320EF700302692C78B9A2
:1054B5007C067D017B017A0979E912EA4F90055C4A
:1054C500E4F0A3740AF022123C31227F0612B27A6C
:1054D5002290055CE0FFA3E0900E4BCFF0A3EFF028
:1054E5007F01122B2578FF7C0E7D017B017A0A79DD
:1054F500817E007F0D12E52C127E4D78647C157D32
:10550500017BFF7A7979C37E007F0D12E52C12D7D6
:10551500B4900E1FE0602A9006DCE024FFFF9006A1
:10552500DBE034FFFE122A1D78A47C0C7D017B0193
:105535007A0979B37E007F3412E52C9008F7740957
:10554500F090055CE4F0A37408F07F0612B27A22AD
:1055550090055CE0FFA3E0900E4BCFF0A3EFF07F4A
:1055650005122B2578FF7C0E7D017B017A0A798156
:105575007E007F0D12E52C127E4D78647C157D0131
:105585007BFF7A7979F77E007F0D12E52C12D7B46F
:10559500900E49E0601DE4FFFD12D5189008A41295
:1055A500E71790167012E7207BFF7A75793E12EDAA
:1055B500A18021900A92E0601BE4FFFD12D51890AE
:1055C500088C12E71790167012E7207BFF7A757921
:1055D5003E12EDA17F0612B27A90055CE4F0A37449
:1055E50008F022900F11E060127B017A0F791312F7
:1055F50035897F0B7D01122AB0805C901575E060BE
:105605000B7B017A157977123589804B900E4BE02B
:105615007004A3E06406700DFF7D0112D5187F208C
:1056250012D6AE8032900E4BE07004A3E064077092
:1056350026900E49E0600E7F067D0112D5187F2069
:1056450012D6AE8012900A92E0600C7F097D01129D
:10565500D5187F2012D6AE900F10E0644560030286
:1056650057717F0212CFEE7F057D01122AB0121FFE
:10567500D67B017A0F791312358990066DE06009A2
:105685007F067D0A7C0012B2DB122B8B900E4BE05D
:105695007004A3E064077024900E49E0601E7B014E
:1056A5007A0F791312F724900569EFF0E4900E490B
:1056B500F090055CF0A37402F002576B900E4BE07E
:1056C5007004A3E064077025900A92E0601F7B01D7
:1056D5007A0F791312F7249008F7EFF07004900A07
:1056E50092F090055CE4F0A37402F08079900E4B83
:1056F500E07004A3E06406706D7B017A0F791312E4
:105705003416EF700E121FE790055CE4F0A37406E3
:10571500F080537B017A0F7913123589900F13E0CE
:10572500701178CD7C0C7D017BFF7A76791012EAB9
:105735004F800F78CD7C0C7D017B017A0F79131298
:10574500EA4F7F087D02122AB0900E1FE0600A9092
:1057550006DB74FFF5F012E638E4900E1FF09005B5
:0B5765005CF0A37409F0E4FF12CFEE2B
:1057700022900F10E0B44E13121FE7900E4BE0FF83
:10578000A3E090055CCFF0A3EFF022901574E064E5
:105790004560030258A07F0212CFEE7F057D011203
:1057A0002AB0121FD67B017A1579771235899006B7
:1057B0006DE060097F067D0A7C0012B2DB122B8B44
:1057C000900E4BE07004A3E064077024900E49E053
:1057D000601E7B017A15797712F724900569EFF046
:1057E000E4900E49F090055CF0A37402F002589A20
:1057F000900E4BE07004A3E064077025900A92E0DD
:10580000601F7B017A15797712F7249008F7EFF083
:105810007004900A92F090055CE4F0A37402F080AA
:1058200079900E4BE07004A3E06406706D7B017A02
:10583000157977123416EF700E121FE790055CE4AD
:10584000F0A37406F080537B017A157977123589BD
:10585000901577E0701178CD7C0C7D017BFF7A7616
:10586000791012EA4F800F78CD7C0C7D017B017A94
:1058700015797712EA4F7F087D02122AB0900E1F29
:10588000E0600A9006DB74FFF5F012E638E4900E53
:105890001FF090055CF0A37409F0E4FF12CFEE2234
:1058A0007F0612B27A2278C57C0C7D017B017A12C8
:1058B000799A7E007F0812E52C900E29E070069000
:1058C0000CC97419F0900CF4E07006900CC5746467
:1058D000F0900561E06018900CF1E0FEA3E0FF7B22
:1058E000017A0C79A41229E1E4900561F0801B9003
:1058F00006DBE0FEA3E0FF7B017A0C79A41229E12C
:105900009006DBE475F00112E63890055CE4F0A344
:105910007402F022E49009E7F0900A0B74FFF09013
:105920000CF1E0FFA3E09006B6CFF0A3EFF0E49017
:105930000E15F0A3F012D90278647C157D017BFF6F
:105940007A7A79047E007F0D12E52C12D7B4900587
:105950005CE4F0A3740BF02290055CE0FFA3E09000
:105960000E4BCFF0A3EFF0900E37E0600F7BFF7A85
:1059700077794112EDA17F0612B27A22900F10E0E2
:1059800064456003025AF0121FD678137C0F7D0124
:105990007BFF7A77796412E966EF601578137C0FE4
:1059A0007D017BFF7A77796812E966EF6003025A1E
:1059B0002E7F0212CFEE7F057D01122AB09006B62F
:1059C000E0FFA3E0900CF1CFF0A3EFF0122A42E445
:1059D000FF12CFEE9006DBE0FEA3E0FF900CF1E0BB
:1059E000B5060FA3E0B5070A9006B674FFF5F012EE
:1059F000E638EF4E7011900A0BF0900E37F09005DC
:105A00005CF0A37402F0229006B6E0FEA3E0FF1261
:105A10002A1D12D90278647C157D017BFF7A7A7980
:105A2000047E007F0D12E52C12D7B4025AF07813D1
:0A5A30007C0F7D017BFF7A77796C13
:105A3A0012E966EF701B7F0212CFEE7F057D01121D
:105A4A002AB090055CE4F0A37404F0E4FF12CFEEF0
:105A5A002278137C0F7D017BFF7A77797012E966D1
:105A6A00EF70657B017A0679B9900563E02401FD40
:105A7A00900562E03400FC123320EF602D7F0212A1
:105A8A00CFEE7F057D01122AB0900CF1E0FEA3E073
:105A9A00FF122A1D900CF1E0FFA3E09006B6CFF0AA
:105AAA00A3EFF0E4FF12CFEE803C7F057D01122ABE
:105ABA00B078647C157D017BFF7A7A79047E007F59
:105ACA000D12E52C12D7B4227F057D01122AB07877
:105ADA00647C157D017BFF7A7A79047E007F0D1242
:105AEA00E52C12D7B422900E15E0FEA3E0FFEE607B
:105AFA0003025BEFEF14605E147003025B9714708D
:105B0A0003025BC624036003025BEF7BFF7A7779AB
:105B1A00749006B7E02401901671F09006B6E0344E
:105B2A0000901670F012EDA17B017A0979B3E4FDB9
:105B3A0090054404F01234B17F04122B2578FF7CBF
:105B4A000E7D017B017A0A79817E007F0D12E52C98
:105B5A00127E4D025BEF7BFF7A7779869006B7E07B
:105B6A002401901671F09006B6E03400901670F099
:105B7A009009D6E0901672F09009D5E0901673F06D
:105B8A009009D4E0901674F012EDA180587BFF7A48
:105B9A007779AA9006B7E02401901671F09006B6BC
:105BAA00E03400901670F09009D8E0901672F090E8
:105BBA0009D9E0901673F012EDA180299006B7E09A
:105BCA002401901671F09006B6E03400901670F039
:105BDA007B017A0979DC90167212E7207BFF7A77CB
:105BEA0079C812EDA17F0612B27A227F06122B25FE
:105BFA0078FF7C0E7D017B017A0A79817E007F0D18
:105C0A0012E52C127E4D90055CE4F0A3740DF07F32
:105C1A000612B27A22900F10E064457044127FE6B1
:105C2A007F057D327B0112C33178E97C097D017BD6
:105C3A00017A0F791312EA4F90099512E717A80112
:105C4A00AC02AD037B017A0979E912E966EF7004C7
:105C5A001236B9221209FF90055CE4F0A3740CF025
:105C6A0022900F10E0B44E1F127FE67F057D327B33
:105C7A000312C3317F067D147C0012B2DB90055CEF
:105C8A00E4F0A3740CF0227F0612B27A229006DBAB
:105C9A00E0FCA3E0FD9008D5E0FEA3E0FFC39DEC85
:105CAA006480F8EE6480984003025DFB122A1D901E
:105CBA000A80E0603C146073147003025D6814701B
:105CCA0003025DA924046003025DD3900A80E00404
:105CDA00F07BFF7A7779DD90167012E720900E1C20
:095CEA00E0901673F07B017A0BC7
:105CF30079A512ED9B025DD3900A80E004F0900930
:105D0300D4E0FF6464602B7BFF7A7779E3901670AD
:105D130012E7209009D6E0901673F09009D5E09031
:105D23001674F0A3EFF07B017A0B79A512ED9B02B9
:105D33005DD3900A80E004F09009D8E0FF64196015
:105D4300247BFF7A7779F590167012E7209016730B
:105D5300EFF09009D9E0901674F07B017A0B79A5E6
:105D630012ED9B806B78A57C0B7D017B017A097911
:105D7300B312EA4F7B017A0979DC12F601EF4E6028
:105D830008900A80E004F08047900A7FE06005E411
:105D9300A3F08006900A8074FFF09008D5E475F0B4
:105DA3000112E638802A78A57C0B7D017B017A09F4
:105DB30079DC12EA4F900A7FE06005E4A3F08006E5
:105DC300900A8074FFF09008D5E475F00112E6386C
:105DD3007B017A0B79A512F601900A95EFF0E0FFAB
:105DE30004F074A52FF582E4340BF583740DF012DF
:105DF3003FAB7F0612B27A22E4FF127C24900E306E
:105E0300E0700302692C121FC622900CD9E06003D4
:105E130002692CE4900A91F0900E27F0900AA3F007
:105E230090055CF0A37410F07F0612B27A22E4FFAF
:105E3300127C24E4900E36F0900E0FE0700690086A
:105E4300D4E0600E7B017A0A79A6900A91E0FD12F4
:105E53002C49900E0FE060189006A8E0FF9006E230
:105E6300E0B5071E9006A9E0FF9006E3E0B5071230
:105E73009008D4E060309006A8E0FF9006E2E06F5F
:105E83006024900937E0900BA5F0900A957401F017
:105E9300E4900AA2F0900A91F0123FAB90055CE403
:105EA300F0A37411F0221245C790056BEFF012E7CF
:105EB300B25ED6015ED6025ED6035ED6045ED6051A
:105EC3005FC4065FD6075FEB0860610960750C006D
:105ED30000608990056BE064057051900567E024CC
:105EE300A7F9E4340AFA7B019016C812E72090164A
:105EF300CBE4F0A37405F07A05796C12F5997B0174
:105F03007A05796C12F724900E2BEEF0A3EFF09044
:105F130006DBE0FCA3E0FDD3EF9DEC6480F8EE64C8
:105F230080984008900E2BECF0A3EDF07FFF127CDD
:105F330024C39006DCE094E79006DBE0648094835E
:105F4300401178F67C0C7D017BFF7A78790112EAA7
:105F53004F80247BFF7A78791290167012E7209095
:105F630006DBE0FFA3E0901673CFF0A3EFF07B0115
:105F73007A0C79F612ED9B9008D5E475F00112E6E0
:045F83003890056BE2
:105F8700E0FF64036004EFB404119006DBE07002E5
:105F9700A3E070079008D5F0A304F0900E4AE060E4
:105FA70009900AA374FFF00260897B017A0C79F6E5
:105FB70012438090055CE4F0A37412F02278F67C1B
:105FC7000C7D017BFF7A78792412EA4F0260897889
:105FD700F67C0C7D017BFF7A78792A12EA4F121F33
:105FE700C6026089D39006DCE094009006DBE0648B
:105FF7008094804054E4900559F0A3F0900E2BE074
:10600700FEA3E0FFC390055AE09F900559E09E501C
:1060170027D39006DCE094009006DBE06480948050
:106027004016E4900CF1F0A3F0122A42900559E4CF
:1060370075F00112E63880C478F67C0C7D017BFF91
:106047007A78793012EA4F803978F67C0C7D017BBB
:10605700FF7A7479F112EA4F802878F67C0C7D017B
:106067007BFF7A78793012EA4F121FC6801478F6D0
:106077007C0C7D017BFF7A78793612EA4FE4900E2B
:1060870027F090056BE0640B60097B017A0C79F6C9
:10609700124380E4900A91F090055CF0A37411F02C
:1060A7007F0612B27A227F0612B27A2290056BE03F
:1060B70014700302617C24FE70030261FF147003F5
:1060C7000261FF1470030262532403600302692C08
:1060D7009008D5E07002A3E0700C7BFF7A78793CDA
:1060E700122BDA0261789008D5E07004A3E064010E
:1060F70070639006DBE0FEA3E0FFC3900A94E09F85
:10610700FF900A93E09EFE3395E0FDFC9009001294
:10611700E6FF90090012E6E77B347A007900780001
:1061270012E67190090012E6FF7BFF7A78794D90AD
:10613700167012E72090090012E6E790167312E630
:10614700FF7B017A05796C12ED9B7B017A05796CEF
:10615700122BDA801C9008D5E07004A3E06402706B
:106167000A7BFF7A7479F1122BDA227F0612B27A50
:1061770022122BCD229006DBE0FCA3E0FD9008D590
:10618700E0FEA3E0FFC39DEC6480F8EE64809850C6
:1061970018122CF07B017A0C79F61243809008D5FF
:1061A700E475F00112E638804B9006DBE0FEA3E0D1
:1061B700FF9008D5E0B50610A3E0B5070B7BFF7A83
:1061C70078795C122BDA802C9006DCE02401FF90B2
:1061D70006DBE03400FE9008D5E0FCA3E0B5070E2F
:1061E700EEB5040A7BFF7A7479F1122BDA227F0667
:1061F70012B27A22122BCD229008D5E0FEA3E0FF3F
:106207004E7029122CF07B017A0C79F6124380E448
:10621700900CF1F0A3F090056BE0B40303122A424F
:106227009008D5E475F00112E638801C9008D5E097
:106237007004A3E06401700A7BFF7A7479F1122B72
:0B624700DA227F0612B27A22122BCD61
:1062520022900E2BE0FCA3E0FD9008D5E0FEA3E027
:10626200FFC39DEC6480F8EE6480985018122CF005
:106272007B017A0C79F61243809008D5E475F0011F
:1062820012E6388024900E2BE0FEA3E0FF9008D5A2
:10629200E0B5060FA3E0B5070A7BFF7A7479F11225
:1062A2002BDA227F0612B27A22122BCD2290056BB4
:1062B200E0640B60097B017A0C79F6124380900549
:1062C2005CE4F0A37411F022E4900A91F0122BBB6B
:1062D20090055CE4F0A37417F07F0612B27A229064
:1062E20008D574FFF5F012E63890055CE4F0A3746B
:1062F20017F0227E007FFF7D007B017A0C79F61277
:10630200EC1B9006DBE0FEA3E0FF9008D5E0FCA3C7
:10631200E0FDC39FEE6480F8EC6480984003026461
:106322000CEDF47002ECF470717B017A1279AE908C
:1063320016C812E7209016CBE4F0A37402F07A0A92
:10634200799D12F5997B017A1279B19016B612E70E
:10635200209016B9E4F0A37402F07A0A799D12F43F
:106362006CE4900AA1F07BFF7A7879629016701241
:10637200E7209016737402F07B017A0A799DA312CA
:10638200E7209016777417F07A0C79F612ED9B904D
:10639200066C74FFF0122E058030E490066CF090CB
:1063A20006DCE024FFFF9006DBE034FFFE9008D518
:1063B200E0B5060BA3E0B50706900CDB74FFF09086
:1063C20008D5E0FEA3E0FF122E9A9008D5E475F0FE
:1063D2000112E6389006DBE07002A3E07006900836
:1063E200D5F0A3F0E4900A91F07B017A0C79F612D1
:1063F2004558900560E0600302692C900E2DE0FF85
:106402007D527B647A0012B6C822E4FF127C24908B
:10641200098374FFF0FB7A78797312EDA190055C21
:10642200E4F0A3740FF02290055CE0FFA3E0900E6D
:106432004BCFF0A3EFF0900E1DE060097BFF7A785E
:10644200799612EDA17F06122B2578FF7C0E7D0135
:106452007B017A0A79817E007F0D12E52C127E4D36
:1064620090055CE4F0A37419F022900F10E06445EB
:1064720060030265257F057D01122AB078E97C0957
:106482007D017B017A0F791312EA4F78E97C097D4D
:106492000190090412E71712E966EF703F127FE6D6
:1064A2007F087D02122AB0122B8BE4900672F0D381
:1064B2009006DCE094009006DBE064809480401259
:1064C2007BFF7A7879B912EDA17F067D287C0012D4
:1064D200B2DB90055CE4F0A37402F0227BFF7A78D1
:1064E20079DC90167012E7207B017A0979E990161F
:1064F2007312E7207A0C79A412ED9B9006DBE0FE82
:0F650200A3E0FF7B017A0C79A41229E19006DB5C
:10651100E475F00112E638127FE690055CE4F0A321
:106521007418F022900F10E0B44E0D121FE7900581
:106531005CE4F0A37418F0227F0612B27A2290066E
:10654100E17401F0E49008D5F0A3F0900998F0907F
:106551000AA5F0900CEDF07BFF7A7879E012EDA1BD
:10656100122C3122E4900E22F0900CF5F0FFFD1276
:10657100D5187BFF7A79790312EDA1900AAAE0641C
:10658100317062900998E0705CD39006DCE0940071
:106591009006DBE06480948040477BFF7A79791430
:1065A10012EDA1900E1B74FFF0FF127C249008D510
:1065B100E0FEA3E0FF122CF09008D5E475F0011283
:1065C100E6389006E1E004F0786C7C057D017B0102
:1065D1007A0C79F612EA4F90055CE4F0A3741CF092
:1065E10022122C3122900AA8E064357060900E1DB1
:1065F100E07027900E2274FFF0786C7C057D01FB22
:106601007A7679A212EA4F7BFF7A79792612EDA187
:1066110090055CE4F0A3741CF0227FFF127C2490AF
:1066210008D5E0FEA3E0FF122A1D786C7C057D01F0
:106631007B017A0979B312EA4F9008D5E475F0012C
:1066410012E63890055CE4F0A3741CF022900AA9CC
:10665100E0B42324900998E0701E900CF574FFF0CB
:10666100786C7C057D01FB7A7679A812EA4F90055A
:106671005CE4F0A3741CF022122C31227E007FFF17
:106681007D007B017A0B79A512EC1B78A57C0B7D33
:10669100017B017A09798D12EA4F7B017A05796CC8
:1066A1009016AD12E7207A0B79A512F4017B017ADD
:1066B1000B79A512F601900A95EFF0FD24A5F5825C
:1066C100E4340BF583740DF07B017A0B79A5122C60
:1066D100499006A8E0FF900A95E004F024A5F58210
:1066E100E4340BF583EFF0900A95E004F024A5F56E
:1066F10082E4340BF583740AF0900A95E004F0E427
:10670100900AA2F0900A91F012400F900E1DE070D5
:106711000A90055CF0A3741DF0800990055CE4F01B
:10672100A3741EF07F0612B27A22900E22E0700648
:10673100900CF5E06004122C3122900CEDE07074A5
:106741009006DBE0FCA3E0FD9008D5E0FEA3E0FFAE
:10675100C39DEC6480F8EE648098503F9006E1E0C0
:10676100D39464502C122CF0786C7C057D017B0154
:106771007A0C79F612EA4F9008D5E475F00112E629
:10678100389006E1E004F090055CE4F0A3741CF09D
:106791002290055CE4F0A37421F022900AA5E07038
:1067A1000990055CF0A37420F02290055CE4F0A34D
:1067B1007421F0229006DBE0FEA3E0FFC39008D62F
:1067C100E09FEE6480F89008D5E06480984024E46E
:1067D100FF127C247F087D02122AB0E4900CEDF0B8
:0367E100900AA576
:1067E400F090099874FFF0E4900E1BF0122C312203
:1067F400E4900CEDF0FF127C24122C3122900AA5B7
:10680400E0603D900CEDE0700990055CF0A374210C
:10681400F022E4FF127C247F087D02122AB0E49067
:106824000CEDF0900AA5F090099874FFF0E4900E36
:106834001BF0900E1DF09006DBF0A3F0122C312219
:106844009006DBE0FCA3E0FD9008D5E0FEA3E0FFAA
:10685400C39DEC6480F8EE6480985026122A1D785B
:106864006C7C057D017B017A0979B312EA4F9008AB
:10687400D5E475F00112E63890055CE4F0A3741CCD
:10688400F022E4900CEDF090055CF0A37420F0226B
:106894007F0B7D327B0112C3319006E17401F0E479
:1068A4009008D5F0A3F0900998F0900AA5F0900C08
:1068B400EDF07BFF7A79793812EDA1122C31229018
:1068C4000AA574FFF0E49006E1F090056C7417F0EB
:1068D400E4A3F090055CF0A3741CF022900CED741A
:1068E400FFF0E49006E1F09006DBE0FEA3E0FFC3D6
:1068F4009008D6E09FEE6480F89008D5E064809814
:10690400400690099874FFF0E4900E1BF090056C1B
:106914007404F0E4A3F090055CF0A3741CF02290DE
:09692400055CE4F0A37402F0220A
:10692D009012AFE0900960F09012AEE090095FF028
:10693D009012B2E090095DF09012B1E090095CF018
:10694D009012B5E090096CF09012B4E090096BF0E4
:10695D009012A5E0900963F09012A4E0900962F006
:10696D009012A8E0900966F09012A7E0900965F0EA
:10697D009012ABE0900969F09012AAE0900968F0CE
:06698D007F0712B27A221E
:0100120022CB
:01001A0022C3
:10262E0060460E6801000101010101000000000179
:10263E000100000101010001010001000101010181
:10264E000101000001010001010001010001010171
:10265E000101010001010000000101010101010160
:10266E000101010101000101010160460EAE0101EF
:10267E000101000101000000010001000001010044
:10268E000101010000010101010101000001010130
:10269E000001000101010001010101010100010120
:1026AE000000010001010101010101010101000110
:0426BE000101010114
:01001E0022BF
:107A1E00900E55EBF0A3EAF0A3E9F07F557D081226
:107A2E00D518900E55E0FBA3E0FAA3E0F912E55548
:107A3E007016900E58F0E4FF12D261900E58E004CA
:107A4E00F0E0C3941C40EF22900E55E0FBA3E0FA49
:107A5E00A3E0F912E55524D0900E5AF090000112D1
:107A6E00E56E24D0900E5BF090000312E56E24D0EC
:107A7E00900E5CF090000412E56E24D0900E5DF036
:107A8E00E4900E58F0E4900E59F0900E59E0FFC3BA
:107A9E0094074003027B40900E58E0FE600464029F
:107AAE007052EE7009EF7006900E59E004F0EE7011
:107ABE000C900E5AE07006FF12D261806C900E5838
:107ACE00E0245AF582E4340EF583E075F007A42421
:107ADE0068F582E4340EF583C083C082900E59E0BF
:107AEE00D082D0832582F582E43583F583E0FF12C0
:107AFE00D2618035900E58E0245AF582E4340EF5AA
:107B0E0083E075F007A424AEF582E4340EF583C04D
:107B1E0083C082900E59E0D082D0832582F582E414
:107B2E003583F583E0FF12D261900E59E004F00226
:107B3E007A98900E58E0B401057F0112D261900E32
:0E7B4E0058E004F0E0C394045003027A93223E
:107B5C00900E5EEFF07F107D0812D518900E5EE04F
:057B6C00FF12D26122AE
:107B7100900E5FEBF0A3EAF0A3E9F07F207D0812FD
:107B8100D518900E5FE0FBA3E0FAA3E0F912E555EA
:107B9100FF12D261900E5FE0FBA3E0FAA3E0F9903F
:107BA100000112E56EFF12D261900E5FE0FBA3E0CF
:0F7BB100FAA3E0F990000212E56EFF12D26122F2
:107BC000900E62EBF0A3EAF0A3E9F07F2E7D08129D
:107BD000D518900E62E0FBA3E0FAA3E0F912E55598
:107BE000FF12D261900E62E0FBA3E0FAA3E0F990ED
:107BF000000112E56EFF12D261900E62E0FBA3E07D
:107C0000FAA3E0F990000212E56EFF12D261900E25
:107C100062E0FBA3E0FAA3E0F990000312E56EFF37
:047C200012D26122F9
:107C2400900E65EFF07F3D7D0812D518900E65E04B
:057C3400FF12D26122E5
:107C3900900E66EFF07F517D0812D518900E67748B
:107C490003F0900E67E0FFD39400401C900E66E0AD
:107C5900C39F50077F0112D2618005E4FF12D261F0
:107C6900900E67E014F080DA900E66E0C394045039
:0D7C7900067F0112D26122E4FF12D26122C7
:107C860012D2A9900EFBE04401F054F9F012D2A3EF
:067C960012D2A0D29C22D4
:0E7C9C00900EFBE04402F054F9F012D29B224D
:107CAA00900EF8E0A3E0FAA3E0F912E7D8C299220D
:107CBA00900EF4EBF0A3EAF0A3E9F012D2A9900E29
:107CCA00F4E0F9A3E0FAA3E0900EF8C9F0A3EAF011
:107CDA00A3E9F0A3E04408F054EFF012D2A0127C1A
:027CEA00AA22CC
:0E7CEC00900EFBE04410F054F7F012D29B22F1
:087CFA00900EFBE04404F022AF
:107D0200900EFBE0900EF7F054FBFF900EFBF0227A
:067D1200E4900EFBF022DC
:087D18006203060409303B0080
:0C8AE6002573002D24252B00256275004F
:107D20007E007F287D007B017A0F798612EC1BE4B0
:077D3000782FF6782DF622F2
:107D3700900F85E0FF7D49E4FBFA12B6C8E4FF1215
:0E7D4700D1E1900FAEE0F55AAF5A12CFEE2206
:0A7D5500127D3712C4A5127D202212
:0C7D5F001283FF127D37E4FF12B27A227B
:0F7D6B00900FAEE55AF0E4FF12B219127D2022FC
:107D7A00782EE624FB7003027E0C147003027E3B0D
:107D8A0024056003027E4812C69F4003027E4C907F
:107D9A000FAEE55AF0E4FF12CFEE12C4A5900F859C
:107DAA00E0FF7D527B507A0012B6C8782E76057FA6
:107DBA000112D1E190107EE0547824F0601A24F088
:107DCA00602424E0602E243870787F0112CFEEE41C
:107DDA00FF7D05FC12B2DB227F0112CFEEE4FF7DAC
:107DEA000AFC12B2DB227F0112CFEEE4FF7D14FC03
:107DFA0012B2DB227F0112CFEEE4FF7D1EFC12B22B
:107E0A00DB2290107EE054786005E4FF12CFEE1278
:107E1A008402900F85E0FF12B773BF4507782E766C
:107E2A0006127D5512C69F4019782E7601127D558D
:107E3A002212C69F400C782E760112C4A522782EF3
:037E4A007601229C
:107E4D00900F01E0FFD394405022900F00E0D39F9C
:107E5D00501A900EFFE0D394475011900F02E0D3CB
:107E6D0094075008A3E014D39403400A7F357D0195
:107E7D00E4FBFA12C3AA787E7C107D017B017A0E99
:107E8D0079FF7E007F0D12E52C901082E0FE1460CC
:107E9D003C1460281460141470469010397442F02C
:107EAD00E4A3F090103CF090107DF0900FF474422C
:107EBD00F0E4A3F0900FF7F0901038F0900FAF743E
:107ECD0042F0E4A3F0900FB2F0900FF3F0900F108A
:107EDD007442F0E4A3F0900F13F0900F54F0800B68
:107EED007F357D02EEFB7A0012C3AA901085E0FB70
:107EFD00A3E0FAA3E0F912E5556029901083E0FFA5
:107F0D00A3E0FD12D518901085E0F9A3E0FAA3E0E7
:107F1D00901670C9F0A3EAF0A3E9F07BFF7A8A7995
:107F2D00E612EDA1C24E901088E0FBA3E0FAA3E0AB
:107F3D00F912E5557003027FE2901082E064016052
:107F4D0003027FE212F601900F0CEFF0901080E02B
:107F5D00FEEFD39E500D90107FE0FF900F0CE0C30D
:107F6D009F500E7F357D03900F0CE0FB7A0012C3FE
:107F7D00AAE4900F0DF0900F0CE0FFA3E0FEC39F5D
:107F8D005035901088E0FBA3E0FAA3E0F98E8275DE
:107F9D00830012E56EFF901081E0FD12C5E8EF70D1
:107FAD000E7F357D04900F0DE0FB7A0012C3AA9071
:107FBD000F0DE004F080BF900F0CE0900F11F078E2
:107FCD00137C0F7D01901088E0FBA3E0FAA3E0F98C
:097FDD0012EA4FD24E127D6B2214
:107FE600900F107444F0900FAFF0900FF4F09010D3
:0C7FF60039F0900FAEE55AF0127D5F22CA
:10800200EF24BFFFC394105016EF75F003A424555C
:10801200F582E4340FF583EBF0A3EAF0A3E9F02252
:10802200124A54900403E07865F66006E6D3944061
:10803200400D7F377D017865E6FB7A0012C3AA788E
:1080420065E6B4041978047C047D017BFF7A8A79A1
:10805200E912E966EF7007FF12D1E112C5CBE478AD
:1080620068F67865E664037074900404E064247032
:108072006C90107EE030E032901082E06401702A51
:10808200900405E0FF12F38D5010900406E0FF12F9
:10809200F38D5006786876018010900405E0B425CF
:1080A20009A3E0B4250478687603900405E0FFB4E0
:1080B2002B12A3E0B42D0D901082E0B40106786873
:1080C2007602801990107EE030E212EFB42B0E900F
:1080D2000406E0FF12F38D5004786876047868E6AF
:1080E2001470030282B614700302834D14700302EB
:1080F200836A147003028384240460030283A790BA
:10810200107EE030E1030283A7E47867F690107FE7
:10811200E0FF7865E6FEC39F400CA3E0FFEED39F2D
:108122005004786776FFE47866F67866E6FFC3184F
:108132009650257867E6B4FF1F74042FF582E43465
:1081420004F583E0FF901081E0FD12C5E8EF7003B3
:108152007867F678660680D27867E6705690108265
:10816200E0FE146030146020146010147036901019
:1081720039744EF0E4A3F090103CF0900FF4744E7A
:10818200F0E4A3F0900FF7F0900FAF744EF0E4A379
:10819200F0900FB2F0900F10744EF0E4A3F0900F35
:1081A20013F0800B7F377D02EEFB7A0012C3AA1216
:1081B2007D5F22782DE6702A7865E6900F11F02413
:1081C20001FFE433FE78137C0F7D017B017A047991
:1081D2000412E52C900402E0900F54F0782D060270
:1081E2008271782DE6640170297865E6900FB0F00F
:1081F2002401FFE433FE78B27C0F7D017B017A0417
:10820200790412E52C900402E0900FF3F0782D0629
:10821200805D782DE6640270297865E6900FF5F0AE
:108222002401FFE433FE78F77C0F7D017B017A04A1
:10823200790412E52C900402E0901038F0782D06B3
:10824200802D782DE6B403277865E690103AF02465
:1082520001FFE433FE783C7C107D017B017A0479D6
:108262000412E52C900402E090107DF0782D069027
:108272001082E0FE782DE6C39E50030283A7EE141F
:10828200601B14601214600914701A90103974453E
:10829200F0900FF47445F0900FAF7445F0900F100A
:1082A2007445F0800B7F377D03EEFB7A0012C3AA80
:1082B200127D5F22304E14E4900F11F0FE7F41FDDB
:1082C2007B017A0F791312EC1BC24E901080E0FFF3
:1082D200900F11E0C39F40030283A790169874FF8A
:1082E200F0A3748AF0A374EEF0A3E4F0A37400F098
:1082F200A37469F07B017A04790512F115BEFF12AD
:10830200BFFF0F7F377D047869E6FB3395E0FA12F1
:10831200C3AA7869E6FF901081E0FD12C5E8EF700C
:06832200030283A7786945
:10832800E6FF900F11E0FE04F074132EF582E4349A
:108338000FF583EFF0900F11E02413F582E4340F6A
:10834800F583E4F02290107FE0FF900F11E0C39FC7
:10835800404D127D5F900F107445F0900F5474F0EB
:10836800F022900F11E0D394004034E014F024136D
:10837800F582E4340FF583E4F0C24E22127D5F905B
:108388000406E0540F7869F675F003A42455F582C5
:10839800E4340FF583E0A3E0FAA3E0F912E7D8226A
:1083A800900403E06050E4FF782FE6FEEFC39E5090
:1083B80020EF25E02486F582E4340FF583E0FCA362
:1083C800E0FD900400E06C7003A3E06D60280F806E
:1083D800D7EEC39414501F900400E0FCA3E0FDEF17
:1083E80025E02486F582E4340FF583ECF0A3EDF064
:0783F800128022782F0622FB
:10879200AE07EE14B41B0040030288799087A5F857
:1087A2002828730287F60287FC02880102880602E3
:1087B200880B02880E028813028816028819028822
:1087C2001C02887902881F02882202882702882ACE
:1087D20002882D02883802884302884E0288590294
:1087E200886002886702886C028871028879028731
:1087F200F9028876D20822D20722D210D20822D2D7
:108802000DD20822D241D20822D20922D209D20E96
:1088120022D21A22D21922D20B22D20B22D21E2209
:10882200D20CC23122D21122D20A22D20AD212C2CE
:1088320016C215C21722D20AD217C216C215C21206
:1088420022D20AD216C217C215C21222D20AD215D7
:10885200C217C216C21222D20AD213C21422D20ADA
:10886200D214C21322D20AD24322D20AD24422D230
:108872000AD21C22D231227F387D01EEFB7A00120D
:03888200C3AA2264
:10888500AE07EE14B41B004003028949908898F89E
:108895002828730288E90288F30288F60288F9021B
:1088A50088FC02890102890402890702890A028972
:1088B5005402894902890D02891002891302891619
:1088C50002892B02892E02893102893402893702F5
:1088D500893A02893D028940028943028949028811
:1088E500F0028946C210C20DC24122C20722C2103F
:1088F50022C20D22C24122C209C20E22C20E22C2CA
:108905001A22C21922C20B22C21E22C20C22C21175
:1089150022C20AC212C217C216C215C213C214C29B
:1089250043C244C21C22C21222C21722C21622C24C
:108935001522C21322C21422C24322C24422C21CDF
:1089450022C231227F397D01EEFB7A0012C3AA22B1
:10895500AE07EE24FB601624FD601514601B24FD94
:10896500601124FD6010240E7012D20022D2012263
:10897500D20222D20422D20522D246227F3A7D019A
:08898500EEFB7A0012C3AA22E6
:10898D00AE07EE24FB601624FD601514601B24FD5C
:10899D00601124FD6010240E7012C20022C201224B
:1089AD00C20222C20422C20522C246227F3B7D01A1
:0889BD00EEFB7A0012C3AA22AE
:1089C500304C09900F0EE0FF12879222900F0EE0B7
:0589D500FF128885225D
:1089DA00304D09900F0FE0FF12895522900F0FE0DA
:0589EA00FF12898D223F
:1089EF00C216C215C20DC210C214C213C212C20BDC
:1089FF00C20AC209C208C211C218C21EC21DC219C0
:108A0F00C21AC20CC20FC20EC217C207C246C2059B
:108A1F00C204C203C202C201C200C244C243C24165
:058A2F00C231C21C224F
:108A3400900F107444F0E4A3F0900F54F0FE7F41C3
:108A4400FD7B017A0F791312EC1B900FAF7444F085
:108A5400E4A3F0900FF3F0FE7F41FD7B017A0F79E0
:108A6400B212EC1B900FF47444F0E4A3F0901038AD
:108A7400F0FE7F41FD7B017A0F79F712EC1B901019
:108A8400397444F0E4A3F090107DF0FE7F41FD7B47
:108A9400017A10793C12EC1BE4FFEF75F003A42477
:108AA40055F582E4340FF58374FFF0A37400F0A34A
:108AB4007422F00FEFB410E21289EFD24C900F0E33
:108AC4007401F01289C5D248E4FFFE12B664900F17
:108AD40085EFF0127D20782E7601E4F55A900FAEE2
:028AE400F0227E
:05002600782E76012296
:1083FF00D24922E4C232755600753F0075400075B0
:10840F003401E4F50EF50F1284F51284272096033C
:10841F00D534EF7400F54822C234D247850E358526
:10842F000F367A1112861F85830E85820F8B128A63
:10843F001330D2030284BBC226C227C224C232C267
:10844F0020C223C242C221C225C21FC222C245126C
:10845F008AF22020301296DF20232A128FDB202170
:10846F00241292A120251E129456201F18129BE051
:10847F00202712129E9720240C12A32120320612BD
:10848F00A64130220BC2491284BC1283A820491C7A
:10849F00851083851182A3E0601285108385118278
:1084AF0085830E85820F74FFF0028427227F01756A
:1084BF00A003A831900400E4FCFEE549FD900404FC
:1084CF00E220E70BF06DFDE02EFE0CA30880F1E437
:1084DF00F0900400EDF0A3EC2EF0A3E549F0A3EC2F
:1084EF00F0C375A000225389F0438902758AFF7586
:0B84FF008CFF900000D28CC22CE534F2
:10850A00A2B392287F028011E540C3953F92D650CC
:10851A0001F4B401004002E53430280F1285E94025
:10852A00171285D31285D9502B800D1285D9400890
:10853A001285D31285E9501C0285BBC2AFC58A7564
:10854A008C00A28DC28D13F0D2AFA3E583B40302CF
:10855A00805FB22CE4202C2B20281430B2DD308D21
:10856A0003758CFF30B2D420964720B3EE803D309D
:10857A00B2C9308D03758CFF30B2C020963330B348
:10858A00EE802920281420B2B2308D03758CFF208A
:10859A00B2A920961C20B3EE801220B29E308D0321
:1085AA00758CFF20B29520960830B3EE209602DF34
:1085BA00028004B228809DC28CE58230E00474FFF8
:1085CA00F0A374FFF0A3E4F02274E2D5E0FD227870
:1085DA0028790030B319209614D9F8D8F6800E7885
:1085EA0028790020B309209604D9F8D8F6D322C3F3
:1085FA00227850790030B3F7D9FBD8F980EF785058
:10860A00790020B3EAD9FBD8F980E20582D5820243
:10861A001583158222853583853682E58230E0010D
:10862A00A3E0A3AB82AC8370030286C40460163055
:10863A00480CB4640040071286DC607E40078B82D7
:10864A008C83A380DC8B828C837D007E00E0606A51
:10865A00047007E58230E03C8032F930482EB46479
:10866A00004029E58220E024BE0013BD0600500E1A
:10867A00C083C082E91286DCD082D083800C940643
:10868A00F58250021583E91286D64008A30DBD0073
:10869A00010E80B9BE0009EDB5020050030286251D
:1086AA00304708C2478583108582118C838B828C60
:1086BA00358B36AB06AA05C2D222128615E07003A4
:0686CA00128615858310E5
:1086D000858211D2D22278FFD2D58002C2D575F020
:1086E0000A84F975F0067FFFE0A36020B50700500B
:1086F00001FF30D50A15F0E0A3B500005001F8D510
:10870000F0E6EF30D50328C313B50100227006F45C
:10871000FAFBD2D222BB0008CAFD7C007E00801882
:10872000AC02FAE4CBFD7E08ED20E70CC3EB33FB93
:10873000EC33FCED33FDDEF18AF0846017ADF02BF5
:10874000FBBE00E48011D3EB33FBEC33FCED33C311
:108750009AFDDED5BE00EFEAC313B50500AA03AB50
:1087600004EDC2D222202A0B855383855282E55123
:10877000F0801E8583538582527AFFA3A3E0B50261
:10878000005001FADBF5855383855282E0F551EA0A
:02879000F022D5
:108AF200A208720D72417207400122AB12AA13BB87
:108B02000006BA1300500122850F39850E380ABAC1
:108B120000010B740A12870D6005128F7040E8EA9B
:108B2200B44200505CB40300405714F54914F5599F
:108B3200755063304803755034D229D22A753101F9
:108B4200753C0075572A300703755724128BFB407A
:108B520030128CB1B42A04F557803FB55702803ADF
:108B6200129B74E54703F547128CB1B42A04F557FA
:108B72008003B5570CC22975315F74BC129ABC8050
:108B8200198084128BFB40F9128CB160F4D5490232
:108B92008014129ABCB5570280E7E539240AF539E8
:108BA2005002053880DDB557D830290A74BC129AB4
:108BB200BC75310180020531E557B42A028009757E
:108BC20049E9A207402E802D754910128FC2502408
:108BD200D220300D0E128E0B20D51A304105128F85
:108BE200245012128D30400D128D90754910303480
:108BF20003754911C3B3922022302A0F7B031287D7
:0F8C020065304807C333B5510040737F09D22C4A
:108C1100129AEB406AE0FAE54DC313B50200505FCA
:108C2100853982853883AF4AAE4B129BA54050F5FA
:108C310042AF4CAE4D129BA54045F541128C8A4086
:108C41003E853883853982D22CE4FAFBF5437F09CE
:108C5100E0202C09B54100B3EA33FA800BB542009C
:108C6100B350020543EB33FBA3B22CDFE38A478BFE
:108C710046202908129B74E54703F547C38001D3B9
:108C8100302A05C22A12876522AA4AAB4B75F00524
:108C910012AA714017AA4AAB4CEAB503004002CBB5
:108CA100CAEA75F003842AB503004002C322D32225
:108CB100AB47EB30D077E5437007EBF4540FFB8003
:108CC1001FB40269E54AB54C004006AC4CAD4A8080
:108CD10004AC4AAD4CECC3132C4005B50500404D26
:108CE1007A00EBC3134006CA240DCA80F6703EE534
:108CF10046C2E42A2402838035244B52514F4E54FC
:108D01007E4D4C537E502F41484745444A7E434255
:108D1100497E462B3138373534307E3332397E3611
:108D210025552E2D59582A7E5756207E5AE4227AEF
:108D310000758303853182E020E728800DE0128DE4
:108D41006C2A75F02B84AAF005820582E015823029
:108D5100E7EBE0128D6CB5020AD23430000374BC2B
:108D6100F08002C234A234A000B322B44100400317
:108D7100943722B43000400394302224E183222628
:108D8100000000272A00000000002900242528C235
:108D910034301075758303754801853149854982E1
:108DA100E0FA854882F020E75D0549854982E0FBCC
:108DB100B44100404DB45B005048EAB42405EB24B3
:108DC100C08033B42F05EB24E0802BB42B05EB24BA
:068DD100208023B4252CD4
:108DD700EB24C183801A1B1C1D1E1F3B3C3D3E3FDD
:108DE7005B5C5D5E5F7B7C7D7E7F0040607F7F7F1D
:108DF700854882F005480549D234809B054880970D
:108E070075310122C0A075A00378507A05E4F208F5
:108E1700DAFC758303853182E020E70505820A8045
:108E2700F7BA06437F001582E0C39430403324022B
:108E370083802B00010203040506070809FFFFFFD3
:108E4700FFFFFFFFFF0A0B0CFF0D0E0FFF101112A4
:108E57001314FF15161718191A1B1C1D1E1FB4FF14
:108E67000BD3D2D5D0A022C3C2D580F8604AFE78F2
:108E770060E4F2087A047B07EF2B83F2080BDAF839
:108E870080180000000100000032000010240003D9
:108E9700276801048576335544327D05EE13FE506D
:108EA7000778547964128F16DD02800C7864796430
:108EB700128F1680E7028E2DEF2404FFB418F67B7D
:108EC700057F0078507960E2FA54F060178092E2EB
:108ED700FAC4540FFC2375F00A8425F02FD4FFEC55
:108EE7004430F309EA540FBB0103FE8005FC2FD47D
:108EF700FFEC4430F30908DBD6EF540F6E60030232
:108F07008E6E7480F3C3753160754912028E697A6B
:108F170005C3E2FBE33BD4F21819DAF6227A007BA9
:108F270000758303853182E020E70FB43A0050379C
:108F3700B43000403205820A80EDBA072A1582E074
:108F4700540FFC8531827A02E0540F8AF0A42BFB80
:108F570005820ABA08F275F00B84E5F0B5040874C7
:108F6700BCF0C375491322D322FF128FA4502AE005
:108F770004700DA3A31F1F858239858338EF6019FD
:108F8700C083C082E511142582F582E5833400F59C
:048F970083E0D08221
:108F9B00D083047002C322D322C083C08285108386
:108FAB00851182128615E0D082D083B4FF071F1F74
:108FBB00BF0002C322D322758303853182E0B42420
:108FCB000D7800A308E030E7FAB80302C322D322DE
:108FDB0030090CAB12AA13BB0006BA1100500122C8
:108FEB00850F82850E83740A12870DB407F1EA236D
:108FFB00F549B441005061F559755064304803751B
:10900B005046D22AC22F2048077B04128765800561
:10901B007B0D129AD5C22AA3A3A3A385823985837C
:10902B0038753C00D234D22C12916C4028854144C7
:10903B00854245850F39850E38D22C7F041291431A
:10904B00858239858338128765BC000FD22975312B
:10905B0001D22C8020128765028FEA53040EBC02CA
:10906B00F7C22975315F74BC129ABCC22CE53970FA
:10907B00021538153912919E40DE85823985833869
:10908B001549D549F0D234753C00D22C7F032029E9
:10909B00047F04C22C12916E40BE853982853883C1
:1090AB00D22C7F0375F004202907C22C7F0475F0A6
:1090BB0000129143E5F0B5049F30290A74BC129A53
:0190CB00BCE8
:1090CC0075310180020531302F0A20011FE559B49A
:1090DC000215801830010512923A40081290FB30AC
:1090EC00D5055006029063754920D221C22F22303B
:1090FC000E24E559B40E1FA83175A003E275A0002B
:10910C00B4301320010512923A4008ECF005317589
:10911C004921C3D2D522C2D5227C08AA42AB451222
:10912C009BBC4011AA41AB44129BBC4008854144F6
:10913C00854245C322D322853982853883E4FAFBE4
:10914C00FCE0A3302C09B54200B3EA33FA8007B532
:10915C004100B3EB33FBA2E0EC33FCB22CDFE22298
:10916C007F0A129AEB4014AF4AAE4B129BA5400BF0
:10917C00F542AF4CAE4D129BA55003029217F54130
:10918C0010340DE54C254C4007954A50037541FFB2
:10919C00C32212916C407430481F20290FE559B539
:1091AC004902800D1414654960078008E549B40232
:1091BC000385414412912540528539828538837F3D
:1091CC000A1291438A468B47202907129B74AA479F
:0B91DC00AB46EA1292195013202F300E
:1091E70020292DBA002AE55965497024D22F80031A
:1091F700129ABCEB1292195012202F14302911BB6E
:10920700000EA849B80209D22F8003129ABCC322C4
:10921700D32220D01C541E0324028380100037342D
:10922700303239360031383500330000006002C370
:1092370022D3227A007B00758303853182E020E701
:10924700570582E030E7FA1582AD82E0FC1582E02F
:10925700C394302BFBE531B58202800D1582E0C344
:1092670094302AFAE531B582E4EB75F003A42AFAC3
:10927700E435F0600BFBEA2406FA40011BEB70F6BD
:10928700EA75F00A84E5F06003F4240B2430B50492
:10929700078D8274BCF0C322D322301A0CAB12AAFA
:1092A70013BB0006BA1500500122C236850F82850E
:1092B7000E83740A12870DB40704D2368004B401F2
:1092C700E81AEAF549B441005077F559755064300A
:1092D7004803755046303611D22A2048077B0412BE
:1092E700876580057B0D129AD5C22A8582398583C9
:1092F70038753C00D22C3036051293E88003129360
:10930700EC4038854144854245850F39850E38D272
:109317002C7F063036027F0412914385823985837C
:1093270038303608BC001D128765800653043EBCE2
:10933700281AD229753101D22C802B303603128797
:10934700650292B053040EBC02F7800653043FBC7B
:1093570022EFC22975315F74BC129ABCC22CE53961
:1093670070021538153912941840D68582398583CD
:0193770038BD
:10937800D549F2D22C30360C753C007F0320290DDC
:109388007F0480077F052029047F06C22C12916E76
:1093980040AE853982853883D22C30360F7F0375ED
:1093A800F0042029167F0475F000800D7F0575F004
:1093B800112029077F0675F005C22C129143E5F0AC
:1093C80053041FB5040280030292B030290A74BC0A
:1093D800129ABC75310180020531D22575493022B7
:1093E8007F0C80027F0A129AEB4061AF4AAE4B12A3
:1093F8009BA54058F542AF4CAE4D129E07F541B4BF
:10940800FF0CE54CB54A005043E54C04F541C32236
:109418001293EC4037304808854144129125402C7E
:109428008539828538837F0A1291438A468B472083
:109438002907129B74AA46AB47BB00028003BB01F5
:109448000BEA1292194005129ABCC322D322301992
:109458000CAB12AA13BB0006BA1100500122C23687
:109468000ABA00010B740612870D70F1EA1414F59C
:1094780049B44100504EF559755064304803755051
:1094880046C22A850F39850E38753C00D22C1295B4
:039498006D4031F3
:10949B00854144854245850F39850E38D22C7F0690
:1094AB00129143D22C85823985833853043EBC20DC
:1094BB00028005BC0C0ED236D229753101D22C801C
:1094CB001C029465BC02028005BC18F5D236C22979
:1094DB0075315F74BC129ABC753C00D22C1295C1CD
:1094EB0040DF858239858338D549F2D22C753C0013
:1094FB007F0512956F40CA3048077C0212912740B6
:10950B00C0D22C7F0575F01030360375F00620297C
:10951B0010129564C22C7F0675F00130360375F07E
:10952B000C129143E5F053041FB5049530290A74CE
:10953B00BC129ABC7531018002053130020F203606
:10954B000712923A40128005129655400BD21F75A6
:10955B00494030360375494122E5397002153815FB
:10956B0039227F05129AEB4038AF4AAE4B129E0759
:10957B00F542AF4CAE4D129E07F541E5425541B455
:10958B00FF1AE54CB54A005007E54B04F542801F26
:03959B00E54D1487
:10959E00F541E54A04F5428018E542B4FF02804BDE
:1095AE00E541B4FF0CE54CB54A00503FE54C04F5DF
:1095BE0041C322D22C12956D40313048077C0212E5
:1095CE00912740272029101295647F06C22C1291F4
:1095DE0043129649A380077F06D22C129143EC5476
:1095EE003E1295FB4005129ABCC322D322543F0370
:1095FE00B419005044241583603F20360810E63716
:10960E0030E734803410E71E30E62C802C00B0009A
:10961E0037AD3470000032790036000000B93138B1
:10962E00003500000033F8E54B75F003A4B54A0091
:10963E005007E5F07003E8C322D3227F06EC7C00CE
:10964E0013CC33CCDFFA22D2D57B0320D5027B029A
:10965E0075A003A8317A00E220E704080A80F8EA30
:10966E00B50300405D30D5051296D5F5821296D51C
:10967E00F583AE007A007B007C017D0120D51A12A5
:10968E0096D5FF8DF0A42B75F00B84ABF0BD0A00C0
:10969E0040027D000D30D513EF8CF0A42A75F00B2F
:1096AE0084AAF0BC090040027C000CE8B531D03031
:1096BE00D504EAB5820CEBB58308A80674BCF2C3D8
:1096CE008001D375A0002218E2540FB40D02740A63
:1096DE0022300B0CAB12AA13BB000ABA17005005AE
:1096EE00C223C22F22850F82850E830ABA00010B78
:1096FE00740812870D70E9EAB4030040E3B4410028
:10970E0050DEF549F559C223755056304803755051
:10971E0047850E38850F39D22A753C00D229129909
:10972E006D40BDFAA2379229753101400875315F3F
:10973E0074BC129ABCEA1549753C0080051299D684
:10974E004059129ABCE5392408F53950020538D52E
:04975E0049EBC03CD7
:10976200753C00C22FC22312996DD03C400512985D
:1097720009800ED223C22F15597549011297ED4067
:1097820026303723129ABC30290A74BC129ABC754F
:10979200310180020531304605129A70400975493F
:1097A20050D223C22FC3220296EEE549335402F56A
:1097B20049E5392408F53950020538E5392407F519
:1097C20082E5383400F583E0B4FF17C03C43490119
:1097D20012996DD03C4007A849B803278021D223B3
:1097E2008009302306753C0012981A1299D6400F50
:1097F200129ABC0559302FB2C22F12876880ABD3A0
:10980200C22322D22F0559FF853810E5392407F5E6
:109812001150020510EFC322C223D22F2048077B2A
:109822000212877380057B0D129AD522EE75F00322
:10983200842E0422EE20360712982E4049803512DB
:109842009B934042EE75F003842EB507005037EE2D
:109852002557B50700500CE55703547FB506004065
:1098620025800CE55703547F2557B507004017EEB6
:1098720080114012FCB50700400474FF8006EE2FF1
:1098820080001304C322D322EE12982E40F8B507AB
:1098920000400474FF80ED204804EE2F80E4C08372
:1098A200C082853883853982D2D2D2D57E047801AE
:1098B200E0A3A3B54A0510D20A8006B54B0310D522
:1098C20002F608DEEBE9B502005004EAAA01F9E962
:0298D2002A1357
:1098D400354B133400254A133400FBC3202A23E5F7
:1098E4004B03547F254BC3954AB34016EA03547F78
:1098F4002AFDC3954A500BAB05E903547F29C39550
:109904004AB3EBD082D08322853883853982AF4A2B
:10991400AE4B7D04A2369234D23612988A4048A2C5
:10992400349236F542853883853982A3AF4CAE4DE7
:109934007D031298364030F541853883853982D2CB
:109944002C7A007B07E0B54200202C03B54100B31C
:10995400EA20290313800133FAA3B22CDBE7202980
:1099640002EA03F548C322D3227F07D22C202A051A
:109974001299FA8003129AEB401B1299A2D2361262
:10998400990CC236400F129A20400AC2D5B4410045
:109994004005C38003D2D5D3302A02C22A22853897
:1099A40083853982755700A37E03E0A3A3B54D0ECA
:1099B400E5576005B54D028018854D57800FB54CAD
:1099C4000EE5576005B54C028007854C57DEDBF584
:1099D40057227F07D22C202F051299FA8003129A5E
:1099E400EB401112990C400C129A204007B441002C
:1099F4005002C322D322C04A129AEBD0024007ABD2
:0C9A04004A7C05129BBC227583030531CF
:109A10008531820582E030E7FA158274BCF0C322FA
:109A20007B00EB241683B5480CEB241083A2E7924D
:109A300037C2E780370B0BBB30E88032033006318A
:109A400009326033123442352136243730384839F0
:109A50000C2D1824453A512F542E152B1AC129C20A
:109A60000BC30EC42C414A4268433844C322D3225C
:109A70007900758303853182E020E70CC3942424A8
:109A8000198329F9058280F0E9540FD3700C1582EF
:109A9000E01582F0058274BCF0C3220B80808080C8
:109AA00080800F800A0E0D000102030405060708DE
:109AB000090C80808080808010111213C083C082C6
:109AC000758303853182F030290405318002153118
:109AD000D082D08322858353858252E0F5518BF06A
:109AE000A4C4540FC5F0C445F0F0228538838539ED
:109AF00082AE07E4FAFBF54AF54CF4F54BF54DE080
:109B0000A3FC2AFA50010BEC302C10B54A0040029D
:109B1000F54AB54B005002F54B800EB54C004002A3
:109B2000F54CB54D005002F54DB22CDFD2EE128748
:109B30000DEA500104C53C600DFAAB3CAC50530437
:109B40000F129BBC402CE550C4540FFAE53C8AF040
:109B500084B54B00501CB54D005017E53C8AF0A46D
:109B6000C5F0700CC5F0B54A004007B54C00400286
:109B7000C322D322E5467F057A0013CA33CADFFA2F
:109B8000850246E5477F057A0013CA33CADFFA85A6
:109B9000024722F5F0C31325F04009C5F003030383
:109BA000541F25F022EE129B93400FB5070040048E
:109BB00074FF8004EF2E1304C322D322EAC39B5008
:109BC00002F404F5F0EA2B500713C5F0C313C5F0F7
:049BD000C5F0600874
:0C9BD400C5F084B504004002C322D32277
:109BE000301E0CAB12AA13BB0006BA0D00500122A6
:109BF000850F82850E83740812870DB405F1EAF58E
:109C000049B421005048F5597550643048037550E7
:109C100046C22A858239858338753C00D22CD234DD
:109C2000129D1D4029850F39850E38D22C85398229
:109C30008538837F03129CBCC2E0B40414D229751A
:109C40003101D22CE5827002158315828019029BA6
:109C5000EFB40202800270F6C22975315F74BC1243
:109C60009ABC753C00C22C858239858338129D7E52
:109C700040DC858239858338D549F2202917C22CEA
:109C8000E5827002158315827F03129CBCECC2E250
:109C9000B401BB800AD22C7F03129CBCBC02AF3043
:109CA000290A74BC129ABC75310180020531300456
:109CB00005129E1B4098D227754970227C007BFFBD
:109CC000E0FDB503005001FBA3E0B4FF01EBFEEDA6
:109CD00075F00484F5F02D500274FFB506004007BE
:109CE000EDC395F0B50600B3EC33FCDFD322853924
:109CF000828538837A007B007C00E0A3302C0BB592
:109D000042028001B3EA33FA8009B541028001B30F
:109D1000EB33FBA2E0EC33FCB22CDFDE227F081237
:109D20009AEB403EAF4AAE4B129E07F542AF4CAEA7
:0E9D30004D129E07F54110342BE542B4FF2280
:109D3E00E541B4FF1FE54D254C1304F5F0E54B2529
:109D4E004A1304B5F000500CE54A04F542E54D14F3
:109D5E00F541C322D322E541B4FF05E54D254C1351
:109D6E00F544E542B4FF05E54B254A13F545C322FC
:109D7E00129D1D402D3048077C02129127402385ED
:109D8E0039828538837F08129CEE8A468B472029BC
:109D9E0007129DE3AA46AB47129DB24005129ABC2C
:109DAE00C322D322EA7006EB6009F480026BF454EE
:109DBE000F701CEA540F240283801030313233347A
:109DCE0035363738390000000000006002C322D358
:109DDE00227F0780027F04C007E5467A0013CA334C
:109DEE00CADFFA850246E547D0077A0013CA33CA9E
:109DFE00DFFA85024722EE8003EEC3132E4005B52F
:109E0E0007005006EF2E1304800274FF22C2367A2A
:109E1E00007B00758303853182E020E70505820A09
:109E2E0080F7BA020040607A001582AD82E0FC1520
:109E3E0082E0C3943023A236340075F00A84A2E087
:109E4E009236E5F02BFBE531B58202800D1582E0EE
:109E5E00C394302AFAE531B582D5EBA23634002A06
:109E6E00FA500C7B01EA2406FA40011BEB70F6EA6D
:109E7E0075F00A84E5F06003F4240B2430B5040772
:099E8E008D8274BCF0C322D322C2
:109E9700A20C7231500CAB12AA13BB0006BA0D000C
:109EA700500122850F82850E83850F39850E387400
:109EB7000612870DB40137EAB443005031F549D291
:109EC70029753101D23A129F3D501CC2290539E547
:109ED700397002053875315F74FF129ABC129F3DC5
:109EE7004051B46A4E800FB4670040478008029F14
:109EF7003A129F3D403D129ABCD5491E30290DB4F8
:109F07006A3174FF129ABC753101801AB467004038
:109F170022B46A00501D0531800CE5392406F53955
:109F27005002053880CB12A2D2400812A1D14003BB
:109F3700D22422029EA9129F50400D129FA012A068
:109F470013400512A038400022C2D58538838539D1
:109F570082D236E0794BF775F005A3800F853883F9
:109F6700853982E0F46030F4C31380E8E0203602DC
:109F7700C31309F719274008F709A3D5F0EE8005A1
:109F87001036DA8012303A0DC23AE54C20D504C3B8
:109F970013254CF54BC322D32275F00B129FC678BD
:109FA70007ED7FFF801074FFF6E546C395F0F54691
:109FB700E5479400F5477002A64618B800E8227BEB
:109FC70000E54B254D50010B254F50010BFA8B47F0
:109FD7008A46E5F012870D50010AE547C313FDE5F0
:109FE7004613FCEAF5F0232CFC50010D8C468D47F7
:109FF70022C000B50100400E7802F5F0E6B5F0008A
:0CA00700500608B808F67800E8D00022E7
:10A01300784BE6129FF8601BF608B850F5784B7939
:10A0230003E6F70809B850F9202906EBCFFBECCE7D
:10A03300FCC322D322EB2D2FB40B212C2EB40F0003
:10A04300401AB415005015A2E09235EBC39CC39D92
:10A053002E240975F0038485F048800302A1CFED17
:10A06300141475F01FA4FAEE141475F009A42A242D
:10A073006FFAEC141475F01DA4F4042AFAEB14140B
:10A0830075F006A4F4042AB4F10050D0240383022B
:10A09300A1864EFFFFFFFFFFFFFFC9FFFFFFFFFF8B
:10A0A300FFC3FFFFFFFFFFFFFFBEFFFFFFFFFFFF3A
:10A0B300FF3BFFFFFFA8FFFF38EACBFFFF25FFFFB2
:10A0C300A04F4AFF22FFFFB22F44FFFF57FFFF2C91
:10A0D300FFFFFFFF9CFF5EFF4CFFFF99160BFFFF87
:10A0E300C7FFFF01D488FFC1FFFF139085FFFFE186
:10A0F300FFFF8DCDD8FFFF39FFD1DB3C1DFF36B30A
:10A1030089E6301A92A99E5F0617DA8255262D0337
:10A1130065B59411232AFF56D9640EFF5CFFFF9B9C
:10A123006352FF68FFFF98150AFFFFC5FFFF00D3C7
:10A1330087FFBFFFFF698F84FFFFFFFFFF8CFFE2F5
:10A14300FFFFFFFFD0FFFF3AFFFFFFA7FFFF37B47B
:10A15300BDFFFF24FFFF9F6048FF21FFFFB12E4299
:10A16300FFFFFFFFFF2BFFFFFFFFFFFF5DFFFFFF72
:10A17300FFFFFF67FFFFFFFFFFFFFFC6FFFFFFFFBD
:10A18300FFFFC0F46046F4A23530E701B3403DC29F
:10A19300E7FA75F00484240283801B4055550000C0
:10A1A3008000005455050002080046555555190016
:10A1B30000A800806A01C5F06008C5F0030315F02C
:10A1C30080F4E5F05403B54803EAC322D322C23432
:06A1D300755900758303BD
:10A1D900853182753164754864C237C238C239E045
:10A1E9000582B46704D237800AB46804D238800380
:10A1F900B4692DE00582B467005062303725B44058
:10A20900005005242002A292B46000500424C080AA
:10A2190078B462028049B46302804CB4645B804DB7
:10A2290002A2C3303818B4600050042420805AB404
:10A239006202802BB46302802EB4653D8035B4641C
:10A24900005010FA75F00A84243012A2C5E5F024F2
:10A25900308036B464028015B4651E80168039D208
:10A2690039B237B238808CC237C238801FC237D270
:10A27900388019C238D2378013B46610203408E503
:10A28900597009D2348005741D12A2C5303906C22D
:10A2990039B237B23802A1FCB46A1FE559B441009A
:10A2A900501874BC12A2C7200C0530340D800675F5
:10A2B9004980303403754981C322D3220559C082AC
:10A2C900854882F00548D0822275830385318275DD
:10A2D9004701E00582FA0582E01582B46A0280200E
:10A2E900E08547F0A4ABF02A50010BFABB000280CD
:10A2F90009C39467FA50011B80F20547058280D68D
:10A30900EA75F06784E0B5F00D746AF0058205829C
:10A31900E0F47002C322D32230110CAB12AA13BB92
:10A329000006BA1F00500122850F82850E83850F12
:10A3390039850E38740612870DB401EBEAB443006F
:10A3490050E5B4050040E0F549D229753101D23A0A
:10A3590012A3C15017C2290539E5397002053875AC
:10A36900314874FF129ABC12A3C14049B42F4680E8
:10A379000802A3BE12A3C1403C129ABCD54914B429
:02A389002F3370
:10A38B0030290A74FF129ABC753101801005318097
:10A39B000CE5392406F5395002053880D512A5A9EC
:10A3AB00401112A4F0400CD2327549903034037531
:10A3BB0049912202A33012A3D4400D12A3D912A4A7
:10A3CB001A400512A43F400022D2D5029F5275F0CD
:10A3DB0009129FC67806ED7EFF801074FFF6E546E6
:10A3EB00C395F0F546E5479400F5477002A646186D
:10A3FB00B800E822C000B50100400E7802F5F0E687
:10A40B00B5F000500608B807F67800E8D0002278BF
:10A41B004BE612A3FF601BF608B850F5784B790397
:10A42B00E6F70809B850F9202906EBCFFBECCEFC78
:10A43B00C322D322EB2D2FB4090C2C2EB40D0040CC
:10A44B0005B41100400302A4EEEE1414FAED14143B
:10A45B0075F004A42AFAEC141475F010A42AFAEB84
:10A46B00141475F040A42AF5487F00EF241283B52D
:10A47B004807EF240C8302A4EC0F0FBF60ED02A47E
:10A48B00EE032FA00005010A020F03500455055AD5
:10A49B00060007A508F009400A450B4A0C900D95DC
:10A4AB000EE00F141019111E126413B414011506CB
:10A4BB00160B175118A119541A591B411C461D9103
:10A4CB001EA41F15201A216522782352248025856E
:10A4DB0026D02716282929422A562B942C812D6900
:10A4EB002EC322D3227559007583038531827531B2
:10A4FB0064754864E00582B42F56E00582B42F07DB
:10A50B0074BC12A575C322B42B005018B40A0040BA
:10A51B000C12A56A500512A5808004240724301262
:10A52B00A57380D6D234F8E00582C8B42B0912A5E6
:10A53B0069401D940980E8B42C0A12A569401112D8
:04A54B00A58B80DB81
:10A54F00B42D0B12A5694004241780CFD322B42E4B
:10A55F00FB12A56940F6245780C1C8B4240050EC03
:10A56F00B40A00220559C082854882F00548D0827E
:10A57F002224DD83222D2E20242F2B2524F7832226
:10A58F001B1C1D1E1F3B3C3D3E3F5B5C5D5E5F7BAE
:10A59F007C7D7E7F0040607F7F7F75830385318266
:10A5AF007FFEE020E704058280F81582158275474B
:10A5BF000175480279007A00E0FE1582E0FDFAAFDE
:10A5CF00821582AC018547F012A629A9040547E53B
:10A5DF0047B415004003754701AC028548F012A639
:10A5EF0029AA040548E548B4100040037548011531
:10A5FF0082E0B42FCEE975F02F84EDB5F01AEA752D
:10A60F00F02F84EEB5F011742F8F82F00582058242
:10A61F000582E0F47002C322D322E0A4ABF02C50E9
:10A62F00010BFCBB00028009C3942FFC50011B805F
:02A63F00F22205
:10A64100300A12850F82850E83AB12AA13BB000656
:10A65100BA2100500122850F82850E83850F47851F
:10A661000E4812A6BF20D2ED7B02D22A128765C204
:10A671002A12A71F12A7E120D2394037C23AC23BA2
:10A68100C23C12AA8420D22B203C1412AB0D20D242
:10A6910022203B0B12AB7F20D219203A0280D2122A
:10A6A100AEE920D20E40CA12A72D20D206D2221224
:10A6B1008765221287658547368548358097C23878
:10A6C100C237C239EB702D85823AE53A2A14F53B3F
:10A6D100EAB42B005007D2387559008017B43B00FB
:10A6E1005009D237D23875592B8009D238D237D296
:10A6F1003975593BA215721672175012A23882157C
:10A701009238A23782169237A23982179239A2372C
:10A71100B0129237A23872377239B392D22275834E
:10A72100037582017A13E4F0A3DAFC22E4A23E92DB
:10A73100E0A23F92E1FF7582027583037A12E0C2C3
:0FA74100E42430F00582DAF67A05203F077A0229
:10A75000203E027A00303B0A7549D07B0D75820598
:10A760008047303A1F7549A0302C037549A8201C3A
:10A770000C7B0F7582022043300582802C7B1B7579
:10A78000821580257B0F7582027549E0E0B430198F
:10A790007549B82043137549B0058230440BE0B4C5
:10A7A000340705827549C0800085823175820FEAC1
:10A7B000600E1AE0C0828B82F0D0820B058280EF9F
:10A7C000853182E0B430004015B43A005010A3EB5C
:10A7D000B582F074BCF0E5492FF549C2D222D2D23D
:10A7E0002212A887500302A87F12A9B330D2030215
:10A7F000A883754A00754B06854739854838E53981
:10A800007A0614B53A02802ADAF8E539C39404F5D9
:10A81000395002153812B04220D268401574022512
:10A820004BF582758303EAF0E54AC404C4F54AD5C2
:10A830004BCCE53BC39547B40B00403FE54785480B
:10A84000382405F53950020538754B06E5397A0587
:10A8500004B53B028025DAF812B04220D225401B15
:10A86000740FC3954BF582758303EAF0054AE53909
:10A870002404F53950020538D54BD1C2D2C322C2C7
:10A88000D2D322D2D2D322755004800375500580D2
:10A8900025854883854782E58220E01A12AA605008
:10A8A00015A312AA60500FA312AA60500912A9089A
:10A8B0004004C3C234220547E4B547020548E53BDE
:09A8C00024FCB547CCE512703D03
:10A8C900E5596039B51336139401250FF547E50E9F
:10A8D9003400F548755900854883854782C236E5B5
:10A8E9008220E01912AA605004D2368006A312AA67
:10A8F90060500AA312AA605004D234C322D322C2E0
:10A90900D5303907741B12A92E5016303707741326
:10A9190012A92E500C30380BD2D5741B12A92E4017
:10A9290002C322D322FFC083C0822582F582E58338
:10A939003400F58312A978D082D083400530D52D13
:10A94900C2D5C083C0820F0FC3E5829FF582E5831C
:10A9590094005009D082D08330D512800EF583122D
:10A96900A978D082D083400330D502C322D322C034
:10A9790083C082E0FAA3E0F9A3E0FBD082D083EAA6
:10A989002B138550F084FDEAC39B5002F404C313D2
:10A99900B505005014E92A138550F084FDE9C39ADE
:10A9A9005002F404C313B505002285488385478204
:10A9B900E4FAFBFCFD7F0530341DC083C0823036CC
:10A9C9000CE0A3A3A3A3F0D082D0838010A3A3E0BB
:10A9D900D082D083F08006E58220E008E02AFA5090
:10A9E900010B8006E02CFC50010DA3DFEAEDC31337
:10A9F900FFEC132CFCED3FFDEA2CFEEB3DFF404E36
:10AA0900EAC39CFAEB9DFB9235500AEAF42401FA59
:10AA1900EBF43400FBEE75F007A4FDAEF0EF75F032
:10AA290007A42EFEEB600FEE13FEED13FDEBC3132F
:10AA3900FBEA13FA80EEEAAB06AA0512870D20D2CB
:10AA490010EB700DEA34004008F549C2D222D2D287
:10AA5900227549FFC2D2228550F0C083C082E0FA34
:10AA6900A3A3E0FBD082D083EA2B1384FDEAC39B26
:10AA79005002F404C313FCB5050022303940E54AFD
:05AA8900B4663B74E51A
:10AA8E0012AD2F754E1212ADF020D272402B7419EA
:10AA9E0012AD2F754E0312ADF020D2624060C2D5BA
:10AAAE0012AD4EE54DB43F13D22912ADD4C2D5121C
:10AABE00AD4E74E512AD2F800E8041C229E54CB427
:10AACE003F3A741F12AD2FE54DD2D5C2D612AD84CA
:10AADE00402AC36001D382124022C2D512ACE330A9
:10AAEE000515758303758202E0B400080582E0B493
:10AAFE0004028003203405D23CC2D222C2D22230BC
:10AB0E00374DE54A30130A30140754F0B4404080F4
:10AB1E0003B4443B74ED12AD2F754E1212ADF020FE
:10AB2E00D24E404A741112AD2F754E0312ADF02065
:10AB3E00D23E403CD2D512AD4EE54DB40F13D229C4
:10AB4E0012ADD4D2D512AD4E74ED12AD2F800E8053
:10AB5E001DC229E54CB40F16741712AD2FE54DB476
:10AB6E00000CD2D512ACE34005D23BC2D222C2D2E7
:10AB7E002230384BAA4A740612AC4A50035302F0E4
:10AB8E00BA603FC229E5472404B53B0280318548AF
:10AB9E0083E5472403F5825002058375500512AAFA
:10ABAE0060501C74E512AD2FC3953AB40700500FD8
:10ABBE00754E1212ADF04007740512AD2F804D0286
:10ABCE00AC47AA4A74FE12AC4A500353020FBA069F
:10ABDE0068D229E547B53A02805F8548838547826A
:10ABEE0012861575500512AA60504E741912AD2FAB
:03ABFE002406FA30
:10AC0100E53BC39AB40700503D754E0312ADF040C9
:10AC11003574FF12AD2F12ADD4C2D512AD4EE54D34
:10AC2100D2D5D2D6D22812AD86401B12AC57302CC9
:10AC3100097583037582037401F0C2D512ACE34038
:10AC410005D23AC2D222C2D22212AD2F85388385D3
:10AC51003982E02402227583037A06758209E4F0C1
:10AC61000582DAFB758202E0FAE4F075820EEAF001
:10AC710075820378017F15E0C2E4F6C0828F8224D9
:10AC810030F0D082E4F005820F08B807EA7582033C
:10AC9100E4F00582E9F00582EAF00582EEB40300F2
:10ACA1005010EEF075820BEBF00582ECF00582EDB1
:10ACB100F022B4030EEBF0058275820CECF00582F4
:10ACC100EDF022B4040CEBF00582ECF075820DED91
:10ACD100F022EBF00582ECF00582EDF075820DEECD
:10ACE100F0227583037A027B037F0630D5027F054C
:10ACF100E4FCFD8A82E0C2E42CFC8B82E0C2E42DFC
:10AD0100FD0A0A0B0BDFECED75F003A42C75F00ABC
:10AD110084E5F06005740AC395F0FB8A82E0C2E421
:10AD2100B50304C234C322D2343005F9D322854895
:10AD31003830E710F404F539E547C39539F5395052
:10AD4100021538222547F53950020538227582034C
:10AD5100758303E4F54DF54C7A06E0A2E4E54D3345
:10AD6100F54D0582DAF47A06E0A2E4E54C33F54CC0
:10AD71000582DAF430D50B534D0FE54C0303540F24
:10AD8100F54C22C228C22C30D615302809C2282001
:10AD9100E504D22C8001F4543F6036B40701E4602D
:10ADA10021B40B00402BB41D00502624F7838012E0
:10ADB100018002038080808004800708808005096B
:05ADC100800620E70CF4
:10ADC60030D507758303758202F0C322D322740936
:10ADD600FBFA1A7583037D068A82E0FC8B82E0CC3F
:10ADE600F08A82ECF01A0BDDEF22853883853982F2
:10ADF600E54E20E02020E00C128615E0F544A3E5A0
:10AE06004E20E028E0F541A3E0F542A3E0F543A398
:10AE1600E54E20E0E6E4FEFF7A04E02EFE50010F48
:10AE2600A3DAF78F468E45E54E20E0C9AB46AA4524
:10AE360030E510E5442402400ABB0046E544B5026D
:10AE460000403FE54912870D50010A8A4F740EAB48
:10AE560046AA4512870D50010AEAFB75F003A4FCC9
:10AE6600AD03AE04AF04EB75F005A4C5F060037541
:10AE7600F0FFE54E30E402AFF030E208AD04AEF08C
:10AE860080028057AA4FE54EA2E1203501B39236E3
:10AE9600E541303604C39A80012A4043B503004099
:10AEA6003AB507005035E542203604C39A80012A98
:10AEB600402DB503004024B50400501FE54E20E3A5
:10AEC60016E543303604C39A80012A4012B50500C0
:10AED6004009B506005004C2D2C322D3C2D222D240
:10AEE600D2D322C23EC23FA21372145006302906A4
:10AEF60002AF9F02AFB6E53BC39539FA70178538A6
:10AF0600838539827A0D12861F20D2E4E539240220
:10AF1600B582DD8005B40E0040D6E5392402F53948
:10AF260050020538754E0612ADF020D251406AE542
:10AF3600392403F5395002053875570F754A00E56F
:10AF46003BC39539B40300403812B0424033758391
:10AF560003855782F00557054AE54AB40502802164
:10AF6600E53BC39539B406004017754E0912ADF09E
:0AAF7600400FE5392406F5395002BA
:10AF8000053880C102AFBEE54AB4020912AFC24023
:10AF90000ED23E800AB4050712AFEE4002D23FA2A5
:10AFA00013B014B03E4013A214B013B03F400BA234
:10AFB0003EB3B03F4004C2D2C322C2D2D322D2D2C7
:10AFC000D32275830375820F7B00E0A2E4CB33CBE1
:10AFD000C2E475F00AA4FA0582E0A2E4CB33CBC246
:10AFE000E42A75F00484EBB5F002C322D322758302
:10AFF000037A0F7B107E05E4FCFD7F018A82E0A2CC
:10B00000E4CF33CFC2E42CFC0A0ADE0280118B822B
:10B01000E0A2E4CF33CFC2E42DFD0B0B1E80DDEDAB
:10B0200075F009A4FAEC75F003A42A75F00A84AA55
:10B03000F0EFD2D6C2D512AD844005B50202C322CC
:10B04000D322853982853883E582A2E0923D20357E
:10B0500001B39236E4FFFE75F0047902C240E0F7D6
:10B06000B4FE02D2402EFE50010F09A3D5F0EF8F9F
:10B07000468E45EF601975F0047902E7C313F709AE
:10B08000D5F0F8EFC313FFEE13FE80E702B14EEEEA
:10B090008549F084FFE549C313B5F00050010F75F1
:10B0A000F0047902E7303604C39F80012F40DDF7BA
:10B0B00009B236D5F0EE8A418B428C438D44EE7551
:10B0C000F00E84FAE5F0B4080040010A78047F032A
:10B0D0007903EF8AF0A4F7090F0FD8F612B15620C2
:10B0E000D26CE541254225432544B407028016B4BD
:10B0F000065C30405979417A04E7B403030780E2E3
:10B1000009DAF68049AA41E542232AFAE5432323D6
:10B11000232AFAE54475F00CA42A24E88380221639
:10B12000001403FFFFFF180115FF0912071705FFA1
:10B13000FF0211FF131908FF04FFFFFF10FFFFFFBD
:06B1400006A2E4303D010F
:10B14600B392E4FAC2D2C322D3C2D222D2D2D3223B
:10B156007941E7B502004029B50300500477018024
:10B1660019B50400500477028010B5050050047725
:10B17600038007B506005009770409B945D4C2D241
:04B1860022D2D222DD
:10B18A0090108BEFF0A3ECF0A3EDF0901095E0FE99
:10B19A00C39414400B7F277D01EEFB7A0012C3AAE9
:10B1AA0090108BE0FEC39414400B7F277D02EEFBC8
:10B1BA007A0012C3AA90108BE0FE25E025E02496BF
:10B1CA00F582E43410F583E06449600B7F277D0340
:10B1DA00EEFB7A0012C3AA90108BE0FF25E025E06F
:10B1EA002496F582E43410F5837453F090108CE0C1
:10B1FA00FCA3E0FDEF25E025E02498F582E4341075
:0FB20A00F583ECF0A3EDF0901095E004FFF02237
:10B2190090108EEFF0901095E0FF90108EE0FEC335
:10B229009F400B7F287D01EEFB7A0012C3AA901084
:10B239008EE0FF25E025E02496F582E43410F583BD
:10B24900E0B44418EF25E025E02497F582E43410B2
:10B25900F583E0FF7D49E4FBFA12B6C890108EE051
:10B2690025E025E02496F582E43410F5837452F044
:01B2790022B2
:10B27A0090108FEFF0901095E0FF90108FE0FEC3D2
:10B28A009F400B7F297D01EEFB7A0012C3AA901022
:10B29A008FE0FF25E025E02496F582E43410F5835B
:10B2AA00E0B44418EF25E025E02497F582E4341051
:10B2BA00F583E0FF7D49E4FBFA12B6C890108FE0EF
:10B2CA0025E025E02496F582E43410F5837453F0E2
:01B2DA002251
:10B2DB00901090EFF0A3ECF0A3EDF0901095E0FF41
:10B2EB00901090E0FEC39F400B7F2B7D01EEFB7A0D
:10B2FB000012C3AA901090E025E025E02497F58278
:10B30B00E43410F583E0B4FF19E4FFFE12B6649049
:10B31B001090E025E025E02497F582E43410F583C6
:10B32B00EFF0901090E0FF25E025E02496F582E405
:10B33B003410F5837444F0EF25E025E02497F58273
:10B34B00E43410F583E0FF7D52901091E0FAA3E016
:05B35B00FB12B6C82240
:10B36000AE07901095E0FFEEC39F5011EE25E0254B
:10B37000E02496F582E43410F583E0FF227F2A7DF5
:09B3800001EEFB7A0012C3AA22BF
:10B3890090109474FFF0E4901093F0901095E0FF02
:10B39900901093E0FEC39F400302B466EE25E025BA
:10B3A900E02496F582E43410F583E064447045EEB8
:10B3B90025E025E02497F582E43410F583E0FF12B7
:10B3C900B773BF452F901093E025E025E02497F54A
:10B3D90082E43410F583E0FF7D49E4FBFA12B6C834
:10B3E900901093E025E025E02496F582E43410F5E9
:10B3F900837452F0901093E025E025E02496F582BD
:10B40900E43410F583E06452704A901093E0FF250C
:10B41900E025E02496F582E43410F5837445F0EFD5
:10B4290025E025E02498F582E43410F583E0FEA3B5
:10B43900E0AA06F912E7D8901093E025E025E02468
:10B4490096F582E43410F583E0B445087452F0E4CB
:10B45900901094F0901093E004F002B3949010943B
:03B46900E0FF22DF
:10B46C00E4FF901095E0FEEFC39E5018EF25E02509
:10B47C00E02496F582E43410F583E0B4450374526D
:05B48C00F00F80DE223C
:07B4910012B389EF60FA22FB
:10B49800E4901095F0FFEF25E025E02496F582E48E
:10B4A8003410F5837449F0EF25E025E02497F58200
:10B4B800E43410F58374FFF0EF25E025E02498F5D7
:10B4C80082E43410F5837400F0A37422F00FEFB413
:03B4D80014C42277
:03001F00D250229A
:031FDD00C25022CD
:10B4DB00786B06E670021806305055E4FF9010EFBB
:10B4EB00E0FEEFC39E5049EF75F003A4242CF582C8
:10B4FB00E43411AD82FCF583E064527030A374FF29
:10B50B00F5F012E6388D828C83A3E0FAA3E04A7043
:10B51B001C8D828C837445F0EF25E024F0F582E4DA
:10B52B003410F583E0FCA3E04C6002D24F0F80ADEA
:01B53B0022ED
:10B5FC007F037D017C0012B2DB304F5BC24FE490C5
:10B60C0010E6F09010EFE0FF9010E6E0FEC39F50C4
:10B61C0046EE75F003A4242CF582E43411AD82FCC3
:10B62C00F583E0B44529EE25E024F0F582E43410EE
:10B63C00F583E0FCA3E04C6016EE25E024F0F582E7
:10B64C00E43410F583E0FEA3E0AA06F912E7D890E3
:08B65C0010E6E004F080AC22CE
:10B664009010E7EEF0A3EFF09010EFE0FEC3941E0D
:10B67400400B7F2C7D01EEFB7A0012C3AA9010EFE1
:10B68400E0FF75F003A4242CF582E43411F58374EF
:10B6940049F0EF75F003A4242DF582E43411F58309
:10B6A400E4F0A3F09010E7E0FCA3E0FDEF25E02434
:10B6B400F0F582E43410F583ECF0A3EDF09010EF94
:04B6C400E004F0228C
:10B6C8009010E9EFF0A3EDF0A3EAF0A3EBF09010EF
:10B6D800EFE0FF9010E9E0FEC39F400B7F2D7D0156
:10B6E800EEFB7A0012C3AA9010EAE0FFB4492CC21C
:10B6F800AF9010E9E0FE75F003A4242CF582E43441
:10B7080011F5837449F0EE75F003A4242DF582E455
:10B718003411F583E4F0A3F0D2AF22EFB4523D9098
:10B7280010EBE0FEA3E0FFD39400EE9400402DC29E
:10B73800AF9010E9E0FD75F003A4242CF582E43401
:10B7480011F5837452F0ED75F003A4242DF582E40D
:10B758003411F583EEF0A3EFF0D2AF227F2D7D02F6
:0BB768009010E9E0FB7A0012C3AA2257
:10B773009010EDEFF09010EFE0FD9010EDE0FEC3C0
:10B783009D40097F2FEEFB7A0012C3AA9010EDE0D3
:10B7930075F003A4242CF582E43411F583E0FF2231
:10B7A3009010EEEFF09010EFE0FDFF9010EEE0FC54
:10B7B300FB3395E0FAC3EB9F7480F86A98400A7FE5
:10B7C3002EEC3395E0FA12C3AA9010EEE0FF339506
:10B7D300E0FE90112D75F003EF12E70BEE75F00309
:0BB7E300A42583F583E0FEA3E0FF2215
:10B7EE00E49010EFF0FFEF75F003A4242CF582E443
:10B7FE003411AD82FCF5837449F0A3E4F0A3F0EFAD
:10B80E0025E024F0F582E43410F583E4F0A3F00F84
:05B81E00EFB41ED22270
:10C17D0043686B52616D436F6E6669670025754B41
:10C18D006220666F756E640054657374696E672006
:10C19D0020202020002052616D42616E6B202020F6
:10C1AD0020002530326275002025754B62206F6BA3
:10C1BD002100436C656172696E673A202020002072
:10C1CD00202020202020202020202000436C6F6381
:10C1DD006B2020204265616D0042757A7A65722070
:10C1ED0020204B6579004461746520262054696DCB
:10C1FD0065200025303262753A25303262753A2558
:10C20D0030326275000C2573003732350055AA00A7
:0DC21D006618E7817E7E81E7186600AA554D
:08B823007F0C7D3212D03D22A2
:09B82B0012D0D1500312C3122205
:10B8340012B82B12E019EFF4600A7F21E4FDFB7AC1
:10B844008012C3AA12D73AEF600B7F207D047B00DD
:10B854007A8012C3AAE4FF7D0112D5187BFF7AC156
:10B86400797D12EDA175164412D4087F4312D423B6
:10B87400EFF4600B7F257D3A7B007A8012C3AA78AF
:10B88400F87CFF7D017BFF7AC2791A7E007F081263
:10B89400E52C7F3312D423EFF4600B7F257D3A7BB4
:10B8A400007A8012C3AA78F87CFF7D017BFF7AC2FC
:10B8B40079227E007F0812E52C7F2312D423EFF433
:10B8C400600B7F257D3A7B007A8012C3AA78F87CCE
:10B8D400FF7D017BFF7AC2791A7E007F0812E52C76
:10B8E4007F1312D423EFF4600B7F257D3A7B007A1B
:10B8F4008012C3AA78F87CFF7D017BFF7AC279228B
:10B904007E007F0812E52C7F0712D423EFF4600B2E
:10B914007F257D3A7B007A8012C3AA78F87CFF7D6C
:10B92400017BFF7AC2791A7E007F0812E52C7F43DF
:10B9340012D423EFF4600B7F257D3A7B007A8012CA
:10B94400C3AA78F87CFF7D017BFF7AC2791A7E0056
:10B954007F0812EBF2EF60037516347F3312D423A1
:10B96400EFF4600B7F257D3A7B007A8012C3AA78BE
:10B97400F87CFF7D017BFF7AC279227E007F08126A
:10B98400EBF2EF6015E516B4440D7F257D3A7B2F6D
:10B994007A0012C3AA80037516247F2312D423EFDE
:10B9A400F4600B7F257D3A7B007A8012C3AA78F875
:10B9B4007CFF7D017BFF7AC2791A7E007F0812EB3F
:10B9C400F2EF6017E516C39434400D7F257D3A7B72
:10B9D4001F7A0012C3AA80037516147F1312D4238E
:10B9E400EFF4600B7F257D3A7B007A8012C3AA783E
:10B9F400F87CFF7D017BFF7AC279227E007F0812EA
:10BA0400EBF2EF6017E516C39424400D7F257D3AD1
:10BA14007B0F7A0012C3AA80037516087F0712D41D
:10BA240023EFF4600B7F257D3A7B007A8012C3AA52
:10BA340078F87CFF7D017BFF7AC2791A7E007F084B
:10BA440012EBF2EF600B7F227D017B007A8012C340
:10BA5400AA12D41012B823E4FF7D0212D5187BFF7A
:10BA64007AC1798AE51624FCFFE434FFFEEF7805F9
:10BA7400C333CE33CED8F9901671F0EE901670F031
:10BA840012EDA17F6412D3F27F6412D3F27F6412A9
:10BA9400D3F27F6412D3F27F6412D3F27F107D0855
:10BAA40012D518E490118AF0E4FF12D26190118A41
:10BAB400E004F0E0D3947040EF12D6457F0112D336
:10BAC400F2E4FFFD12D5187BFF7AC1799512EDA13E
:10BAD400E4FF7D0112D5187BFF7AC179A212EDA192
:10BAE40012D408786C7601E51624FCFF786CE6FE27
:10BAF400C39F502CEE2404FF12D423EFF4600B7F79
:10BB0400247D3A7B007A8012C3AA7E087F00786C79
:10BB1400E6FD7B017A80790012EC1B786C0680C705
:10BB2400786C7601E51624FCFF786CE6FEC39F5022
:10BB340066EE2404FF12D423EFF4600B7F247D3AD5
:10BB44007B007A8012C3AAE4901188F0A3F09011CC
:10BB5400867480F0A3E4F0901186E475F00112E697
:10BB64004E85F082F583E0FF786CE6FEEF6E600BA5
:10BB74007F227D0EEEFB7A0012C3AA901189E004A5
:10BB8400F07006901188E004F0C3901188E09408E6
:10BB940040C5786C06808D12D41012B82B12D408CC
:10BBA400786C7601E51624FCFF786CE6C39F4003AD
:10BBB40002BCDE7F087D0112D5187BFF7AC179AF04
:10BBC400786CE6901670F012EDA1E4FF7D0212D5B8
:10BBD40018786CE62404FF12D423EFF4600B7F245E
:10BBE4007D3A7B007A8012C3AA7E087F0090C21B34
:0CBBF400E493FD7B017A80790012EC1BC9
:10BC0000E4901188F0A3F09011867480F0A3E4F022
:10BC1000901186E475F00112E64E85F082F583E01E
:10BC2000FF90C21BE493FEEF6E600B7F227D0F7BC3
:10BC3000007A8012C3AA901189E004F07006901176
:10BC400088E004F0C3901188E0940840C37E087F28
:10BC50000090C21AE493FD7B017A80790012EC1BFC
:10BC6000E4901188F0A3F09011867480F0A3E4F0C2
:10BC7000901186E475F00112E64E85F082F583E0BE
:10BC8000FF90C21AE493FEEF6E600B7F227D107B63
:10BC9000007A8012C3AA901189E004F07006901116
:10BCA00088E004F0C3901188E0940840C37BFF7AD9
:10BCB000C179B5786CE62401FFE433FEEF7805C363
:10BCC00033CE33CED8F9901671F0EE901670F01294
:10BCD000EDA112B82312B82B786C0602BBA812D4BF
:10BCE000107F6412D3F27F6412D3F27F6412D3F216
:10BCF0007F6412D3F27F6412D3F212B82BE4FFFDFB
:10BD000012D5187BFF7AC179BF12EDA1E4FF7D0146
:10BD100012D5187BFF7AC179A212EDA1E4FF7D0252
:10BD200012D5187BFF7AC179CC12EDA1786C76011F
:10BD3000E51624FCFF786CE6C39F504912B8237FB8
:10BD4000087D0112D5187BFF7AC179AF786CE69037
:10BD50001670F012EDA1786CE62404FF12D423EFE4
:10BD6000F4600B7F247D3A7B007A8012C3AA7E8028
:10BD70007F007D007B017A80790012EC1B12B82BCA
:10BD8000786C0680AB7F6412D3F27F6412D3F27FAB
:0FBD90006412D3F27F6412D3F27F6412D3F222D3
:10BD9F0012B82312D645E4FFFD12D5187BFF7AC1E6
:10BDAF00799512EDA1E4FF7D0112D5187BFF7AC1C1
:10BDBF0079D912EDA1E4FF7D0212D5187BFF7AC16C
:10BDCF0079E612EDA19011D47463F0A3740CF0A373
:10BDDF00741FF0E4A3F0A37417F0A3743BF0A374E3
:10BDEF0039F0788F7C127D017B017A1179D47E0036
:10BDFF007F0812E52C12CA06E4FF7D0412C6E67F07
:10BE0F00087D8012C6E6E490118DF012B82312D689
:10BE1F0045E4FFFD12D5187BFF7AC179F312EDA12E
:10BE2F00E49011E6F0A3F07B017A12796912CB72DC
:10BE3F007F017D0112D5187BFF7AC2790090126BBA
:10BE4F00E0901670F090126AE0901671F0901269FF
:10BE5F00E0901672F012EDA17F037D0212D5187BD0
:10BE6F00FF7AC2790090126DE0901670F090126E0A
:10BE7F00E0901671F090126FE0901672F012EDA133
:10BE8F0012C69F500F12D0BE500A12B8237FFF1256
:10BE9F00D0A58005E4FF12D0A512B82B9011E7E0D2
:10BEAF0004F070069011E6E004F0C39011E7E094FF
:10BEBF00A59011E6E09400500302BE36E4FF12D0C5
:10BECF00A512B82378D47C117D017B017A12796990
:10BEDF007E007F0812EBF2EF700A7F1F7D37FB7A2F
:05BEEF008012C3AA222D
:041FFB0012CFBD2222
:10BEF4009011E2E0F51612B5B812D28E12C47B404E
:10BF04000302C12012E0ED121F8A12C22A12D216B5
:10BF14007516059011DD7485F07E007F807D007BB1
:10BF2400017A1179E812EC1B9012727401F0A37477
:10BF340011F0A374E8F07B017A1279717D4D12E35C
:10BF440001EF6401600302BFC7901271E06074A343
:10BF5400E0F9A3E0FAA3E09016C8C9F0A3EAF0A3BD
:10BF6400E9F0A3E4F0A37444F07B017A11798E1212
:10BF7400F599E49011D2F0901272E0FBA3E0FAA3D9
:10BF8400E0F990004312E56EFF901268F012F38D11
:10BF9400500C901268E024509011DDF0802590122E
:10BFA40068E0FF12F370501B901268E0FFC36480D6
:10BFB40094C1400FD3EF648094C65007EF24499096
:10BFC40011DDF09011DDE09011D3F012D222901522
:10BFD4005E74B0F090156304F090155D04F0901554
:10BFE4005B04F09015607410F01200929016707457
:10BFF400FFF0A374C2F0A37416F07BFF7AC2791227
:10C0040012EDA1121FDDD2AFE4FF12D16812B834D1
:10C01400E49011E5F0FFFD12D5187BFF7AC179CCCD
:10C0240012EDA1E4FF7D0112D5187BFF7AC179CC12
:10C0340012EDA1E4FF7D0212D5187BFF7AC179CC01
:10C0440012EDA17F057D01E4FB12D2BF121FFF1286
:10C05400B49812B7EE12CFA9127D12128A3412C408
:10C06400C612DDC6E4FF7C7D7D7A12B18A7F017C35
:10C07400B57DE812B18A7F027CDD7D5B12B18A7FD7
:10C08400037CB57DFC12B18A7F047CCD7D5412B152
:10C094008A7F057CC37D7B12B18A7F067C4F7DB18C
:10C0A40012B18A7F077C697D2D12B18A7F087C00DA
:10C0B4007D1212B18A7F097C007D1A12B18A7F0A2F
:10C0C4007CDC7D6412B18A7F0B7CE47D5912B18AD9
:10C0D4007F0112B2197F0212B2197F0312B2197FC3
:10C0E4000412B21912B82B12BD9F9011E47402F01D
:10C0F40012CFD7121FFBE4FF12D168123DE212C423
:10C104008412C47B500B7F1F7D387B007A8012C35E
:10C11400AA12001F9011DE74FFF080449011E4E035
:10C1240024FE7019E4FF12C712EF5406FFBF060D78
:10C1340090118D7401F0E4FF7D0412C6E67F0212B3
:10C14400D3F212D222121FFB12D2ACEF700A7F1F5D
:10C154007D39FB7A8012C3AA123F50E49011DEF0BD
:06C1640012C57212C4A511
:10C16A00123F8BD2AF12D0BE400312C4DE12B4917A
:03C17A0080FB2225
:10C6A900426174746572794C6F7720200046415558
:10C6B9004C5420434F4445005052474D2046415564
:10C6C9004C54005025303262750043253032627572
:0DC6D900004D253033750052455345540087
:0426C200411285FF3D
:10C22A00E4F528F527F526F525F524F523F522F575
:10C23A0021F520F538F537F536F535F534F532F5CB
:10C24A0031F530F541F540F53FF53EF53DF53CF564
:10C25A003BF53AF539F54AF549F548F547F546F516
:10C26A0045F544F543F542F553F552F551F550F5C8
:10C27A004FF54EF54DF54CF54BF557F556F533F5AB
:08C28A0055F554F559F5582251
:10C29200901275EEF0A3EFF0E4A3F0A3F090127504
:10C2A200E0FEA3E0FFC3901278E09F901277E09E39
:10C2B20050157F3212D3F2901278E004F07006909B
:08C2C2001277E004F080D6229F
:06C2CA007F0512B27A228A
:10C2D00012D0BE501A9011E2E516F012C2CA124CEA
:10C2E0009612B46C12D6457F3212D3F21220162267
:10C2F000E4FF7D0212D5187BFF7AC679A912EDA161
:06C300007F6412D3F2225B
:0CC3060012C2F012D0BE500312C2D022AE
:0CC3120012C2F012D0BE500312201622FE
:04C31E0012000022E7
:07C3220012D3E612C31E2234
:08C329007F057D1412D03D22B6
:10C33100901279EFF0A3EDF0901279E0FFC3940130
:10C341004037EFD394105031EBD394014020901239
:10C351008AEFF090127AE0FE901283F0EB149012C3
:10C3610086F07F05EE2406FDE433FC12B2DB901269
:0AC3710079E0FFA3E0FD12D03D22A9
:10C37B0090128AE0FF901283E0FD12D03D9012865E
:10C38B00E014F0E0D3940040107F05901283E0247A
:0FC39B0006FDE433FC12B2DB227F0512B27A22D8
:10C3AA0090127BEFF0A3EDF0A3EAF0A3EBF0E4FF29
:10C3BA0012D0A512C32912C32912D645E4FFFD12D1
:10C3CA00D51890127DE0FEA3E0FFEE30E714547F0B
:10C3DA0090127DF0EFA3F07BFF7AC679B612EDA139
:10C3EA0080097BFF7AC679C112EDA1E4FF7D0212B2
:10C3FA00D5187BFF7AC679CC90127BE0901670F044
:10C40A0012EDA17F047D0212D5187BFF7AC679D37B
:10C41A0090127CE0901670F012EDA17F087D021256
:10C42A00D5187BFF7AC679DA90127DE0FFA3E090F7
:10C43A001670CFF0A3EFF012EDA19011E5E0B4FF72
:10C44A001090127BE0FFA3E0FD90127EE0FB124CFD
:10C45A00A97FA07E0012C29212C32990127BE0B477
:10C46A00200312C59912D0BE500312201612C322FD
:01C47A00229F
:09C47B00E519B4AA02C322D32280
:04C484007519AA225A
:04C4880075195522AB
:04C48C007518AA2253
:0EC49000901287E0FF7D49E4FBFA12B6C82245
:07C49E0012C49012C2D0226B
:10C4A50012D0BE5012901287E0FF7D52901281E0AB
:08C4B500FAA3E0FB12B6C82255
:09C4BD00901281EEF0A3EFF022D1
:10C4C6007EC47F9E12B664901287EFF07F647E0072
:04C4D60012C4BD22AD
:04C4DA0012C3062261
:0CC4DE00E4FF12D18C12C490124A6222BA
:07C4EA0012C4A5124BD92278
:10C4F100901284E024FE601B04702812D0D15003F6
:10C5010012C4DA12D0BE402112C4DE901284740229
:10C51100F0801612D0BE501112C4EA901284740138
:10C52100F080069012847401F0901289E014602268
:10C5310014703712D0E4901288EFF0600E901285DB
:10C5410074FFF0901288E0FF124C6290128974011E
:10C55100F02212D0E4EF700B901285E06005E4F058
:10C561001200169012897402F0229012897402F05E
:01C5710022A7
:10C5720012D0BE50089012847401F080069012848A
:10C582007402F012D0E4EF60079012897402F02274
:07C592009012897401F022F0
:10C5990012C48C9016C874FFF0A374C6F0A374E09B
:10C5A900F0A3E4F0A37405F07B007A00791812F582
:10C5B9009912D6451220007F31E4FDFB7A8012C31F
:02C5C900AA22A4
:10C5CB0012C48C12C48812D645E4FFFD12D5181282
:0DC5DB0020007F31E4FDFB7A8012C3AA220C
:10C5E80090127FEFF0A3EDF0E0B40800400302C61C
:10C5F8008D90C600F828287302C61802C63002C6F5
:10C608003C02C62402C66702C64802C65402C67E59
:10C6180090127FE0FF12F3C7E433FF2290127FE00D
:10C62800FF12F38DE433FF2290127FE0FF12F370C4
:10C63800E433FF2290127FE0FF12F39EE433FF22DF
:10C6480090127FE0FF12F3D8E433FF2290127FE0CC
:10C65800FF64306004EFB431037FFF227F00229033
:10C66800127FE0FF12F38D400790127FE0B42E0393
:10C678007FFF227F002290127FE0C3948050037FC7
:10C68800FF227F00227F30901280E0FD90127FE031
:07C69800FB7A0012C3AA2285
:0100220022BB
:0AC69F0012D157EF7002C322D3221C
:10C6E60090128BEFF0A3EDF012DED67FA212DF439D
:10C6F60090128BE0FF12DF6B90128CE0FF12DF6569
:0CC7060012DF3712DEDB7F0512D3F222B7
:10C7120090128DEFF012DED67FA212DF4390128DBF
:10C72200E0FF12DF6B7FA212DF4E12DF7690128ED5
:10C73200EFF012DF3712DEDB7F0512D3F290128E9A
:03C74200E0FF22F3
:10C7450090129EE0FF7C127DAE12B5CF90129FE055
:10C75500FF7C127DB112B5CF9012A0E0FF7C127D57
:10C76500B412B5CF9012B0743AF09012B3F0E490D1
:10C7750012B6F090129CE0FF7C127DA412B5CF900A
:10C78500129BE0FF7C127DA712B5CF90129AE0FFB5
:10C795007C127DAA12B5CF9012A6742FF09012A923
:07C7A500F0E49012ACF02259
:10C7AC009012A2E0FF7D527B047A0012B6C8E4908E
:10C7BC0012A3F09012B87442F012DED612DEE075BD
:10C7CC000C12750DBB786FE618F6050DE50DAE0C69
:10C7DC007002050C14F5828E83E0FF12DEEC9012D1
:10C7EC00B8E0644560409012A2E0FF12B773BF45F9
:10C7FC001112DEDB7F639012A3E0FD7B047A001242
:10C80C00C3AA786E16E670089012B87445F080CE04
:10C81C00050DE50DAE0C7002050C14F5828E83E04F
:10C82C00FF12DEEC80B812DEF212DEDB9012A2E018
:0AC83C00FF7D49E4FBFA12B6C822A2
:08C84600E4FF7D0112C6E622A9
:08C84E00E4FF7D0412C6E6229E
:10C856009012BBEFF0786E76010876019012A2E096
:10C86600FF7D527B047A0012B6C8E49012A3F090C2
:10C8760012B87442F012DED612DEE0750C12750D97
:10C88600BB786FE618F6050DE50DAE0C7002050CCB
:10C8960014F5828E83E0FF12DEEC9012B8E0644558
:10C8A60060409012A2E0FF12B773BF451112DEDBA3
:10C8B6007F639012A3E0FD7B047A0012C3AA786E10
:10C8C60016E670089012B87445F080CE050DE50D99
:10C8D600AE0C7002050C14F5828E83E0FF12DEECBE
:10C8E60080B812DEDB9012A2E0FF7D49E4FBFA126B
:03C8F600B6C8229F
:10C8F900EFD39410400302C9C5786EEFF608F6909D
:10C9090012A2E0FF7D527B047A0012B6C812DED66D
:10C91900E49012A3F09012B87442F012DEE6750AA0
:10C9290012750BBB786FE618F612DEF6050BE50BF0
:10C93900AC0A7002050A14F5828C83EFF09012B8E4
:10C94900E0644560649012A2E0FF12B773BF45111D
:10C9590012DEDB7F589012A3E0FD7B047A0012C33C
:10C96900AA786E16E670089012B87445F080CE78F1
:10C979006EE6D39401401612DEF6050BE50BAC0A00
:10C989007002050A14F5828C83EFF080B012DEFA8A
:10C99900050BE50BAC0A7002050A14F5828C83EFCE
:10C9A900F09012B87445F0809412DEF212DEDB903A
:0DC9B90012A2E0FF7D49E4FBFA12B6C8228D
:07C9C6009012B7E024FF22EC
:0CC9CD007F0412B2199012CC7401F02209
:10C9D9009012BEE0FFC41313540370209012CBE0F1
:10C9E900B403199012ADE0C394605006E02404F03A
:0DC9F9008005E49012ADF0E49012CBF02226
:10CA0600901290E014D3940B40047F0180027F00C3
:10CA160090128FE0D3946340047E0180027E00EE84
:10CA26004FFF901291E014D3941E40047E018002C1
:10CA36007E00EE4FFF901292E0D3940640047E01F2
:10CA460080027E00EE4FFF901293E0D394174004CD
:10CA56007E0180027E00EE4FFF901294E0D3943B5D
:10CA660040047E0180027E00EE4FFF901295E0D3D7
:10CA7600943B40047E0180027E00EE4F600A7F33C5
:10CA86007D01E4FBFA12C3AAE49012BBF0A374047E
:10CA9600F0E4A3F0901295E0FF75F00A84FEC4540A
:10CAA600F0FEEF75F00A84E5F04E9012BEF090129B
:10CAB60094E0FF75F00A84FEC454F0FEEF75F00AA8
:10CAC60084E5F04E9012BFF0901293E0FF75F00AE5
:10CAD60084FEC454F0FEEF75F00A84E5F04E901221
:10CAE600C0F0901291E0FF75F00A84FEC454F0FE87
:10CAF60090128FE0FD5403FCC4333354C04EFEEF56
:10CB060075F00A84E5F04E9012C1F0901290E0FFA5
:10CB160075F00A84FEC454F0FE901292E0FBC43312
:10CB260054E04EFEEF75F00A84E5F04E9012C2F026
:10CB3600ED1313543F25E025E09012ADF09012CB93
:10CB4600ECF0786E760808760812C7AC789A7C12F4
:10CB56007D017B017A12798F7E007F0812E52C1207
:0CCB6600C74512C9CD9012B774FFF02231
:10CB7200901297EBF0A3EAF0A3E9F07F0212C856F5
:10CB82007F0512C8F912C9D99012BBE0FFC4540F35
:10CB920075F00AA4FEEF540F2EFF901297E0FBA34C
:10CBA200E0FAA3E0F9900006EF12E5AD9012BCE0C6
:10CBB200FFC4540F75F00AA4FEEF540F2E90000527
:10CBC20012E5AD9012BDE0FF5430FEC4540F75F073
:10CBD2000AA4FEEF540F2E90000412E5ADEF54406C
:10CBE200FFC41313540390000712E5AD9012BEE088
:10CBF200FF5430FEC4540F75F00AA4FEEF540F2EFA
:10CC020090000212E5ADEFC413135403FF9012AD6E
:10CC1200E02F12E59B9012BFE0FF5410FEC4540FA8
:10CC220075F00AA4FEEF540F2EFE901297E0FBA3BC
:10CC3200E0FAA3E0F9900001EE12E5ADEFC413545F
:0BCC42000790000312E5AD12C9CD22DF
:10CC4D009012BBE0FF540FFE44309012B5F0EFC4CC
:10CC5D00540FFD44309012B4F0ED75F00AA42E90EF
:10CC6D0012A0F09012BCE0FF540FFE44309012B2AF
:10CC7D00F0EFC4540FFD44309012B1F0ED75F00A91
:10CC8D00A42E90129FF09012BDE0FF540FFE443081
:10CC9D009012AFF0EF5430FFC4540FFD443090129A
:10CCAD00AEF0ED75F00AA42E90129EF09012BEE03B
:10CCBD00FF540FFE44309012A5F0EF5430FFC454D2
:10CCCD000FFD44309012A4F0ED75F00AA42E9012D1
:10CCDD009CF09012BFE0FF540FFE44309012A8F06C
:10CCED00EF5410FFC4540FFD44309012A7F0ED75B2
:10CCFD00F00AA42E90129BF012C9D99012BEE0FF3B
:10CD0D00C413135403FF9012ADE02FFD90129AF04F
:10CD1D0075F00A84E5F044309012ABF0AF05EF7575
:10CD2D00F00A8444309012AAF09012BDE05440FFF6
:10CD3D00C4131354039012A1F09012BFE0FFC4135B
:07CD4D00540790129DF02233
:10CD54009012CCE024FD700302CE0C24FE7003027A
:10CD6400CF1024FE700302CF842406600302CFA2F6
:10CD74009012BB7402F0786E760108760112DED64A
:10CD84009012A2E0FF7D527B047A0012B6C8901282
:10CD9400CC7403F0E49012A3F09012B87442F01231
:10CDA400DEE0750C12750DBB050DE50DAE0C7002C1
:10CDB400050C14F5828E83E0FF12DEEC9012B8E0CD
:10CDC400644560409012A2E0FF12B773BF45111290
:10CDD400DEDB7F639012A3E0FD7B047A0012C3AA1A
:10CDE400786E16E670089012B87445F080CE050D82
:10CDF400E50DAE0C7002050C14F5828E83E0FF1273
:10CE0400DEEC80B812DEF2229012B8E064456003D2
:10CE140002CED2786E76050876059012A2E0FF7DE8
:10CE2400527B047A0012B6C812DED6E49012A3F044
:10CE34009012B87442F012DEE6750A12750BBB78D4
:10CE44006FE618F612DEF6050BE50BAC0A70020568
:10CE54000A14F5828C83EFF09012B8E064456064A4
:10CE64009012A2E0FF12B773BF451112DEDB7F58A8
:10CE74009012A3E0FD7B047A0012C3AA786E16E632
:10CE840070089012B87445F080CE786EE6D39401A1
:10CE9400401612DEF6050BE50BAC0A7002050A1407
:10CEA400F5828C83EFF080B012DEFA050BE50BAC53
:10CEB4000A7002050A14F5828C83EFF09012B8749C
:10CEC40045F0809412DEF29012CC7405F022901298
:10CED400A2E0FF12B773BF451F12DEDB9012A2E07F
:10CEE400FF7D49E4FBFA12B6C87F639012A3E0FD0C
:10CEF4007B047A0012C3AA229012B8E0644E600345
:10CF040002CFA8786FE618F612C7AC229012B8E0E8
:10CF14006445703112DEDB9012A2E0FF7D49E4FB30
:10CF2400FA12B6C89012BAE0FFA3E06F600790123D
:10CF3400CC7407F0229012CC7401F07F047D027C43
:10CF44000012B2DB229012A2E0FF12B773BF451F9A
:10CF540012DEDB9012A2E0FF7D49E4FBFA12B6C8B0
:10CF64007F589012A3E0FD7B047A0012C3AA22909A
:10CF740012B8E0644E702D786FE618F612C7AC2232
:10CF84007F047D0F7C0012B2DB9012CC7401F09010
:10CF940012BBE09012BAF012CC4D124C3F22901208
:05CFA400CC7401F02235
:10CFA900E49012B7F012DED6E4FFFE12B6649012D6
:04CFB900A2EFF022D1
:10CFBD009012CC7401F0FB7A12799A12CB7212C7CF
:0ACFCD00459012BBE09012BAF0226A
:10CFD700788F7C127D017BFF7A7D79187E007F0830
:07CFE70012E52C12CA06221C
:10CFEE00EFB404005048C083C082F5F012D4087F1D
:10CFFE000212D423531FFCE5F02390D00C73801E35
:10D00E008004800A8010431F02755A018013431F4B
:10D01E0001755A02800B431F03755A038003755A1C
:10D02E0000908000E51FF012D410D082D08322ED44
:10D03E006004FAEF700122C2AF5389F0438901AB4D
:10D04E000204F9838010EDD3BCB19E8C7D75685DB2
:10D05E00574E453D3A33FF7A0012870D0BEF2323CF
:10D06E00FCFD5304FC5305036304FF6305FF8D8C25
:10D07E008C8AC28DD28C308DFDC28CB2B5DAEFDBCC
:10D08E00EDD2B5204B02C2B5D2AF22790278FAD8D2
:10D09E00FED9FAD5E0F522BF0004D2B48007C2B49F
:10D0AE007F0112D3F222BF0004D2B48002C2B42296
:10D0BE0012D4087F0112D423908000E0A2E3B312B1
:10D0CE00D4102212D4087F0112D423908000E0A243
:10D0DE00E0B312D4102212D4087F0112D423908010
:10D0EE0000E030E50A10E40B10E10C7F03800C7FAA
:10D0FE000080087F0180047F02800012D41022126B
:10D10E00D4087F0112D423908000E0A2E212D41042
:10D11E0022EFC083C082C0A8C2AFF5F012D4087F40
:10D12E000212D423E5F02390D13973800280054397
:10D13E001F008005431F048000908000E51FF01241
:10D14E00D410D0A8D082D0832220960B7F0A12D37F
:10D15E00F22096037F01227F0022EFB40000401DD3
:10D16E00C083C08254022390D1797380088000C29C
:10D17E00B5C24B8004D2B5D24BD082D08322EFB44D
:10D18E000000402FC083C082F5F012D4087F021237
:10D19E00D423531FFBE5F0540290D1AB7380028071
:04D1AE0005431F0412
:10D1B2008000908000E51FF012D410D082D083222C
:10D1C200C0A8C2AFBF0004C2938002D293D0A822EB
:10D1D200BF00057590FC800375907C22C29622EFF9
:10D1E200B40200502EC083C082F5F012D4087F0230
:10D1F20012D423531FDFE5F02390D1FF7380078001
:10D2020000431F208000908000E51FF012D410D050
:10D2120082D08322900000E4F0A3E58330E7F82275
:10D222007F2F12D2767FA312D2769011D3E0FF1213
:10D23200D2767FA012D2767FC812D2767FAF12D278
:10D2420076227FAE12D2767FA512D27622E9C0E094
:10D2520079009080FAE030E702D9F7D0E0F92212A3
:10D26200D408EFC0E07F0312D423D0E09080F9F01D
:10D2720012D4102212D408EFC0E07F0312D423127A
:0CD28200D24F9080F8D0E0F012D41022BF
:10D28E0012D29812D29B12D2A922C2AC22C29CC236
:10D29E009822D2AC22D29C22D24A22C24A22901189
:10D2AE00E0E0FF9011DFE0FD9011E1E0FB12D2D241
:10D2BE00229011E0EFF09011DFEDF09011E1EBF024
:10D2CE0012D2D222BF07005042EFF8BD0400503BED
:10D2DE00ED1392D513E833A2D533F8BB0200502BD1
:10D2EE00EB13E83390118CF0C2ACC2AD759800759B
:10D2FE00C830EF2390D31C93F5CBEF230493F5CADC
:10D30E00D29EEB13929FD2CA7FFF227F0022FB8018
:10D31E00FDC0FEE0FF70FFB8FFDCFFEE90118CE069
:10D32E0023540E90D33573800E8025801280278073
:10D33E0015802880158028EF547FA2D0B3800DEF82
:10D34E00547FA2D08006EFD38002EFC392E7801302
:10D35E00EFA2D0B3800BEFA2D08006EFD38002EF06
:10D36E00C3929BF59922AF9990118CE023540E90A5
:10D37E00D38173800E80258010802A8011802F80AB
:10D38E00138031EFA2D0B3800EEFA2D08009EFA2AE
:10D39E00E7B38003EFA2E7547FFF801BEFA29A2032
:10D3AE00D015B38012EFA29A30D00CB38009EFA241
:10D3BE009AB38003EFA29A400302404B027CFA30EC
:10D3CE004A051200FE8010309805C29812D37430B0
:10D3DE009905C299127CAA22E4F588F5C8F589F55B
:10D3EE00A8F5B822EF7001227FE4DFFE7FE4DFFEB6
:0AD3FE001480F2EF700122DFFE221E
:10D40800D083D082C01EE473D083D082D0E05493FE
:10D41800531E6C451EF51EF590E473EF7B00B516A0
:10D42800005003B400037F0022C2AFB405005010BF
:10D43800531E642390D4407380548058805C80606D
:10D44800C3940475F01084232390D455737B74809F
:10D458000A7B6480067B6580027B66E5F0751E7634
:10D46800851E90531F27C32390D474738038803E41
:10D47800804180448047804A804D80508053805648
:10D488008059805C805F806280658068806B751ED3
:10D498007402D510751E7502D510751E7602D5104A
:10D4A800751E7702D510431FD8BB7452804B431F9B
:10D4B800D0804B431FC88046431FC08041431F98FC
:10D4C800803C431F908037431F888032431F8080F1
:10D4D8002D431F588028431F508023431F48801E18
:10D4E800431F408019431F188014431F10800F43A7
:10D4F8001F08800A431F008005751E67800A9080F8
:10D5080000E51FF08B1E8000851E90D2AF7FFF22A2
:1026C6004115620041156100628512D400000000C8
:1026D6000000009E0000000E000E0028FE28FE28C6
:1026E6004854FE5424462610C8C46C92AA44A0003E
:1026F6000A06000000384482000082443800281090
:102706007C102810107C101000C060000010101003
:10271600101000C0C0000040201008047CA2928A5D
:102726007C0084FE800084C2A2928C62828A9662B9
:10273600302824FE204E8A8A8A7278949292600209
:10274600E2120A066C9292926C0C9292523C006CC7
:102756006C000000AC6C0000102844820028282879
:10276600282882442810000402A2120C6492F282E5
:102776007CFC222222FCFE9292926C7C8282824413
:10278600FE82824438FE92929292FE121212127CBD
:10279600829292F4FE101010FE0082FE82004080AB
:1027A600827E02FE10284482FE80808080FE04180D
:1027B60004FEFE081020FE7C8282827CFE1212122B
:1027C6000C7C82A242BCFE1232528C8C9292926295
:1027D6000202FE02027E8080807E3E4080403E7E77
:1027E6008070807EC6281028C60E10E0100EC2A289
:1027F600928A8600FE8282000408102040008282AF
:10280600FE0008040204088080808080000204081C
:102816000040A8A8A8F8FE9088887070888888402C
:1028260070888890FE70A8A8A83010FC12020418C0
:10283600A4A4A47CFE100808F00088FA800040805A
:10284600887A00FE205088000082FE8000F808305A
:1028560008F0F8100808F07088888870F82828288A
:102866001010282830F8F81008081090A8A8A840DA
:10287600087E88804078808040F8384080403878EC
:102886008060807888A020A08818A0A0A07888C83A
:10289600A8988800106C82000000FE000000826C80
:1028A600100008082A1C08081C2A08081CA2E22294
:1028B6002478828042F870A8ACAA3040ACAAACF06A
:1028C60040AAA8AAF040AAACA8F040AEAAAEF0185A
:1028D600A4E4241070ACAAAC3070AAA8AA3070AADE
:1028E600ACA830008AF88200008CFA8400008AFCCA
:1028F6008000F02A282AF0F02E2A2EF0F8A8ACAA9A
:10290600A8E8A8F0A8B0FC12FEA2A2708C8A8C706F
:10291600708A888A70708A8C887078848244F87885
:10292600828440F818A2A0A2787886848678788275
:102936008082783048FC482010FC9294805254F8EB
:1029460054527E0A2EF0A090907C121200000000D5
:012956000080
:10D518009012CDEDF0E0FE64086015901560E0FD16
:10D52800EFC39D400302D5FDEE6408700302D5FDEC
:10D53800901562E0700A90155CEFF090155FEEF0C0
:10D54800EE64086009EF75F006A4FF2410FFEFC42D
:10D55800540F44109012CEF0EF540FA3F0EE701950
:10D5680090155EE0FF12D2769012CEE0FF12D276CE
:10D578009012CFE0FF12D276229012CDE0B40119BA
:10D58800901563E0FF12D2769012CEE0FF12D276A9
:10D598009012CFE0FF12D276229012CDE0B4021999
:10D5A80090155DE0FF12D2769012CEE0FF12D2768F
:10D5B8009012CFE0FF12D276229012CDE0B4031978
:10D5C80090155BE0FF12D2769012CEE0FF12D27671
:10D5D8009012CFE0FF12D276229012CDE0B4081557
:10D5E8007FB812D2769012CEE0FF12D2769012CF88
:06D5F800E0FF12D27622D2
:10D5FE009012D0EFF0E024E0F0E4FF12D261E4905C
:10D60E0012D1F09012D1E0FFC3940550299012D0A0
:10D61E00E075F005A424D4F582E5F03412F583E527
:10D62E00822FF582E43583F583E0FF12D2619012EA
:07D63E00D1E004F080CD22D1
:10D64500E49012D2F09012D2E0FFC39404505990A6
:10D65500155EE02FFF12D2767F1112D276E4FF120B
:10D66500D276E49012D3F0E4FF12D261E4FF12D235
:10D6750061E4FF12D261E4FF12D261E4FF12D261CC
:10D68500E4FF12D261E4FF12D261E4FF12D261908D
:10D6950012D3E004F0E0C3940C40CCE4FF12D26155
:09D6A5009012D2E004F0809D22F5
:10D6AE008F14EFC39420401B901560E0FF90155C23
:10D6BE00E0C39F500BE004F0AF1412D5FEAF14225E
:10D6CE007F0022E514B40A1190155FE0045403FFA5
:10D6DE00F0FDE4FF12D518800EE514B40C0912D635
:0AD6EE0045E4FFFD12D518AF142229
:10DDF200257300000000000006050300000607016D
:10DE02000000013741424301344A4B4C0131535423
:10DE120055012E2C3B3F04000000000000000000D2
:10DE220006060400000608020000013844454601C7
:10DE3200354D4E4F0132565758013024253A0120B4
:10DE42002B2D2F000000000000090000000200003E
:10DE52000000013947484901365051520133595A9D
:10DE62002A03000000000000000000FFD926FFD9AD
:10DE720038FFD992FFD9ACFFD9E3FFDA1AFFDA2AC9
:10DE8200FFDA3FFFDA56FFDAD1FFDAE8FFDAF8FF0E
:10DE9200DB08FFDB11FFDA3FFFDB28FFDAD1FFDA15
:10DEA200E8FFDAF8FFDB08FFDB11FFDA3FFFDB6F89
:10DEB200FFDAD1FFDAE8FFDAF8FFDB08FFDB11FF58
:10DEC200D926FFDBD0FFD992FFD9ACFFDC10FFDAF5
:04DED2001AFFDC3B1C
:10D6F8007F0312D423EFF4600A7F407D01E4FBFA34
:10D7080012C3AA7E01E42EF582E43480F583E0FD9D
:10D7180020E003AF0622ED20E105EE2408FF22AF4A
:10D7280005ED20E205EE2410FF220EEEB408D67FA8
:02D73800FF22CE
:10D73A0012D4087F0312D423EFF4600A7F407D01DC
:10D74A00E4FBFA12C3AA908004E030E20B90800056
:10D75A00E020E004E030E10612D4107FFF2212D468
:04D76A00107F00220A
:0BD76E007F0A12B27A7F0212B27A2208
:06D7790012D76EC252221D
:08D77F007F0212B219D25222FE
:10D787009015BCE0FF7D49E4FBFA12B6C8E4787156
:02D79700F62278
:10D79900305117E4901575F07870F6FE7F41FD7BE6
:0BD7A900017A15797712EC1BC25122A7
:10D7B400901566E0FFD394405031901565E0D39FF7
:10D7C4005029901564E0D394035020901569E0D358
:10D7D400940F5017A3E0D394035010901567E0D32F
:10D7E40094075007A3E0D3941F400A7F3F7D01E4D0
:10D7F400FBFA12C3AA78BD7C157D017B017A1579E9
:10D80400647E007F0D12E52C9015747442F0E4A33D
:10D81400F012D787E47870F6FE7F41FD7B017A151C
:10D82400797712EC1B9015C4E0FBA3E0FAA3E0F9AE
:10D8340012E55560299015C2E0FFA3E0FD12D5184A
:10D844009015C4E0F9A3E0FAA3E0901670C9F0A320
:10D85400EAF0A3E9F07BFF7ADD79F212EDA1C2517F
:10D864009015C7E0FBA3E0FAA3E0F912E5557003B5
:10D8740002D8FE12F601901571EFF09015BFE0FE8C
:10D88400EFD39E400E7F3F7D02901571E0FB7A003E
:10D8940012C3AAE4901572F0901571E0FFA3E0FEA4
:10D8A400C39F50359015C7E0FBA3E0FAA3E0F98EBF
:10D8B4008275830012E56EFF9015C0E0FD12C5E885
:10D8C400EF700E7F3F7D03901572E0FB7A0012C368
:10D8D400AA901572E004F080BF901571E090157560
:10D8E400F07870F678777C157D019015C7E0FBA37E
:0ED8F400E0FAA3E0F912EA4FD25112D77F22D8
:0AD902009015747444F012D77922D6
:10D90C009015BDE030E0127F0A7D0C7C0012B2DB7A
:0AD91C009015B8E4F0A37406F022A1
:10D926009015C1E030E10A12D7877873E6FF124DF1
:02D93600A0222D
:10D938009015C1E030E05212D7999015BFE0FF78FA
:10D9480070E6C39F503E7873E6FFA3E0FD12C5E87A
:10D95800EF60317873E6FF7870E6062477F582E4A5
:10D968003415F583EFF0E6FF2477F582E43415F5F6
:10D9780083E4F0901575EFF07F01124CC012D78741
:0AD9880012D90C227F0B124CC022B2
:10D992009015C1E0FF20E00330E10E787176017F3F
:0AD9A20007124CC07F09124CC0228E
:10D9AC009015C1E030E02F12D7879015BEE0FF90A4
:10D9BC001575E0FEC39F40199015BFE0FFEED39F95
:10D9CC00500F7F05124CC012D7799015747445F026
:07D9DC00227F0B124CC02258
:10D9E3009015C1E030E02F12D7877870E6D394000A
:10D9F300401F7F06124CC0787016E62477F582E448
:10DA03003415F583E4F0E6901575F0C25112D90C84
:07DA1300227F0B124CC02220
:10DA1A009015C1E030E00812D7877F08124CC02267
:10DA2A009015C1E030E20D12D7877873E6FF124DE8
:05DA3A002012D90C22AE
:10DA3F009015C1E030E10F12D7877F0A124CC078E2
:07DA4F0074E6FF120008223B
:10DA56009015C1E030E07312D7999015BFE0FF78BA
:10DA660070E6C39F505F7874E6FFA3E0FD12C5E839
:10DA7600EF60437873E69015BBF008E6FF7870E632
:10DA8600062477F582E43415F583EFF0E6FF247774
:10DA9600F582E43415F583E4F0901575EFF07F0216
:10DAA600124CC09015BCE0FF7D527B287A0012B65E
:10DAB600C87871760222E47871F67F0A124CC07F2C
:0BDAC6000B124CC0227F0B124CC02240
:10DAD1007F07124CC09015BCE0FF7D49E4FBFA12B0
:07DAE100B6C878717601223E
:10DAE8009015C1E030E0087F0A124CC012D9AC2270
:10DAF8009015C1E030E0087F0A124CC012D9E32229
:09DB08007F0A124CC012DA1A2245
:10DB11009015C1E030E10F12D7877F0A124CC0780F
:07DB210074E6FF124DA02283
:10DB28009015BBE078736670327875E6FF9015C083
:10DB3800E0FD12C5E8EF60197875E6FF7870E62415
:10DB480076F582E43415F583EFF07F03124CC0803C
:10DB5800057F0B124CC078717603227F0A124CC0E5
:07DB680012D78712D9382201
:10DB6F007F0A124CC09015BBE078736670477876C9
:10DB7F00E6FF9015C0E0FD12C5E8EF60197F0412B3
:10DB8F004CC07876E6FF7870E62476F582E434159B
:10DB9F00F583EFF08014787016E62477F582E4347D
:10DBAF0015F583E4F07F0B124CC07870E690157575
:10DBBF00F012D787227F0A124CC012D78712D9389A
:01DBCF002233
:10DBD0009015BFE0FF7870E6C39F502E7F01124C76
:10DBE000C07873E6FF7870E6062477F582E4341592
:10DBF000F583EFF0E6FF2477F582E43415F583E44E
:10DC0000F0901575EFF012D787227F0B124CC022CF
:10DC100012D7877870E6D39400401A7F06124CC062
:10DC2000787016E62477F582E43415F583E4F0E69F
:0BDC3000901575F0227F0B124CC022F3
:0BDC3B0012D7877873E6FF124D2022FD
:10DC46007871E675F015A4247CF582E434DEF5835C
:0EDC5600E493740193FA740293F912E7D82252
:10DC6400124A5B7872E675F003A424C1F582E434A9
:10DC7400DEF583E493740193FA740293F912E7D8FE
:10DC84007F0A9015B9E02403FD9015B8E03400FC38
:10DC940012B2DBD39015B9E094009015B8E094006B
:10DCA400400CA3E024FFF09015B8E034FFF012C458
:02DCB400A522A7
:10DCB600124A5B3052287871E675F015A4246DF58A
:10DCC60082E434DEF58308E675F00312E70BE4938D
:0FDCD600740193FA740293F912E7D812C4A522CD
:09DCE5007F0A12B27A12C4A522D2
:10DCEE00901573E024FE604F04705B12C69F505C6B
:10DCFE0012C4A59015C1E030E406124A5B124FAA79
:10DD0E009015BDE030E120124A5B7871E675F01592
:10DD1E00A42476F582E434DEF583E493740193FA59
:10DD2E00740293F912E7D87F027D017C0012B2DBF8
:10DD3E009015737402F02212C69F401090157374E2
:0DDD4E0001F012C4A5229015737401F0229B
:10DD5B0012DCEE12D40812D6F89015CAEFF012D4DA
:10DD6B00109015BAE024FE603A0470489015CAE092
:10DD7B00FFF46046EF75F005A424F5F974DD35F07A
:10DD8B00FA7BFF78727C007D007E007F0512E52C0C
:10DD9B0012DCB67F027D017C0012B2DB9015BA74E7
:10DDAB0002F0229015CAE0B4FF1012DCE59015BA10
:0BDDBB007401F0229015BA7401F022F0
:10DDC6009015747444F0E4A3F07EDC7F4612B664CA
:10DDD6009015BCEFF0E47870F612D7877E007F418D
:0CDDE6007D007B017A15797712EC1B227E
:10DED600D292D29522D292D295227FA212DF4322EB
:10DEE6007FA212DF4E22EFF912DF902212DF3722D5
:10DEF60012DFBE2212DF00E9FF22D29275F008007F
:10DF0600D29500000000A29200C2950033D5F0EF32
:10DF1600F9D29200000000D29500000000C29522BE
:10DF2600D292D29500000000C29200000000C29575
:10DF360022C29200D29500000000D29222EFC2E0E7
:10DF4600F912DF2612DF9022EFD2E0F912DF261255
:10DF5600DF9022EFF912DFAA22EFF912DFB522EFE6
:10DF6600F912DF9022EFF912DF902212DFBEFF22B4
:10DF760012DFEEFF227400F912DF902200D2950024
:10DF8600000000A2920000C2952275F008E93392C3
:10DF96009200D2950000000000C295D5F0F0D29212
:10DFA60012DF8222334007E92480F912DF90223300
:10DFB60040FCE9F912DF9022D29275F00800D29562
:10DFC60000000000A29200000000C2950033D5F0C8
:10DFD600ECF9000000C29200000000D2950000009B
:10DFE60000C295D292E9FF22D29275F00800D2952E
:10DFF60000000000A29200C2950033D5F0EFF900B0
:10E006000000D29200000000D29500000000C295E8
:03E01600E9FF22FD
:03000300C2A8325E
:03000B00C2A93255
:03001300C2AA324C
:03001B0002B574B7
:0300230002B53CE7
:03002B00C2AD2241
:0A00300031393935204D2E532E00D2
:02002E0058D99F
:0100FF0011EF
:071FE000C293FFFF020000A5
:01FFFF000001
:102000007FFF12D1C27F0212D3F27F0012D1D2021F
:10201000FFFF12D1DE227F0012CFEE7F0012D168C7
:1020200012D24412D4087F0212D423431F14531F28
:10203000DF908000E51FF012D410E4F5A875B0FF22
:0D20400075A0FF7580FF7590FF7587022267
:10B53C00C000C001C002C003C004C005C006C007E3
:10B54C00C0D0C0E0C082C083C0F012D3CDD0F0D048
:10B55C0083D082D0E0D0D0D007D006D005D004D094
:10B56C0003D002D001D00032C28E758CE9758A7F6F
:10B57C00D28EC000C001C002C003C004C005C0060A
:10B58C00C007C0D0C0E0C082C083C0F012B4DBD012
:10B59C00F0D083D082D0E0D0D0D007D006D005D068
:0CB5AC0004D003D002D001D000C28F32C6
:10B5B800C2ABC28EC28F53890F438910758DE9754E
:10B5C8008B7FD28ED2AB22EF75F00A84443043F0E1
:10B5D800308D828C83F0A3E5F0F022127D7A220070
:10B5E80012C4F1220012CD542200124FB1220012CF
:04B5F800DD5B2200F5
:10E019009000007A007B007900E493A36AFAE49304
:10E02900A36BFBD9F4E58370F0EA4B60047F0080B1
:04E03900027FFF2241
:1000590022E493A3F8E493A34003F68001F208DFB6
:10006900F48029E493A3F85407240CC8C333C45477
:100079000F4420C8834004F456800146F6DFE4802B
:100089000B010204081020408090204DE47E01936A
:1000990060BEA3FF543F30E509541FFEE493A360FB
:1000A900010ECF54C025E060A840B8E493A3FAE458
:1000B90093A3F8E493A3C8C582C8CAC583CAF0A3A9
:0E00C900C8C582C8CAC583CADFE9DEE780BEAB
:01295700007F
:10E101000000102120423063408450A560C670E7B2
:10E1110081089129A14AB16BC18CD1ADE1CEF1EF5A
:10E12100123102103273225252B5429472F762D602
:10E1310093398318B37BA35AD3BDC39CF3FFE3DEAA
:10E14100246234430420140164E674C744A4548552
:10E15100A56AB54B85289509E5EEF5CFC5ACD58DFA
:10E16100365326721611063076D766F6569546B4A2
:10E17100B75BA77A97198738F7DFE7FED79DC7BC4A
:10E1810048C458E5688678A70840186128023823F2
:10E19100C9CCD9EDE98EF9AF89489969A90AB92B9A
:10E1A1005AF54AD47AB76A961A710A503A332A1242
:10E1B100DBFDCBDCFBBFEB9E9B798B58BB3BAB1AEA
:10E1C1006CA67C874CE45CC52C223C030C601C4192
:10E1D100EDAEFD8FCDECDDCDAD2ABD0B8D689D493A
:10E1E1007E976EB65ED54EF43E132E321E510E70E2
:10E1F100FF9FEFBEDFDDCFFCBF1BAF3A9F598F788A
:10E20100918881A9B1CAA1EBD10CC12DF14EE16F69
:10E21100108000A130C220E35004402570466067A1
:10E2210083B99398A3FBB3DAC33DD31CE37FF35EB9
:10E2310002B1129022F332D24235521462777256F1
:10E24100B5EAA5CB95A88589F56EE54FD52CC50D09
:10E2510034E224C314A00481746664475424440541
:10E26100A7DBB7FA879997B8E75FF77EC71DD73C59
:10E2710026D336F2069116B0665776764615563491
:10E28100D94CC96DF90EE92F99C889E9B98AA9ABA9
:10E29100584448657806682718C008E1388228A3E1
:10E2A100CB7DDB5CEB3FFB1E8BF99BD8ABBBBB9AF9
:10E2B1004A755A546A377A160AF11AD02AB33A9231
:10E2C100FD2EED0FDD6CCD4DBDAAAD8B9DE88DC949
:10E2D1007C266C075C644C453CA22C831CE00CC181
:10E2E100EF1FFF3ECF5DDF7CAF9BBFBA8FD99FF899
:10E2F1006E177E364E555E742E933EB20ED11EF0D1
:10E03D00AB07AA068B828A83E0FFECFEEF6D25E02D
:10E04D00FFEE33FE74012FF582EE34E1F583E49398
:10E05D00FC740193FD8B828A83A3E0FEEC6EFFEDD1
:0EE06D00AC02AD038D828C83CFF0A3EFF022C6
:10E07B009015CBEEF0A3EFF0A3ECF0A3EDF0E49052
:10E08B0015D3F0A3F09015CFF0A3F09015CDE0FED3
:10E09B00A3E0FFA3E0FCA3E0FDC39FEC9E503390F5
:10E0AB0015CBE0FEA3E02DF582EC3EF583E0FF7E81
:10E0BB00009015D1EEF0FCA3EFF0FD7E157FD3128F
:10E0CB00E03D9015D0E004F070069015CFE004F021
:10E0DB0080B99015D3E0FCA3E0FAEC2400FFE43AFE
:02E0EB00FE2213
:10E0ED009015D7E0FEA3E0FF9015D5E0FCA3E0FD71
:04E0FD0012E03D22CE
:10E301009015D9EBF0A3EAF0A3E9F0E412E59BED57
:10E31100644D60097F43E4FDFBFA12C3AA7E007FCE
:10E32100807D007B017A1579DF12EC1B7FA412DF5F
:10E3310043E4FF12DF5F7FA412DF4EE49015DCF0AF
:10E3410012DF719015DCE024DFF582E43415F583EA
:10E35100EFF09015DCE004F0E0D3947E40E212DFB0
:10E36100769015DCE024DFF582E43415F583EFF0D7
:10E3710012DF377FFFE49015DCF09015DCE0FED36F
:10E38100947F502974DF2EF582E43415F583E06023
:10E3910014E4FF9015D9E0FBA3E0FAA3E0F9747E41
:10E3A10012E59B80089015DCE004F080CDEF60035E
:10E3B10002E44790165DE09015DEF090165EE09065
:10E3C10015DDF0E490165DF0A3F07E157FDF7D7E14
:10E3D100FC12E07BEF90165EF0EEFF90165DF09080
:10E3E10015DEE0B507329015DDE0FF90165EE0B571
:10E3F10007269015D9E0FBA3E0FAA3E0F99000010C
:10E4010012E729A801AC02AD037B017A1579DF7E01
:10E41100007F8012E52C803D7B007A007900C003EB
:10E42100C002C0019015D9E0FBA3E0FAA3E0F99086
:10E43100000112E7599015D9E0FBA3E0FAA3E0F936
:10E44100E412E59BFF229015D9E0FBA3E0FAA3E0DB
:08E45100F9E412E59B7F0122B2
:0100FE0022DF
:011FFF0022BF
:01E4590022A0
:01E45A00229F
:01E45B00229E
:10E45C00E709F608DFFA8046E709F208DFFA803EA2
:10E46C0088828C83E709F0A3DFFA8032E309F6088F
:10E47C00DFFA8078E309F208DFFA807088828C83F7
:10E48C00E309F0A3DFFA806489828A83E0A3F608AB
:10E49C00DFFA805889828A83E0A3F208DFFA804C85
:10E4AC0080D280FA80C680D4806980F2803380105C
:10E4BC0080A680EA809A80A880DA80E280CA8033C5
:10E4CC0089828A83ECFAE493A3C8C582C8CCC5833D
:10E4DC00CCF0A3C8C582C8CCC583CCDFE9DEE7800D
:10E4EC000D89828A83E493A3F608DFF9ECFAA9F08C
:10E4FC00EDFB2289828A83ECFAE0A3C8C582C8CCE2
:10E50C00C583CCF0A3C8C582C8CCC583CCDFEADEFA
:10E51C00E880DB89828A83E493A3F208DFF980CC5C
:10E52C0088F0ED2402B4040050C2F582EB2402B44E
:10E53C00040050B823234582F582EF4E60AEEF60A5
:09E54C00010EE5822390E4AC739A
:10E55500BB010689828A83E0225002E722BBFE02C4
:09E56500E32289828A83E49322F7
:10E56E00BB010CE58229F582E5833AF583E0225062
:10E57E0006E92582F8E622BBFE06E92582F8E222AC
:0DE58E00E58229F582E5833AF583E49322C6
:10E59B00BB010689828A83F0225002F722BBFE015F
:02E5AB00F32259
:10E5AD00F8BB010DE58229F582E5833AF583E8F0A4
:10E5BD00225006E92582C8F622BBFE05E92582C850
:02E5CD00F22238
:10E5CF00EFF88DF0A4FFEDC5F0CEA42EFEEC88F091
:04E5DF00A42EFE2246
:10E5E300BC000BBE0029EF8DF084FFADF022E4CC1C
:10E5F300F875F008EF2FFFEE33FEEC33FCEE9DECE5
:10E60300984005FCEE9DFE0FD5F0E9E4CEFD22ED2A
:10E61300F8F5F0EE8420D21CFEADF075F008EF2F74
:10E62300FFED33FD4007985006D5F0F222C398FD65
:05E633000FD5F0EA2202
:10E63800C5F0F8A3E028F0C5F0F8E582158270026D
:06E648001583E038F0220A
:10E64E00A3F8E0C5F025F0F0E5821582700215837F
:06E65E00E0C838F0E822DC
:0DE66400EF2BFFEE3AFEED39FDEC38FC2205
:10E67100E88FF0A4CC8BF0A42CFCE98EF0A42CFC48
:10E681008AF0EDA42CFCEA8EF0A4CDA8F08BF0A4C6
:10E691002DCC3825F0FDE98FF0A42CCD35F0FCEB25
:10E6A1008EF0A4FEA9F0EB8FF0A4CFC5F02ECD39EA
:0FE6B100FEE43CFCEAA42DCE35F0FDE43CFC2257
:10E6C000EB9FF5F0EA9E42F0E99D42F0EC6480C8D1
:06E6D00064809845F02271
:10E6D600EB9FF5F0EA9E42F0E99D42F0E89C45F09A
:01E6E6002211
:0CE6E700E0FCA3E0FDA3E0FEA3E0FF22A6
:0CE6F300E0F8A3E0F9A3E0FAA3E0FB22AA
:0CE6FF00ECF0A3EDF0A3EEF0A3EFF0228E
:0CE70B00A42582F582E5F03583F5832219
:09E71700E0FBA3E0FAA3E0F92203
:09E72000EBF0A3EAF0A3E9F022FA
:10E72900BB010DE58229F582E5833AF58302E717F6
:10E739005007E92582F802ECC0BBFE07E92582F8FB
:10E7490002ED00E58229F582E5833AF58302ED12AF
:10E75900BB0120E58229F582E5833AF583D0F0D023
:10E76900E0F8D0E0F9D0E0FAD0E0FBE8C0E0C0F092
:10E7790002E7205018E92582F8D083D082D0E0F949
:10E78900D0E0FAD0E0FBC082C08302ECC9BBFE181E
:10E79900E92582F8D083D082D0E0F9D0E0FAD0E040
:09E7A900FBC082C08302ED0922CD
:10E7B200D083D082F8E4937012740193700DA3A3F6
:10E7C20093F8740193F5828883E47374029368600A
:06E7D200EFA3A3A380DF0A
:06E7D8008A838982E473CC
:10ED3600E55B2470F582E43416F583E0055B2290EA
:10ED4600166D305A03901670E475F00112ECD2027B
:10ED5600E5552053E97F2ED2538018EF540F2490A7
:10ED6600D43440D4FF30570BEF24BFB41A005003FD
:10ED76002461FFE55C6002155C055FE55F700205D6
:10ED86005E305A0E90166DE475F00112ECD2EF0269
:10ED9600E59B02D6AE7403D25A8003E4C25AF55BF1
:10EDA60090166D12E720E4F55CF55EF55FE55C60B4
:10EDB600077F2012ED7980F5F55DC254C253C25526
:10EDC600C256C258C259C25B12ED45FF700D305A89
:10EDD600057F0012ED8AAF5FAE5E22B42561C2D513
:10EDE600C25712ED45FF24D0B40A00501C75F00A34
:10EDF60020D50DC55CA4255CF55C7002D25680E07A
:10EE0600C55DA4255DF55D80D724CFB41A00EF500B
:10EE160004C2E5D25702EF84D25480C4D25380BED6
:10EE2600D25580BAD2D580B8D25880B27F2012EDA2
:10EE3600792055077401B55C0040F112ED36FF12DA
:10EE4600ED7902EDB3D25BD259809312ED36FB1207
:10EE5600ED36FA12ED36F94A4B700679507AF07BA8
:10EE6600FF205533E55C602FAF5DBF00011F7E00BC
:10EE76008E8275830012E56E60050EEE6F70F1C22C
:10EE8600D5EBC0E0EAC0E0E9C0E0EE12EFC8D0E0A2
:10EE9600F9D0E0FAD0E0FB12E555FF60A5EBC0E043
:10EEA600EAC0E0E9C0E012ED79D0E02401F9D0E053
:10EEB6003400FAD0E0FBE55D60DDD55DDA80837B6A
:10EEC600FF7AEF79C4D2558098791080027908C20A
:10EED60059C25B8008D2D5790A8004790AC2D5E482
:10EEE600FAFDFEFF12ED36FC7B0820541312ED36B8
:10EEF600FD7B1030530A12ED36FE12ED36FF7B20F5
:10EF0600EC3382D592D55013C3E43053069FFFE409
:10EF16009EFEE42054039DFDE49CFCE4CBF8C25421
:10EF2600EC700CCFCECDCCE824F8F870F38017C384
:10EF3600EF33FFEE33FEED33FDEC33FCEB33FB99A1
:10EF46004002FB0FD8E9EB305405F8D0E0C448B2D4
:10EF560054C0E00AEC4D4E4F78207B0070C2EAC0E8
:10EF6600E012EFCAD0F0D0E0205404C4C0E0C4B22E
:10EF760054C0F012ED62D0F0D5F0EB02EDB312E71B
:10EF8600B2EE5153EECF58EE224CEE1E42EED34F68
:10EF9600EEDB44EEDB49EE3743EEE155EEC546EED9
:10EFA600C545EEC547F07350EE262DEE2A2EEE4DE2
:10EFB6002BEE2E23EE4B20F05E2A0000EE453F3F5F
:10EFC6003F00790AA2D5205614305809B910020418
:10EFD60004B9080104A2D52059025001042055663F
:02EFE600925542
:10EFE800B55C005032C0E07F203056177F30A25504
:10EFF80072597258500D12F01FC255C259C2587F2B
:10F0080030800F305803E9C0E012ED79305803D052
:10F01800E0F9D0E0B55CCE3058177F30B9100C124B
:10F02800ED797F583057077F788003B9080312EDD0
:10F03800793055057F2D02ED797F20205BF87F2BF5
:10F048002059F322925580CF286E756C6C29002DBB
:10F0580050434958D25412ED363054F8C254785CB3
:10F0680030D504D253785DF602EDE412ED36240370
:10F07800B405004001E490F0579312ED6A743A1217
:0AF08800ED6AD256755C0402EECF6B
:10F09200E560305F0104F823282498F582E43416F1
:10F0A200F58322901695305F03901698E475F0016F
:10F0B20012ECD202E55560EAC5647002156314C50C
:10F0C20064205F04FF02F81090169574FFF5F002B9
:10F0D200ECE9FF02F818E5616006D561037F0022C2
:10F0E2000564E56470020563205F0302F7FC901675
:10F0F2009512E71712E555FF60A8901695E475F092
:10F102000102ECD212F0E2EFC0E012F0D4D0E04003
:10F11200F380A3D25F8002C25F90169512E720E4CB
:10F12200F562F560F563F564756100C25EC25CC2AA
:10F132005DC26012F0A5FF7005AF627E0022B425A9
:10F142003012F0A5FF24D0B40A00500C75F00AC5A5
:10F1520061A42561F56180E924CFB41A00EF500261
:10F16200C2E502F33CD25D80D8D25C80D4D260800A
:10F17200D0EF12F0D4500512F10680ACEFC0E012CD
:10F18200F0E2D0E06F60A1EF606E12F0B880AA7476
:10F1920001C5616002F56112F0E2EF605B20600E72
:10F1A20012F092E475F00112ECD2EF12E59BD561F8
:10F1B200E62060040560056280C012F0D8EFC0E06E
:10F1C20012F0D4D0E0500412F0B8E4FF20600E1226
:10F1D200F092E475F00112ECD2EF12E59BEF70DAD7
:10F1E200206004056005628091E56160020561129C
:10F1F200F10612F0D8EF70C6305F04E412F0B8E501
:10F2020062600302F13B7EFF7FFF2220601174FFE8
:10F21200FCFDFEFF12F09212E71712EC7505600278
:10F22200F12A7910803FEF12F0B87908803712F195
:10F232000612F0E2EF60C1BF301712F0E2EF60B8E1
:10F24200BF780280DDBF58DE12F10612F0E2EF60F5
:10F25200E4790AEFB42D04D25E8019B42B02801433
:10F2620012F0B8790AE56160020561E9C0E012F1C5
:10F2720006D0E0F9D261E4FCFDFEFFE9C0E0ECC09B
:10F28200E0EDC0E0EEC0E0EFC0E012F0D8EFF8D061
:10F29200E0FFD0E0FED0E0FDD0E0FCD0F0E8604D31
:10F2A200B461004007B47B005002C2E524D0503D57
:10F2B200FA24F6500724F95034240AFAEAB5F00089
:10F2C200502BCFA9F0A42FFF92D5E9C5F0CEA4A26E
:10F2D200D53EFE92D5E9C5F0CDA4A2D53DFD92D58D
:10F2E200E9C5F0CCA4A2D53CFCC261808EE8C0E0A6
:10F2F20020602A2061080562305E0312EC6712F07A
:10F302009212E7170560205C0B205D0DEE8FF01264
:10F31200EC48800912EC758004EF12E59BD0E012F4
:10F32200F0B802F12A20601012F09212E71705607D
:08F33200E5638564F012EC486C
:10F33A0080E812E7B2F1EB53F22458F16B4CF16713
:10F34A0042F16748F22C4FF24A44F19143F23049B4
:10F35A00F26555F20D46F20D45F20D47F16F2AF3AB
:06F36A00274E0000F173C4
:10F37000EFC394414006EFC3945B400CEFC394612C
:0DF380004009EFC3947B5003D38001C322EA
:10F38D00EFC394304009EFC3943A5003D38001C3C7
:01F39D00224D
:10F39E00EFC394414006EFC3945B4018EFC39461F2
:10F3AE004006EFC3947B400CEFC394304009EFC38B
:09F3BE00943A5003D38001C322EC
:10F3C700EFC394204009EFC3947F5003D38001C358
:01F3D7002213
:10F3D800EFC394414006EFC394474018EFC39461CC
:10F3E8004006EFC39467400CEFC394304009EFC365
:09F3F800943A5003D38001C322B2
:10F401009016AAEBF0A3EAF0A3E9F09016B0EBF0A6
:10F41100A3EAF0A3E9F09016AAE0FBA3E475F001DA
:10F4210012E64EA9F0FA12E55570EB9016AB74FF97
:10F43100F5F012E6389016ADE0FBA3E475F0011289
:10F44100E64EA9F0FA12E555FF9016AAE0FBA3E4F7
:10F4510075F00112E64EA9F0FAEF12E59B70D69015
:0BF4610016B0E0FBA3E0FAA3E0F922E4
:10F46C009016B3EBF0A3EAF0A3E9F0E49016BBF02E
:10F47C00A3F0D39016BAE094009016B9E06480948F
:10F48C0080500302F5269016B3E0FBA3E0FAA3E04C
:10F49C00F99016BBE0FEA3E0F5828E8312E56E6058
:10F4AC00109016BCE004F070069016BBE004F080DF
:10F4BC00D59016B6E0FBA3E0FAA3E0F912E555608F
:10F4CC003F9016B6E0A3E475F00112E64EA9F0FAEF
:10F4DC0012E555FF9016B3E0FBA3E0FAA3E0F99018
:10F4EC0016BBE475F00112E64E85F082F583EF123F
:10F4FC00E5AD9016B974FFF5F012E63845F070B131
:10F50C009016B3E0FBA3E0FAA3E0F99016BBE0FE83
:10F51C00A3E0F5828E83E412E5AD9016B3E0FBA375
:06F52C00E0FAA3E0F92261
:10E7DE00E3F5F009E208B5F06D606B80F3E3F5F058
:10E7EE0009E608B5F060605E80F387F009E608B5CB
:10E7FE00F054605280F487F009E208B5F0486046A4
:10E80E0080F488828C8387F009E0A3B5F0386036F7
:10E81E0080F488828C8387F009E493A3B5F0276097
:10E82E002580F388828C83E3F5F009E0A3B5F0161A
:10E83E00601480F388828C83E3F5F009E493A3B52A
:10E84E00F004600280F202E909808580E7808E8004
:10E85E00D2803C8015806C807E809B80B5808B80C2
:10E86E00A1804F8070803A02E91F89828A83ECFA78
:10E87E00E493F5F0A3C8C582C8CCC583CCE493A3BA
:10E88E00C8C582C8CCC583CCB5F070606E80E189F6
:10E89E00828A83E493F5F0A3E208B5F05E605C80B3
:10E8AE00F289828A83E0F5F0A3E608B5F04D604B5D
:10E8BE0080F389828A83E0F5F0A3E208B5F03C602C
:10E8CE003A80F389828A83E493F5F0A3E608B5F0E3
:10E8DE002A602880F2805D89828A83ECFAE493F5BF
:10E8EE00F0A3C8C582C8CCC583CCE0A3C8C582C876
:10E8FE00CCC583CCB5F004600280E27F00F845F011
:10E90E00600EE863F0806480D395F01F40027F01B3
:10E91E002289828A83ECFAE0F5F0A3C8C582C8CCBE
:10E92E00C583CCE0A3C8C582C8CCC583CCB5F0CB1B
:10E93E0060C980E389828A83ECFAE0F5F0A3C8C54A
:10E94E0082C8CCC583CCE493A3C8C582C8CCC5838A
:10E95E00CCB5F0A760A580E288F0ED2402B40400E7
:10E96E005099F582EB2402B40400508F2323458284
:05E97E002390E857732F
:10F532009016BDEBF0A3EAF0A3E9F09016C0E0FB51
:10F54200A3E0FAA3E0F912E555FE9016BDE0FBA395
:10F55200E0FAA3E0F912E555FD6E702AED600E9017
:10F5620016C374FFF5F012E63845F070037F0022EF
:10F572009016BEE475F00112E6389016C1E475F0FB
:10F582000112E63880B5D3EE6480F8ED64809840CD
:07F59200037F01227FFF222D
:10E98300E709F60870FA8046E709F20870FA803E54
:10E9930088828C83E709F0A370FA807EE309F60886
:10E9A30070FA8076E309F20870FA806E88828C83AD
:10E9B300E309F0A370FA806289828A83E0A3F608F0
:10E9C30070FA805689828A83E0A3F20870FA804A3B
:10E9D30080D280FA80C680D4806580F28031801036
:10E9E30080A680EA809A80A880DA80E280CA80319B
:10E9F30089828A83ECFAE493A3C8C582C8CCC58311
:10EA0300CCF0A3C8C582C8CCC583CC70E9800D897E
:10EA1300828A83E493A3F60870F9ECFAA9F0EDFB7C
:10EA23002289828A83ECFAE0A3C8C582C8CCC58355
:10EA3300CCF0A3C8C582C8CCC583CC70EA80DD897D
:10EA4300828A83E493A3F20870F980CE88F0ED24E0
:10EA530002B4040050C4F582EB2402B4040050BA9B
:09EA6300232345822390E9D373BB
:10F599009016C5EBF0A3EAF0A3E9F0E49016CDF0DC
:10F5A900A3F09016CB74FFF5F012E64E45F0603CDF
:10F5B9009016C8E0FBA3E0FAA3E0F912E555FF9025
:10F5C90016C5E0FBA3E0FAA3E0F99016CDE475F0C7
:10F5D9000112E64E85F082F583EF12E5ADEF60C2C8
:10F5E9009016C9E475F00112E63880B69016C5E0A8
:08F5F900FBA3E0FAA3E0F922F4
:10F60100E4FFFE12E555600C0FEF70010E09E97081
:05F61100F20A80EF2267
:10F616009016CFEBF0A3EAF0A3E9F09016CFE0FB4B
:10F62600A3E0FAA3E0F912E555FF12F818500C9082
:10F6360016D0E475F00112E63880E0D2629016CF5B
:10F64600E0FBA3E0FAA3E0F912E555FF642B6004A2
:10F65600EFB42D1D9016CFE0FBA3E475F00112E682
:10F666004EA9F0FA12E555642D6003D38001C392CA
:10F67600629016D212EC8F000000009016CFE0FBCD
:10F68600A3E0FAA3E0F912E555FF12F38D506A7F65
:10F696000A7E007D007C009016D2E0F8A3E0F9A374
:10F6A600E0FAA3E0FB12E671C8ECC8EDC0E0EEC0DC
:10F6B600E0EFC0E09016CFE0FBA3E0FAA3E0F9127A
:10F6C600E555FF3395E0FEEF24D0FFEE34FFFEE470
:10F6D600FCFDD0E0FBD0E0FAD0E0F9EB2FFFEA3EEC
:10F6E600FEED39FDEC38FC9016D212E6FF9016D0EE
:10F6F600E475F00112E63880823062109016D2E08E
:10F70600FCA3E0FDA3E0FEA3E0FF80119016D2E08B
:0EF71600FCA3E0FDA3E0FEA3E0FF12EC6722DF
:10F724009016D6EBF0A3EAF0A3E9F09016D6E0FB2E
:10F73400A3E0FAA3E0F912E555FF12F818500C9073
:10F7440016D7E475F00112E63880E0D2639016D63D
:10F75400E0FBA3E0FAA3E0F912E555FF642B600493
:10F76400EFB42D1D9016D6E0FBA3E475F00112E66C
:10F774004EA9F0FA12E555642D6003D38001C392BB
:10F7840063E49016D9F0A3F09016D6E0FBA3E0FA58
:10F79400A3E0F912E555FF12F38D503F9016D6E021
:10F7A400FBA3E0FAA3E0F912E555FF3395E0FEEF81
:10F7B40024D0FBEE34FFFA9016D9E0FEA3E0FF7CE0
:10F7C400007D0A12E5CFEF2BF0EE3A9016D9F090B7
:10F7D40016D7E475F00112E63880AD30630A90164E
:10F7E400D9E0FEA3E0FF800F9016D9E0FEA3E0FF6E
:08F7F400C3E49FFFE49EFE2226
:10EA6C00E3F5F009E208B5F06BDFF58067E3F5F04C
:10EA7C0009E608B5F05EDFF5805A87F009E608B5BF
:10EA8C00F052DFF6804E87F009E208B5F046DFF66B
:10EA9C00804288828C8387F009E0A3B5F036DFF6DC
:10EAAC00803288828C8387F009E493A3B5F025DF4C
:10EABC00F5802188828C83E3F5F009E0A3B5F0148E
:10EACC00DFF5801088828C83E3F5F009E493A3B51D
:10EADC00F002DFF402EB9B808780E9809080D48089
:10EAEC003E8015806E807E809D80B7808D80A38057
:10EAFC00518074803C02EBA789828A83ECFAE49300
:10EB0C00F5F0A3C8C582C8CCC583CCE493A3C8C513
:10EB1C0082C8CCC583CCB5F076DFE3DEE1807089AA
:10EB2C00828A83E493F5F0A3E208B5F062DFF48007
:10EB3C005E89828A83E0F5F0A3E608B5F051DFF533
:10EB4C00804D89828A83E0F5F0A3E208B5F040DFBE
:10EB5C00F5803C89828A83E493F5F0A3E608B5F04E
:10EB6C002EDFF4802A8002805789828A83ECFAE4B3
:10EB7C0093F5F0A3C8C582C8CCC583CCE0A3C8C5A7
:10EB8C0082C8CCC583CCB5F006DFE4DEE280007F22
:10EB9C00FFB5F0020F2240027F012289828A83ECAA
:10EBAC00FAE0F5F0A3C8C582C8CCC583CCE0A3C8F5
:10EBBC00C582C8CCC583CCB5F0D5DFE5DEE380CF0C
:10EBCC0089828A83ECFAE0F5F0A3C8C582C8CCC56B
:10EBDC0083CCE493A3C8C582C8CCC583CCB5F0AFB5
:10EBEC00DFE4DEE280A988F0ED2402B40400509F3B
:10EBFC00F582EB2402B40400509523234582F58260
:0FEC0C00EF4E6096EF60010EE5822390EAE3730E
:10EC1B00EF4E6013EDBB011089828A83EF60010E0A
:10EC2B00EDF0A3DFFCDEFA2289F05007F709DFFCD9
:0DEC3B00A9F022BBFE06F309DF02A9F022BA
:10EC4800BB010A89828A83F0E5F0A3F0225006F717
:0FEC580009A7F01922BBFE06F3E5F009F3192214
:0EEC6700C3E49FFFE49EFEE49DFDE49CFC22BE
:10EC7500BB010789828A8302E6FF5005E9F802EDA8
:0AEC85001EBBFE05E9F802ED2A228D
:10EC8F00A8828583F0D083D08212ECA612ECA61254
:10EC9F00ECA612ECA6E473E493A3C583C5F0C58379
:10ECAF00C8C582C8F0A3C583C5F0C583C8C582C8CF
:01ECBF002232
:09ECC000E6FB08E6FA08E6F92279
:09ECC900EBF608EAF608E9F62270
:10ECD200F8E0FBA3A3E0F925F0F0E58215827002CB
:07ECE2001583E0FA38F0226F
:10ECE900F8E0FBA3A3E025F0F9F0E58215827002B4
:07ECF9001583E038FAF02258
:09ED0000E2FB08E2FA08E2F92244
:09ED0900EBF208EAF208E9F2223B
:0CED1200E493FB740193FA740293F9225D
:10F7FC0010640B12F82DBF0D027F0A02D6AE9016C4
:04F80C00DBE0FF221C
:08F810009016DBEFF0D2642238
:10F81800EFC394094006EFC3940E4004EFB42003ED
:05F82800D38001C322A2
:0CED1E00ECF608EDF608EEF608EFF62221
:0CED2A00ECF208EDF208EEF208EFF22225
:0AF82D003098FDAF99C2987E0022CA
:00000001FF
